:020000040800F2
:1000000000040020B9010008BB010008BB01000882
:10001000BB010008BB010008BB010008BB010008D0
:10002000BB010008BB010008BB01000881BC00083F
:10003000BB010008BB010008BB010008B9CE0008E5
:10004000BB010008BB010008BB010008BB010008A0
:10005000BB010008BB010008C9300008F5300008EA
:10006000213100084D31000879310008BB0100083A
:10007000BB010008BB010008F5D40008BB01000863
:10008000A5310008BB010008BB010008BB01000846
:10009000BB010008BB010008BB010008BB01000850
:1000A000BB010008BB010008A9D00008BB01000883
:1000B000BB010008BB010008D9CE0008BB01000845
:1000C000BB01000831320008BB010008BB01000879
:1000D000BB010008BB010008BB010008BB01000810
:1000E00072B6264880F30888254880F30988254899
:1000F00025490860022080F31488BFF36F8F0BF04E
:1001000037FB0BF011F94FF0553020491B4A914253
:100110003CBF41F8040BFAE71D49194A91423CBF24
:1001200041F8040BFAE71B491B4A1C4B9A423EBF9D
:1001300051F8040B42F8040BF8E700201849194A5B
:1001400091423CBF41F8040BFAE70BF015FB0BF0B2
:1001500010FB154C154DAC4203DA54F8041B8847CC
:10016000F9E705F0EBFF124C124DAC4203DA54F8FC
:10017000041B8847F9E70BF0FDBA000000040020DB
:10018000000C00200000000808ED00E00000002046
:10019000000400206CF20008000C00204011002038
:1001A0004011002094330020E0000008E000000827
:1001B000E0000008E000000892E700F000F8FEE729
:1001C0002DE9F04FC1F80CD0C3689D46BDE8F08F13
:1001D000002383F311882846A04700200BF0D0FCB1
:1001E000FEE70BF003FC00DFFEE7000053B94AB95D
:1001F000002908BF00281CBF4FF0FF314FF0FF302F
:1002000000F074B9ADF1080C6DE904CE00F006F809
:10021000DDF804E0DDE9022304B070472DE9F04782
:100220008C460446089E002B40F086808A42154684
:1002300048D9B2FA82F24AB1C2F1200701FA02F3B8
:1002400020FA07F7954047EA030C94404FEA154E11
:10025000BCFBFEF71FFA85F80EFB17C307FB08F976
:10026000210C41EA0343994509D9EB1807F1FF3105
:1002700080F0E180994540F2DE80023F2B44A3EB01
:100280000903B3FBFEF00EFB103300FB08F1A4B230
:1002900044EA0344A14209D92C1900F1FF3380F04C
:1002A000C880A14240F2C58002382C4440EA074091
:1002B0000027641A1EB10023D440C6E90043394622
:1002C000BDE8F087002A54D0B2FA82F2002A40F04A
:1002D000B4800127491B4FEA15481FFA85F9B1FB85
:1002E000F8FE08FB1E1109FB0EF04FEA144C4CEA15
:1002F0000143984207D9EB180EF1FF3102D2984220
:1003000000F2EB808E461B1AB3FBF8F008FB1033AB
:1003100009FB00F9A4B244EA0344A14507D92C190A
:1003200000F1FF3302D2A14500F2DB801846A4EBB6
:10033000090440EA0E40BDE78B4208D9002E75D073
:100340000027C6E9000138463946BDE8F087B3FA10
:1003500083F77FB98B4202D3824200F2BC80841AB9
:1003600061EB030301209C46002EA8D0C6E9004C97
:10037000A5E7FFDEC7F12005BB4022FA05FC4CEAE9
:10038000030C21FA05F44FEA1C4EB4FBFEF91FFAE8
:100390008CF80EFB194420FA05F3B94009FB08FA62
:1003A00019430B0C43EA0444A24502FA07F200FA8F
:1003B00007F30BD91CEB040409F1FF3080F08980AE
:1003C000A24540F28680A9F102096444A4EB0A0424
:1003D000B4FBFEF00EFB104400FB08FA89B241EAC0
:1003E0000444A24508D91CEB040400F1FF316CD28F
:1003F000A2456AD90238644440EA0940A0FB028958
:10040000A4EB0A044C454146CE4655D352D0002EAB
:100410006AD05A1A64EB0E0404FA05F522FA07F3BF
:10042000FC401D43C6E90054002748E737463046E4
:1004300045E718463AE70F4621E79540C2F1200309
:1004400021FA03F04FEA1548B0FBF8F71FFA85F9D7
:1004500008FB170E24FA03FC914007FB09FA4CEA4B
:100460000101080C40EA0E40824504FA02F407D963
:10047000281807F1FF332AD2824528D9023F2844A1
:10048000A0EB0A00B0FBF8FC08FB1C000CFB09F316
:1004900089B241EA00418B4208D969180CF1FF305A
:1004A00011D28B420FD9ACF1020C2944C91A4CEA83
:1004B000074714E74345AAD2B8EB020169EB0C02E7
:1004C00001389646A3E78446F0E7084694E71F46BE
:1004D000D6E781467AE7384646E7AEF1020E2B446E
:1004E00011E702382C4422E73746E8E6704700BFA0
:1004F00008B5062000F0FAF901200CF005FB00BF5A
:10050000032A70B412D940EA0105AD0704460B4630
:1005100020D11946204653F8045B54F8046BAE42D0
:1005200018D1043A032A20461946F2D8541E72B153
:1005300003780A789A4208BF241806D00CE010F815
:10054000013F11F8012F934206D1A042F7D10020BC
:1005500070BC7047541EEBE7981A70BC704700BF20
:10056000844641EA000313F0030349D1403A23D300
:100570000B6803604B6843608B688360CB68C36023
:100580000B6903614B6943618B698361CB69C3610B
:100590000B6A03624B6A43628B6A8362CB6AC362F3
:1005A0000B6B03634B6B43638B6B8363CB6BC363DB
:1005B00040304031403ADBD230320BD30B6803601D
:1005C0004B6843608B688360CB68C3601030103128
:1005D000103AF3D20C3205D351F8043B40F8043BF7
:1005E000043AF9D2043208D0D2071CBF11F8013BFB
:1005F00000F8013B01D30B8803806046704700BFC1
:10060000082A13D38B07B1D010F00303AED0C3F187
:100610000403D21ADB071CBF11F8013B00F8013BB1
:10062000A4D331F8023B20F8023B9FE7043AD9D328
:10063000013A11F8013B00F8013BF9D20B78037045
:100640004B7843708B78837060467047F0B48607B0
:1006500046D0541E002A3CD0CAB2034602E014F130
:10066000FF3436D303F8012B9D07F8D1032C29D989
:10067000CDB245EA05250F2C45EA054533D9A4F14D
:100680001006360903F1200707EB061703F11002E5
:1006900042E9045542E902551032BA42F8D1721CBF
:1006A00014F00C0F03EB021204F00F0613D0331FEB
:1006B00023F003030433134442F8045B9342FBD159
:1006C00006F003042CB1C9B21C4403F8011B9C4280
:1006D000FBD1F0BC704734461346002CF3D1F8E749
:1006E00014460346C2E71A462646E0E738B5124BE1
:1006F00005461C68A06B18B10023C0E9045338BD3F
:10070000182000F0A1F9A06378B101220023C0E90C
:1007100004230A4B0B24836000230949094A84817E
:10072000C0E90012C0E9045338BD0246064B42211D
:10073000064800F041F900BF000C0020ECDE050087
:100740000E33CDAB34126DE69CF10008B4F1000815
:1007500038B51A4B1C68A26B92B1146918495369D9
:1007600001FB04F1174800FB0313A4FB0045611CC7
:100770001D4445F1000323F00040C2E9041338BDD5
:10078000182000F061F90246A06388B10124002519
:100790000B21C0E904450C4B0948136003460B4D7F
:1007A0000B4C91810B49C2E90154C2E9041338BDD5
:1007B000094B4E21094800F0FFF800BF000C002053
:1007C0002DF451582D7F954C0E33CDAB34126DE680
:1007D000ECDE05002E7F954C9CF10008B4F100087A
:1007E00010B58021044600F093F9606440B1002206
:1007F000031F7C3043F8042F8342FBD1002010BD3F
:100800004FF0FF3010BD00BF436C0BB100207047AC
:10081000E6E700BF1F2970B5054608D8436C1646A9
:100820000C464BB153F8240043F8246070BD1622E7
:100830004FF0FF302A6070BDFFF7D2FF08B96B6C34
:10084000F0E74FF0FF3070BD1F2938B5054620D8BE
:10085000426C0C466AB152F8213053B1012B16D0CC
:10086000591C10D00025204642F8245098472846AD
:1008700038BD284600F070F8224601462846BDE8FB
:10088000384000F055B8162301202B6038BD0020F9
:1008900038BD16234FF0FF302B6038BD1F2921D8FB
:1008A00038B5436C05460C4683B153F8242003EB5E
:1008B00084034AB1511C10D0012A0CD000252046D7
:1008C0001D609047284638BD012038BDFFF788FFDE
:1008D00028B96B6CE9E7032038BD022038BD4FF022
:1008E000FF3038BD4FF0FF30704700BF024B01466C
:1008F0001868FFF7A9BF00BF000C0020024B0A4692
:1009000001461868FFF786BF000C0020034B1868EB
:10091000436C0BB10020704762E700BF000C002061
:10092000024B01461868FFF7B9BF00BF000C00205A
:1009300070B50D460023074C064611462846236035
:100940000CF0EAF8431C00D070BD2368002BFBD0EC
:10095000336070BD6C3300200CF0E6B820F003016A
:1009600010F00300C0F1000051F8043B00F1040C4A
:100970004FEACC0C6FF000021CBF22FA0CF21343BA
:100980004FF0010C4CEA0C2C4CEA0C4CA3EB0C0283
:1009900022EA030212EACC1204BF51F8043B0430ED
:1009A000F4D0C2F1000102EA0102B2FA82F2C2F10D
:1009B0001F0200EBD200704700B50A4C05462068C4
:1009C00085B01C46C06852B1074BCDE90132009199
:1009D0002B462246054900F023F8FFF789FD044B1A
:1009E0001A46F2E7000C0020E8F10008F8F10008D0
:1009F000F4F1000808B513460022FFF7DDFF00BF41
:100A00000CB410B582B004AC54F8042B2346019406
:100A100000F024F902B0BDE8104002B0704700BFFA
:100A20000EB430B582B005AC54F8042B054D014628
:100A300023462868019400F011F902B0BDE8304067
:100A400003B07047000C0020024B0146186800F00C
:100A50005FB800BF000C0020024B0146186800F090
:100A600003B800BF000C002000293AD038B551F877
:100A7000043C0C1F002BB8BFE418054601F088FAAF
:100A8000224B1A682AB1A2420DD92168601882420D
:100A900021D0626028461C60BDE8384001F07EBA73
:100AA000A34203D81A465368002BF9D11168501895
:100AB000A04217D022D821686018834203BFD3E92F
:100AC00000030918C4E90013636054602846BDE8B8
:100AD000384001F063BAD2E900020144C4E90012CF
:100AE000D8E7704720680144501883421160EDD167
:100AF000D3E900030144C2E90013E7E70C232846C9
:100B00002B60BDE8384001F049BA00BF4011002019
:100B1000F8B5CD1C25F0030508350C2D38BF0C2584
:100B2000002D064633DBA94231D82A4F01F030FAB6
:100B30003A6852B113685B1B04D43FE023685B1B27
:100B400029D522465468002CF8D1796800293BD079
:100B5000294630460BF0BCFF431C28D0C41C24F0AF
:100B60000304A04205D0211A30460BF0B1FF01303A
:100B70001DD02560304601F011FA04F10B0020F081
:100B80000700231DC21A01D01B1AA350F8BD0C2266
:100B900000203260F8BD0B2B05D8A242636811D04B
:100BA0005360E7E7144623601C442560E2E70C230A
:100BB0003046336001F0F2F90020F8BD0B2BF1D87C
:100BC000144653683B60D5E730460BF081FF7860F0
:100BD000BEE700BF401100209368013B002B9360EB
:100BE0000FDA10B49469A34208DB0A2906D013680F
:100BF000581C10601970084610BC704710BC00F0FB
:100C00009FBB1368581C106019700846704700BFDE
:100C10009BB1F8B513440F4606465D1E541E01E015
:100C2000AC4208D03A4614F8011F3046FFF7D4FF13
:100C3000431CF5D1F8BD0020F8BD0020704700BF6F
:100C4000936810B5144613B95360184610BD00F0F0
:100C50009BFE0023C4E9013310BD00BF2DE9F04F16
:100C60009FB08B4690461C46039018B18369002BB9
:100C700000F0C880AE4B9B4500F0CA80AD4B9B4551
:100C800000F0CA80AC4B9B4504BF039BD3F80CB06B
:100C9000DBF86430BBF80C20DB0702D4970540F189
:100CA0005781160740F12B81DBF81030002B00F044
:100CB000268100202021302298F800300127059459
:100CC0000B908DF831109D4E8DF83220002B00F0E6
:100CD0008880252B00F01181454603E0252B00F08C
:100CE0009F8025466B786C1C002BF7D1B4EB080A6B
:100CF00077D04246534659460398FFF789FF0130A3
:100D00006FD00B9B6A7853440B93002A69D0002361
:100D10004FF0FF3201340693CDE908338DF85B3094
:100D20001C93079206E02C46069B801B07FA00F0F6
:100D3000184306902546052215F8011B304601F0A0
:100D40007BF8AA460028EED1069BD80644BF202295
:100D50008DF85B20190748BF2B22217848BF8DF8FA
:100D60005B202A2961D1059A116804320029059275
:100D7000C0F2988009916178A51C2E296ED0704C24
:100D80000322204601F058F8002800F0818040221C
:100D9000069B001B02FA00F00343069305F10108CD
:100DA0002B780622194667488DF8303001F044F858
:100DB00000287DD0644B002B6DD005AB00935A46C4
:100DC000624B06A90398AFF300808146B9F1FF3F5B
:100DD00007D00B9B4B440B9398F80030002B7FF40B
:100DE00078AFDBF8643013F0010FBBF80C3002D1A0
:100DF0009A0540F1B4805B0600F194800B981FB017
:100E0000BDE8F08F00F0A8FC494B9B457FF436AF5E
:100E1000039BD3F804B03BE7039BD3F808B037E754
:100E2000B4EB080A3FF473AF63E7A1F13002092A7B
:100E300088BFA246A1D8099B01E02C46013529783C
:100E400003EB830302EB4303A1F13002092AAA4614
:100E5000F3D92E2904F10205099390D19AF80110D3
:100E60002A292FD1059B0AF102001A680433002AAF
:100E7000079205939AF802100AF1030538DB304C0B
:100E800082460322204600F0D7FF00287FF47FAF80
:100E9000A846554684E7059B073323F0070308332C
:100EA000059396E7494243F002030991069362E7EE
:100EB00005AB00935A46254B06A9039800F0F6F8B7
:100EC000814683E70023A1F13002092A079301D963
:100ED0002BE05546697803EB830302EB4303A1F152
:100EE0003002092A05F1010AF3D90235079346E7D2
:100EF0004FF0FF338246079341E7444607E75946E0
:100F0000039800F07DFA00283FF4D3AEDBF864309C
:100F1000DD0707D4BBF80C309C0503D4DBF8580080
:100F200000F010FF4FF0FF3069E7AA46013526E7D1
:100F3000E4E50008C4E50008A4E5000828F200087C
:100F400030F2000834F2000800000000110C000824
:100F5000DBF8580000F0EEFEBBF80C20A1E6DBF851
:100F6000580000F0EFFEBBF80C3044E710B4044C1E
:100F700013460A460146206810BCFFF76FBE00BF4B
:100F8000000C00202DE9F0470C460969A568914640
:100F90008D42B8BF0D46156094F8431006461F46B3
:100FA000DDF8208011B16A1CC9F800202368990679
:100FB0005CD5D9F800200232C9F80020236813F06C
:100FC000060F19461DD1E1688A1A002AD8BF1946B2
:100FD00017DD002504F1190A05E0E368D9F80020BF
:100FE0009B1AAB420CDD0123524639463046C047BE
:100FF000013005F10105F0D14FF0FF30BDE8F08779
:10100000216894F84330003318BF01238A060AD5BB
:101010003021E21882F8431094F845105A1C2244FB
:1010200082F84310023304F1430239463046C04788
:101030000130E1D02368A26803F00603042B216984
:101040001DD08A4226DD4FF00009521A9144002536
:101050001A3401E04D451DDA012322463946304657
:10106000C047013005F10105F4D1C5E713F0060FC3
:1010700013D094F84330003318BF0123D3E7D9F8D5
:101080000000E3688A42A3EB000323EAE379DCDC97
:10109000002BDCDC0020BDE8F087E168D9F80020F7
:1010A0008A1A002AD8BF194693DCAAE72DE9F04333
:1010B0000C46097E85B06E2906461746984604F10F
:1010C000430C0C986DD039D9732900F0F48044D9C1
:1010D000752900F00281782940F00F817823226879
:1010E000DFF854E284F845300168150651F8043BF6
:1010F000016040F1A180D10744BF42F0200222608C
:10110000002B00F093801022002184F843106068C7
:101110000028A060C0F2C680216821F0040121608F
:10112000002B40F0A280002840F0BE806546082ACF
:1011300000F0AB80ACEB0503236141E0632900F0D4
:10114000E3801AD8002938D0582940F0D68084F896
:1011500045102268DFF8E4E1C6E76F2900F0BD80A2
:10116000702940F0CA8078232268DFF8CCE142F091
:101170002002226084F84530B6E7642902D069294C
:1011800040F0BB8022680368110603F1040557D5BF
:10119000196805600B46002959DB0A22DFF89CE13B
:1011A000B5E7036822681D1D6169056015061B68A7
:1011B00002D4500600F1BB8019600023654623610C
:1011C000CDF800803B4603AA21463046FFF7DAFE01
:1011D000013020D02A46236939463046C0470130C5
:1011E00019D0226803989207E36819D51A1A002AC1
:1011F00016DD002504F1190904E0E36803981A1AC2
:10120000AA420DDD01234A4639463046C047013027
:1012100005F10105F1D14FF0FF3005B0BDE8F083D5
:101220009842B8BF184605B0BDE8F0832168102287
:1012300021F02001216067E7500648BF9BB25AE7C2
:101240005106A5D5B3F9003005601946A3E72D2056
:1012500061685B42002984F84300A16002DB22F050
:10126000040222600A22DFF8D4E0654600E00B4663
:10127000B3FBF2F102FB11301EF80000934205F8B7
:10128000010DF4D2082A7FF455AF2368DB077FF500
:1012900051AF626823699A423FF74CAF3023013D5A
:1012A0002B7047E7002BE0D19EF8003004F1420597
:1012B00084F842303BE703686268191D01601D68CD
:1012C0000021284600F0B8FD002832D0401B6060A5
:1012D0002061002384F8433072E72268036812F02B
:1012E000800F03F104051AD01B6805606F290CBF3D
:1012F00008220A22DFF844E006E7012384F84210BE
:10130000236104F14205E4E70122036804F1420588
:10131000191D1B68016084F842302261D9E712F080
:10132000400F0DBF1B6805601B880560DEE7198054
:1013300043E76068CCE700BF50F200083CF20008C9
:10134000F8B50D461446064608B1836943B3254BEC
:101350009C422AD0244B9C4229D0244B9C4208BF5B
:10136000F468A269A389A2601A0722D5236903B38E
:1013700022686169D31AEDB299422F4629DD013303
:10138000A168501C0139A1602060157062699A4201
:1013900016D0A389DB0701D50A2D11D03846F8BD38
:1013A00000F0DAF90F4B9C42D4D17468D9E7B468E5
:1013B000D7E72146304600F023F838B92369D7E74C
:1013C0002146304600F032F90028E7D04FF0FF37D1
:1013D000E4E72146304600F029F90028F6D1012340
:1013E0002268CDE7E4E50008C4E50008A4E50008AC
:1013F000024B0A4601461868FFF7A2BF000C002006
:101400003B4B70B51D6806460C460DB1AB69DBB1B0
:10141000384B9C421ED0384B9C424AD0374B9C42A2
:1014200008BFEC68B4F90C2093B2190718D52069ED
:1014300008B313F001022CD000226369A2605B4262
:10144000A36160B3002070BD284600F085F9294BE8
:101450009C42E0D16C68B4F90C2093B21907E6D431
:10146000DD063CD5580726D4206942F00803A38145
:101470009BB20028DDD103F42072B2F5007FD8D0F2
:101480003046214600F08EFCA389206913F001024A
:10149000D2D1990758BF6269A2600028D2D1B4F9AD
:1014A0000C301A06CFD543F04003A3814FF0FF3034
:1014B00070BDAC68B6E7616B51B104F14403994269
:1014C00004D03046FFF7D0FAB4F90C200023636350
:1014D0000023206922F02402C4E90003C5E70923A0
:1014E00042F0400233604FF0FF30A28170BD00BF78
:1014F000000C0020E4E50008C4E50008A4E50008AD
:101500002DE9F0418F890C463A07804641D44B685B
:10151000002B59DDE66A002E53D0002317F48052C9
:10152000D8F80050216AC8F8003051D10123404654
:10153000B047431C5FD0A789E66A216A7F0705D5BB
:101540006268636B801A0BB1236CC01A02460023D9
:101550004046B047461C45D1D8F80030B4F90C20BD
:10156000002B55D01D2B01D0162B5AD100222369F8
:10157000C4E90032616BC8F8005011B304F14403B0
:10158000994202D04046FFF76FFA00206063BDE841
:10159000F0810E69AEB10D680E60B90714BF00236B
:1015A0006369AD1BA3600AE02B463246A76A216A35
:1015B0004046B8470028A5EB000506440ADD002D8B
:1015C000F2DC0020BDE8F0810B6C002BA2DCF8E718
:1015D000606DB3E7A3894FF0FF3043F04003A38170
:1015E000BDE8F081002322696360A3892260DA04E8
:1015F000C0D56065BEE7D8F80030002B9BD01D2B0E
:101600000CD0162B0AD0A38943F04003A381D9E75D
:101610002169C4E90013D304ACD5EAE7C8F8005047
:10162000CFE742F04002A281CCE700BF38B50B699A
:101630001BB30C46054608B183691BB3184B9C428B
:101640001ED0184B9C4220D0174B9C4208BFEC6820
:10165000B4F90C308BB1626ED00701D4990516D560
:1016600028462146FFF74CFF636E0546DA0702D491
:10167000A3899B050FD5284638BD0025284638BDCF
:101680006C68E5E700F068F8D8E7AC68E0E7A06DC3
:1016900000F050FBE4E7A06D00F054FBEBE700BF67
:1016A000E4E50008C4E50008A4E5000820B1054B06
:1016B00001461868FFF7BABF034B0449186800F0E9
:1016C00007BB00BF000C0020A0E500082D16000895
:1016D000014900F0FDBA00BF2D16000808B5436EA1
:1016E000DA0702D483899B0501D5002008BD806DEF
:1016F00000F020FB002008BD08B5436EDA0702D4D5
:1017000083899B0501D5002008BD806D00F01AFB80
:10171000002008BD70B568254A1E05FB02F50E467F
:1017200005F17401FFF7F4F9044640B100210C30D3
:10173000666005F168022160A060FEF787FF204621
:1017400070BD00BF024B0349186800F0C1BA00BF6A
:10175000A0E500082D1600082DE9F84F05463A4887
:1017600000F0E8FAAB69002B69D1384AC5E91233B9
:1017700012682B65AA4208BF0123354908BFAB6137
:10178000A962284600F072F86860284600F06EF8FA
:10179000A8602846002400F069F804236E68E86019
:1017A00021467466C6E90044B460C6E90444B461E5
:1017B000F36006F15C000822FEF748FFDFF89CB0FA
:1017C000AF68DFF89CA0DFF89C90DFF89C80214B8D
:1017D000C6E9086BC6E90AA9C6F830802146FB6055
:1017E0007C66C7E90044BC60C7E90444BC6107F1FA
:1017F0005C000822FEF72AFFEE68174BC7E9087B5A
:10180000C7E90AA9C7F830802146F3607466C6E9C3
:101810000044B460C6E90444B46106F15C000822E7
:10182000FEF714FF0123C6E9086BC6E90AA9C6F84A
:1018300030800548AB61BDE8F84F00F083BA02483C
:10184000BDE8F84F00F07EBA7C330020A0E5000828
:10185000D11600080900010012000200F51F00085F
:101860001D2000085D2000087D20000870B5064698
:10187000244800F05FFA244B1D68AB697BB3483500
:10188000D5E90134013B05D525E0013B5A1C04F1A3
:10189000680420D0B4F90C20002AF6D100251B4B97
:1018A00004F15800E360656600F03CFA154800F06A
:1018B00049FA2560C4E90155C4E90455A5612946E2
:1018C000082204F15C00FEF7C1FEC4E90D55C4E92D
:1018D0001255204670BD2C682CB12546D0E728460D
:1018E000FFF73AFFCBE704213046FFF713FF04462A
:1018F00028600028F1D1034800F024FA0C2333605B
:10190000E7E700BF90330020A0E500080100FFFFDB
:10191000014800F00FBA00BF90330020014800F0EA
:1019200011BA00BF90330020014800F003BA00BF95
:101930007C330020014800F005BA00BF7C33002052
:1019400008B5054800F0F6F9044B05491868BDE8EC
:10195000084000F099B900BF90330020000C00202F
:10196000DD16000808B5054B0549186800F08CF92C
:10197000BDE80840034800F0E5B900BF000C0020B6
:10198000F9160008903300209368002B00F0FC80CB
:101990002DE9F04FB1F90C300C469BB2190783B01A
:1019A000824690462BD522694AB313F00202D8F83A
:1019B000006033D000273D46D4F828B0216ADFF814
:1019C000C492C5B14D452B463A4628BF4B465046BA
:1019D000D847002840F3CE80D8F8083007441B1AB7
:1019E0002D1AC8F80830002B00F0B380D4F828B0C6
:1019F000216A002DE6D1D6E900750836E1E72146D7
:101A00005046FFF7FDFC002840F03781B4F90C3058
:101A1000D8F800609BB213F00202CBD113F0010999
:101A200040F0B4804D46A7682068002D55D09A0537
:101A300040F1C080AF42BB4600F2EE8013F4906FDD
:101A40002FD0D4E9041707EB4707A0EB010B07EBF6
:101A5000D777681C7F105844B8423A4684BF07467F
:101A60003A465B0540F1F08011465046FFF750F8CA
:101A7000002800F0FC805A4621690190FEF770FDB5
:101A8000A289019B22F4906242F08002A281A7EB1E
:101A90000B0203EB0B006761AB462F46236120600E
:101AA000A2605A46494600F00DFA2368A2685B44DA
:101AB000AB460025D71BA7602360D8F80870D9442F
:101AC000A7EB0B07C8F80870002F42D0B4F90C3010
:101AD000A7689BB22068002DA9D1D6E900950836E9
:101AE000A3E70BF1080353F8047C9B4653F8086CFA
:101AF0000833002FF7D03A460A21304600F09CF90F
:101B0000002854D00130A0EB06094B46206821691B
:101B1000BB4228BF3B468842626903D9A568154489
:101B2000AB421ADC9A4200F381801346A56A324622
:101B3000216A5046A847051E1CDDB9EB05096ED089
:101B40000120D8F808302E445B1B7F1BC8F80830F2
:101B500013BB002003B0BDE8F08F31462A4600F0E9
:101B6000B1F9236821462B4423605046FFF75EFD00
:101B70000028E2D0B4F90C304FF0FF3043F04003BE
:101B8000A38103B0BDE8F08F002070473346914633
:101B9000104617464E469B46002FA2D00028B4D1CF
:101BA0003A460A21304600F047F90028AAD17B1CAA
:101BB0009946ABE72369834217D36269AA4214D8D6
:101BC0002F4BA76A9D4294BF2B466FF0004393FBB7
:101BD000F2F3216A02FB03F350464A46B847B0F1DC
:101BE000000BC7DDA5EB0B0567E7AF4228BF2F460B
:101BF00049463A4600F066F9A3682268DB1B3A447E
:101C0000BB46A3602260002BECD121465046FFF773
:101C10000DFD0028E6D0ADE72F46AB4641E7214653
:101C20005046FFF703FD00288BD0A3E71A46314644
:101C30001D46019300F046F9A1682268019BC91A6C
:101C40001344A160236078E7504600F0ADF90346E5
:101C500000287FF41CAF21695046FEF705FF0C22D7
:101C6000B4F90C30CAF8002023F0800384E70C227A
:101C7000B4F90C30CAF800207EE74FF0FF3069E776
:101C8000FEFFFF7F00FCFF7F2DE9F04110F14807C8
:101C90001AD088460026D7E90154013D0ED4A38905
:101CA000013D012B06D9B4F90E30013302D0204694
:101CB000C04706436B1C04F16804F0D13F68002F55
:101CC000E9D13046BDE8F0813E463046BDE8F081BE
:101CD0002DE9F84310F148061ED0884607464FF01C
:101CE0000009D6E90154013D10D4A389013D012B1F
:101CF00008D9B4F90E30013304D021463846C04724
:101D000049EA00096B1C04F16804EED13668002E24
:101D1000E7D14846BDE8F883B1464846BDE8F883B8
:101D2000704700BF704700BF704700BF704700BFDB
:101D3000704700BF704700BF012070470120704707
:101D4000704700BF704700BF70B50C46B1F90E1068
:101D500096B0002916461D4613DB6A460AF0C5FEFA
:101D600000280EDB019A4FF4806302F47042A2F562
:101D70000052B2FA82F2002052092A60336016B093
:101D800070BD0022A3892A601B0604D540230020D1
:101D9000336016B070BD4FF480630020336016B01E
:101DA00070BD00BF8A890B46920706D5012103F159
:101DB000470259611A601A61704770B582B001AB71
:101DC0006A460C460646FFF7BFFF009905463046B7
:101DD000FEF79EFEB4F90C3070B1164A0099B2625B
:101DE000019A43F08003A3812060C4E904018AB909
:101DF0002B43A38102B070BD9A05FBD4012123F0CF
:101E0000030304F1470243F00203A38161612260EE
:101E10002261EFE73046B4F90E100AF072FE10B9F5
:101E2000B4F90C30E4E7A38923F0030343F0010382
:101E30001BB2DDE7D1160008830770B4CDB23DD0E8
:101E4000541E0AB30378AB421FD0431C05E014F1C3
:101E5000FF3419D30278AA4217D013F0030F1846A3
:101E600003F10103F3D1032C11D84CB30378AB4237
:101E70000BD00444431C02E00278AA4205D09C42E5
:101E8000184603F10103F7D1002070BC70470246E9
:101E90000E02B6B22E4346EA064613681046734059
:101EA000A3F1013121EA030313F0803F02F10402A0
:101EB000DCD1043C032C1046EFD8D6E71446D2E719
:101EC0002046E2E78842F0B40DD98B1883420AD944
:101ED000841832B1224613F8014D994202F8014D9F
:101EE000F9D1F0BC70470F2A0ED80346541E002AC1
:101EF000F7D001340C44013B11F8012BA14203F847
:101F0000012FF9D1F0BC704740EA01039B073AD199
:101F1000A2F110073F0901F1200606EB071601F1B7
:101F2000100300F1100453F8105C103344F8105CF7
:101F300053F81C5C103444F81C5C53F8185C44F8EB
:101F4000185C53F8145CB34244F8145CEBD17B1C6E
:101F50001B0112F00C0F194402F00F05034415D0B9
:101F60000E46043DAD0803EB850C1C1F56F8047BA0
:101F700044F8047F6445F9D10135AD002B44294470
:101F800002F00302B2E7541E0346B2E72A46ADE769
:101F90000148FFF7CFBE00BF803300200148FFF7A4
:101FA000D1BE00BF8033002009B3F8B51446CAB1D2
:101FB00006460D4600F066F8A04202D32F4638468A
:101FC000F8BD21463046FEF7A3FD07460028F6D0AF
:101FD00022462946FEF7C4FA30462946FEF744FD5C
:101FE0003846F8BD2746FEF73FFD3846F8BD114696
:101FF000FEF78EBD10B50C46B1F90E100AF05DFD6E
:10200000002803DB636D0344636510BDA38923F4DB
:102010008053A38110BD00BF002070472DE9F0411F
:10202000B1F90C409846E3050D461746B1F90E107C
:10203000064609D424F48054AC8143463A463046DF
:10204000BDE8F0410AF040BD022300220AF03AFD4B
:10205000B5F90C40B5F90E10ECE700BF10B50C4611
:10206000B1F90E100AF02EFDA389421C0EBF23F415
:10207000805343F480536065A38110BDB1F90E1005
:102080000AF024BD51F8043C181F002BBCBF0B58AC
:10209000C01870470E4A0023114610B5147C8442C4
:1020A0000FD11C225343CA18906848B1CB58FF285F
:1020B00018BF43434FF0010018BF5B00013353606A
:1020C00010BD0133082B02F11C02E7D10020F7E715
:1020D000D80E0020F0B50A4D00242E462F7C8742F2
:1020E00007D11C2000FB0464012061762276A376D0
:1020F000F0BD0134082C05F11C05EFD10020F7E7F5
:10210000D80E0020094A30B500231446157C8542BC
:1021100005D11C22012002FB0343596030BD01336D
:10212000082B02F11C02F1D10020F7E7D80E0020A5
:1021300070B50B4C00232546267C864209D11C2015
:102140004343E818E95000238260C36043740120D0
:1021500070BD0133082B04F11C04EDD10020F7E71A
:10216000D80E0020F8B500252E46334C6368002BAE
:102170005ED0E06858BB637CB3FA83F35B09637499
:1021800008F03CFCD4E900239342E06035D266605D
:102190006674E66063699BB1207C984780B1A36850
:1021A000FF2B0DD1677E217EA37E47EA01021A43F1
:1021B00006D0207CFF2823D11A46384606F0D6F9EF
:1021C0000135082D04F11C04D0D10120F8BD08F020
:1021D0005BFC23689842CED26368002BDAD020469D
:1021E00002F0A6F80028EBD0637C207CABB1FF287E
:1021F0000DD1A27E217E607EE0E79B1A6360EBE753
:102200005E28DDD80A46394605F006FBD8E75E2889
:10221000D6D8A37E227E617EF6E7FF2803D11A4638
:1022200019461846CAE75E28CAD81A461946EBE787
:102230006374E360C4E700BFD80E002007B543789D
:102240008DF8003083788DF80130C3788DF8023036
:1022500043798DF80330037968468DF804300BF02C
:1022600053FD03B05DF804FB08B5074B5A78022A0A
:1022700007D8586808F008FCC72894BF0020012040
:1022800008BD0020FCE700BF9C0C0020704708B58B
:10229000002240214FF080400AF0D6FDFFF7F6FF04
:1022A00000BF00BF00BF00BF00BF00BF00BF00BF36
:1022B00000BF00BF00BF00BF00BF00BF00BF00BF26
:1022C00000BF00BF08BD08B501F020F808BD000040
:1022D00008B5064C002120780BF02AFD2078FFF786
:1022E000F2FF052009F051FCF4E700BF682F002041
:1022F00010B5084C236803F07142074B1343236069
:1023000008F07CFB054B18602068BDE8104003F026
:102310006BBA00BF682F00200001010E4C11002095
:1023200008B5012280214FF080400AF08DFD4FF06A
:10233000804380229A61BDE8084001F0B3B80120D3
:1023400070470000144B10B51C78BCB9134B1B78B8
:10235000042B13D103F024F903F038F903F0ECF85F
:1023600003F07CF904F048F804F062F8204608F025
:10237000A5F92046BDE8104008F0BCB90BF08AFF73
:1023800048B10BF04FFC0028FBD1BDE8104044F6EB
:10239000206009F0FABB10BD682F00201833002020
:1023A00038B500230D460B70074C30B108F026FB02
:1023B000002320602B70002038BD206808F064FBEB
:1023C0003228F3D8F7E700BF5C110020084B9A7859
:1023D000012A07D0022A09D0064B1868B0FA80F00B
:1023E0004009704758780128F6D170470120FCE772
:1023F0009C0C00204016002008B5054B9B78013B43
:10240000012B02D9FFF7E2FF08BD0120FCE700BF66
:102410009C0C002008B508F0F1FA014B986008BD4B
:102420009C0C00202DE9F0410C461546074600287B
:1024300038D0B1FA81F35B09A3B14D4E4FF0804221
:102440003378002C32D08021012B91610AD03046A4
:102450000AF0BAFC30460AF09CF84648464B8360C6
:1024600008F0F8F8A74201D0FFF76CFF434E33782D
:10247000A34200D11DB10022414B9A611A773470FA
:1024800024B1631E042B747098BFB470306803F0DD
:10249000ABF93378062B64D8DFE803F06119303AE2
:1024A000444E58000B1C18BF0123C5E74FF4000130
:1024B000042B9161D6D0334BDFF8B8801C70324BBF
:1024C0003046C8F8083008F06BFE4046C8E73120B7
:1024D00045B10BF0E7FB52200BF0E4FB01200BF0C1
:1024E000EDFB51200BF0DEFBFFF794FF2A4621465F
:1024F000384601F0E7FB0120BDE8F0813220002DD5
:10250000F0D00BF0CFFB52200BF0CCFB0220E6E723
:102510003320002DE6D00BF0C5FB52200BF0C2FBA0
:102520000320DCE73420002DDCD00BF0BBFB522075
:102530000BF0B8FB0420D2E73520002DD2D00BF0F1
:10254000B1FB52200BF0AEFB0520C8E73020002D78
:10255000C8D00BF0A7FB52200BF0A4FBC1E7112061
:10256000C0E711200BF09EFBFFF7C2FEBCE700BFE7
:1025700018330020201100203D220008682F002081
:10258000640C0020A8230020A5B20008002313B586
:102590000DF107018DF80730FFF702FF044690B1F7
:1025A0009DF80730013B032B0DD8DFE803F002064E
:1025B0000F1200221146094B02E00022074B9978C6
:1025C0001878FFF72FFF204602B010BD0022062129
:1025D000F1E7024B00225978F2E700BF682F002094
:1025E00013B5124C20460BF0C1FA0123637703F0B8
:1025F000F8F80F4C206008B9FFF77AFEE37843F053
:102600000103E37008F0FAF90A4BFF221860002377
:102610004FF49A6100930848084B09F083FAFFF7DA
:1026200036FE0120FFF7B2FF02B010BD640C00209F
:10263000682F00204C11002060110020D1220008DA
:1026400038B5114C054623782070637008F0D6F930
:10265000032D606016D10120FFF798FF40B90B4AA7
:10266000537812785AB1024619461846FFF7DAFE37
:10267000FFF7D0FEBDE8384053200BF013BB1146E6
:102680001846F3E738BD00BF9C0C0020682F0020DF
:10269000014B1878704700BF9C0C0020014B9870CC
:1026A000704700BF9C0C0020014BD870704700BFE2
:1026B0009C0C0020014BD878704700BF9C0C002078
:1026C0000122014B1A70704758110020F8B5164BC3
:1026D0009C681CB9FFF79EFE0020F8BD134D144EF8
:1026E0002A7892B100232B704FF080431B69F27857
:1026F0009B0963F30002F27032680E4B1340B3F192
:10270000807FE9D000F028FEE7E7F3780A4AC3F3B8
:10271000420352F82370002FDED0204608F0B4F9AF
:10272000B842DFD2D8E700BF9C0C0020581100202F
:10273000682F0020FF00000140E600080C4B10B598
:102740005A781946012A03D0022A08D0002005E051
:102750009C78012C03D100F061FE204610BD486832
:1027600008F092F9C728F1D9FFF730FEF6E700BF6D
:102770009C0C002008B5074BDB780BB1022B04D171
:102780000220FFF75DFF002008BD0320FFF758FF80
:102790000120F9E79C0C002038B5094D0024E878A9
:1027A000032807D1FFF74CFF2046AC7000F0E4FD92
:1027B000012038BD0220FFF743FF2046F9E700BFA4
:1027C0009C0C002070B5754C754D2068A0B108F0C8
:1027D0005BF9B0F5FA6F0FD30026552026600BF099
:1027E00061FA57200BF05EFA287832460146B0FABB
:1027F00080F04009FFF716FE2B781BB1694BDA7F9A
:10280000694B1A702368ABB9684C206808F03CF932
:1028100040F6B73398420DD92B785BB10BF002FA32
:1028200040B9604B5B7F2BB108F0E8F82060532083
:102830000BF038FA4FF080431B69EA789B095C4C37
:1028400063F300020020EA70FFF7A0FE2378032B59
:102850001ED8DFE803F0021E448AE36833B19847CC
:1028600020B10120FFF7ECFE0023A370236933B1F0
:10287000984720B10120FFF7E3FE0223A3706369AC
:1028800033B1984720B10120FFF7DAFE0123A3708E
:1028900070BDA369002BFBD098470028F8D001F049
:1028A0007FFB444B187006F021FC0021424A2B7834
:1028B00013703C4A51776BB9404C2378012B09D0F7
:1028C0004FF08043802220469A610AF07DFA20462C
:1028D00009F05FFE0220BDE87040FFF7B1BEE3697A
:1028E000002BD5D098470028D2D04FF080434FF42A
:1028F00080229A61A37813B3022B0BD86378022B42
:1029000008D0FFF71FFD11200BF0CCF90BF08AF96E
:102910000028FBD100F012FD0023E370264B2A783B
:102920001B789A4202D1A07800F088FAA378012B94
:1029300018D0A3B1022BABD1FFF72EFFA8E7194B9C
:102940005B7E002BE6D111200BF0ACF90BF06AF99D
:102950000028FBD147F2305009F017F9DAE7FFF70A
:1029600009FF95E701F026FD92E7236A002B8FD03F
:10297000984700288CD001220A4B5A770D4B1B78C0
:102980002BB14FF0804304229A6106F095FB00F0D2
:10299000C9FCFFF73FFD00209DE700BF4C11002060
:1029A000682F0020640C0020A82300205411002070
:1029B0009C0C0020481100205011002018330020EA
:1029C0000120704708B5FFF7FBFF08BD37B5044687
:1029D0000D46FFF71FFD29462046FFF7F3FF60B1C4
:1029E000074B1A784AB1074B20461B78D90900914A
:1029F000C3F3001369790BF0A1FC03B030BD00BF35
:102A0000682F0020702F002008B5074807F012F942
:102A1000064807F00FF90BF001F907F00BF9BDE8D4
:102A20000840034807F006B960E600087BE60008A6
:102A3000A2E600082D4B13B51A7804466AB12C4B58
:102A400001211B78DB09009300230BF077FC0BF0CE
:102A5000E9F80028FBD102B010BD0028FBD0031F0D
:102A6000DBB2A02B12D8234B0146186807F07CFE7E
:102A700020B1204602F058FD02F0F0FD204602F0A1
:102A80004BFD02B0BDE8104002F0E8BD00F12003AC
:102A9000DBB2072B07D800F007040120A040C0B22A
:102AA00002F06EFDEDE700F15B03DBB2022B06D80E
:102AB000114AD05C02B0BDE8104007F0FFBD00F144
:102AC0005803DBB21A2B07D80C4A32F8130002B0B5
:102AD000BDE8104007F00EBE3334E4B2122CBAD871
:102AE000012102B0BDE8104001F0AFBE682F002008
:102AF000702F0020C40F002004E6000808E600083C
:102B0000264B13B51A7804466AB1254B1B78DB09AE
:102B10000093002319460BF011FC0BF083F80028FA
:102B2000FBD102B010BD0028FBD0031FDBB2A02BED
:102B300006D802F0F9FC02B0BDE8104002F08EBDEC
:102B400000F12003DBB2072B07D800F007040120B7
:102B5000A040C0B202F01CFDEDE700F15B03DBB268
:102B6000022B05D8104602B0BDE8104007F0A6BD04
:102B700000F15803DBB21A2B05D8104602B0BDE8AD
:102B8000104007F0B7BD3334E4B2122CC9D8114657
:102B900002B0BDE8104001F058BE00BF682F002011
:102BA000702F00202DE9F3410546E0B1134E327835
:102BB000E2B10127DFF84880284601F0D3FD98F8FC
:102BC00000300446DB09E030009332780023012115
:102BD00080B20BF0B3FB0BF025F80028FBD107FA0D
:102BE00004F4A543E8D102B0BDE8F08102F0C8FCCE
:102BF00002B0BDE8F04102F031BD00BF682F0020F7
:102C0000702F00202DE9F3410546E0B1134E3278D4
:102C1000E2B10127DFF84880284601F0A3FD98F8CB
:102C200000300446DB0900930023E0303278194677
:102C300080B20BF083FB0AF0F5FF0028FBD107FA06
:102C400004F4A543E8D102B0BDE8F08102F0A0FC95
:102C500002B0BDE8F04102F001BD00BF682F0020C6
:102C6000702F00202DE9F3410546E0B1134E327874
:102C7000E2B10127DFF84880284601F073FD98F89B
:102C800000300446DB09E030009332780023012154
:102C900080B20BF053FB0AF0C5FF0028FBD107FA06
:102CA00004F4A543E8D102B0BDE8F08102F07EFC57
:102CB00002B0BDE8F04102F0D1BC00BF682F002097
:102CC000702F00202DE9F3410546E0B1134E327814
:102CD000E2B10127DFF84880284601F043FD98F86B
:102CE00000300446DB0900930023E03032781946B7
:102CF00080B20BF023FB0AF095FF0028FBD107FA06
:102D000004F4A543E8D102B0BDE8F08102F056FC1E
:102D100002B0BDE8F04102F0A1BC00BF682F002066
:102D2000702F002038B51C4B1B7863B91B4C1C4D11
:102D30002378052B04D14FF080431B695A0603D436
:102D400007F05CFE286038BD28680028F8D007F03E
:102D50009BFE41F658339842F5D907F04FFE2860A4
:102D600025462378052B05D002F078FCBDE83840D5
:102D700003F042BB07F00BFEB4F84C309B07F0D5D4
:102D800007F0ECFD0028ECD0284609F091FC28461D
:102D900001F082F8E5E700BF682F0020183300201B
:102DA00030160020704700001A4B70B59C6C0F263F
:102DB00044F4C0649C649B6C012301F003048B40C9
:102DC00021F0030101F1804101F5A0518D68A400BB
:102DD000C0F38320A04006FA04F425EA0405284342
:102DE0008860D8430C4912F0010F8C6814BF1C4353
:102DF00004408C6012F0020FCA6814BF1A430240EC
:102E0000CA60054A536111680B431360536803405D
:102E1000536070BD000C0140001800400120704755
:102E200008B5FFF7FBFF38B1BDE8084001220621D5
:102E30004FF08040FFF7B8BF08BD00002DE9F04714
:102E40003023054683F31188824B00269A6C4FF09D
:102E5000010842F4C0629A649A6CD3F890207E4FC5
:102E600042F4C062C3F89020D3F89020DFF81492A7
:102E700022F4C062C3F89020D3F89030FFF7D0FF5F
:102E800057F8040B95B1012D49D1484547D120F0A1
:102E90000F0A00F00F0008FA00F421460522504600
:102EA000240409F0D1FFCAF8184001E0441CEED117
:102EB0000136112EE4D107240127684EDFF8C881BE
:102EC00056F8040B002D36D0012D40F0B680404559
:102ED00040F0B38000F00F01202207FA01F120F04A
:102EE0000F0009F0B1FF00BF00BF00BF00BF00BF6F
:102EF00000BF00BF00BF00BF00BF00BF00BF00BFDA
:102F000000BF00BF00BF00BF00BF56F8040C032283
:102F100000F00F0120F00F00FFF746FF0DE0411C0D
:102F2000C6D000F00F01202208FA01F120F00F00B6
:102F300009F08AFFBCE7421CCCD1013CC0D184F32C
:102F4000118872B6464A47491368424823F0010384
:102F500013600323444A93620C23D362434B0B60F8
:102F600001238460C36042480860A1F5A0418C67DA
:102F700040499462D462A2F5684251611946002228
:102F8000A30003F1604303F56143D3F80001D5B218
:102F9000012D94BF002000F0010008B1C3F880119A
:102FA0000132202AF1D10134082CE8D1324C636877
:102FB00043F00073636009F027FF2B4B1A6802F09F
:102FC00009021A601A6842F46C3242F004021A6074
:102FD00040F2B3321A62294B43F001039847236948
:102FE00043F00403236130BF254B43F001039847AE
:102FF00023691B4A23F004032361136843F0010390
:10300000136008F091F9134B9A6C42F4C0629A6411
:103010009A6C9A6C42F480429A649A6C9A6C42F46C
:1030200080529A649B6CFFF7BDFE02F083FF002381
:1030300083F3118862B6BDE8F087431C3FF47DAF8F
:1030400000F00F01402207FA01F120F00F0009F013
:10305000FBFE72E7000C0140F4E6000894E700086C
:1030600010E000E0005401400000014014000003A3
:1030700010000003FFFF070000ED00E06CE7000810
:1030800038E700080E0400400300004001207047AC
:1030900001207047012303FA01F2024210B50C46E9
:1030A0000DD003290CD006290CD10320FFF7FCFA20
:1030B0002046FFF7EBFF10B12046FFF7E9FF10BDF8
:1030C0000420F3E71846F1E710B5094C6369DB0704
:1030D00007D52368002123F0010323600120FFF7B7
:1030E000D9FF4FF0FF336361BDE8104008F0F6BD33
:1030F0000018004010B5094C606910F0020006D0BD
:103100002368012123F002032360FFF7C3FF4FF080
:10311000FF336361BDE8104008F0E0BD00180040D7
:1031200010B5094C606910F0040006D02368022134
:1031300023F004032360FFF7ADFF4FF0FF3363611B
:10314000BDE8104008F0CABD0018004010B5094C99
:10315000606910F0080006D02368032123F00803FB
:103160002360FFF797FF4FF0FF336361BDE8104026
:1031700008F0B4BD0018004010B5094C606910F0AB
:10318000100006D02368042123F010032360FFF70A
:1031900081FF4FF0FF336361BDE8104008F09EBD32
:1031A0000018004038B5214B5C69A00604F478751E
:1031B00007D51A68052122F020021A602846FFF779
:1031C00069FF610608D5194A06211368284623F0CD
:1031D00040031360FFF75EFF220608D5134A07215C
:1031E0001368284623F080031360FFF753FFE305BD
:1031F00008D50E4A08211368284623F4807313600B
:10320000FFF748FF14F4007F084C07D0236809211A
:1032100023F4007323602846FFF73CFF4FF0FF3391
:103220006361BDE8384008F059BD00BF0018004098
:1032300038B5264B5C69620504F47C4507D51A68ED
:103240000A2122F480621A602846FFF723FF200536
:1032500008D51E4A0B211368284623F40063136027
:10326000FFF718FFE10408D5184A0C211368284617
:1032700023F480531360FFF70DFFA20408D5134A0F
:103280000D211368284623F400531360FFF702FF53
:10329000630408D50D4A0E211368284623F48043A1
:1032A0001360FFF7F7FE14F4004F084C07D02368B3
:1032B0000F2123F4004323602846FFF7EBFE4FF075
:1032C000FF336361BDE8384008F008BD00180040D6
:1032D00010B5074C23784BB900F0A6FE01F05FFA59
:1032E00007F0BEF901F05CFA01232370012010BD44
:1032F0003516002010B5044C23781BB100F096FE63
:1033000000232370012010BD35160020024B1B78CE
:103310000BB10AF091BC70473816002001207047AD
:103320000120704708B5044B1B780BB9FFF7D0FF9D
:10333000FFF7F4FF08BD00BF3516002008B5044BA9
:103340001B780BB1FFF7D6FFFFF7EAFF08BD00BF00
:10335000351600200120704708B5FFF7FBFF08BDB8
:10336000014B1878704700BF36160020014B1870CB
:10337000704700BF36160020014B1870704700BF21
:1033800036160020014B1878704700BF3716002012
:10339000084B10B50446187058B9FFF779F90228A0
:1033A00007D80320FFF74CF92046BDE81040FFF78F
:1033B00075B910BD37160020FFF7EABF024B187829
:1033C00080F00100FFF7E4BF37160020084B1A78A1
:1033D000084B1B784BB982F00102A0F5A443203BB7
:1033E0001F2B8CBF1046012070470022F5E700BF5D
:1033F000371600203616002000231946054A93721E
:103400001360054A01330B2B917242F80C1BF9D162
:10341000704700BF54160020C00C002008B502F011
:10342000FBFDFFF7E9FF0022014B1A6008BD00BF5A
:103430004016002008B505F0A1FE18282CD8172842
:1034400003D2062801D00DD880B9002328201A46BF
:10345000194604F0E1F900235C201A46194604F0ED
:10346000DBF903E00828F0D00A28EED007F000F9D5
:10347000820705D5442328201A46194604F0CCF9C2
:1034800007F0F6F8430705D544235C201A46194691
:1034900004F0C2F9012008BD1C28E7D31E28D4D9A6
:1034A0002028E2E708B5FFF713FFFFF799F800F0CF
:1034B00095FD48B1012204214FF0804009F0C4FC81
:1034C0004FF0804304229A6108BD000000230E4A99
:1034D00010B513700D4A4FF0804413700C4A1360FE
:1034E000FEF798FF05F022FE01280AD005F016FE2F
:1034F0004FF48023A36100F07DFDBDE8104002F091
:1035000004BA0423F6E700BF341600203916002061
:103510003C16002008B502F0C9F904F033F902F0B6
:1035200059F9084B188060F07F001870188802F075
:1035300054F900F0C9FD18B1BDE80840FFF7C6BF57
:1035400008BD00BF702F002037B504460D4600F0BF
:10355000CCFD002800F0BD80002D00F0BA8047F6B9
:1035600004639C4200F0858029D847F601639C42A1
:103570005BD00AD847F603439C4200F0A780B4F51D
:10358000FC4F3CD0284603B030BD47F602639C4256
:103590005DD047F603639C42F4D100230DF107018F
:1035A00001208DF80730FEF7FBFE9DF80730042B55
:1035B00002D013F0FD0FE5D10122042130E047F6DF
:1035C00012639C427BD00BD847F605639C4263D0C4
:1035D00047F611639C42D5D10020FFF7D9FED1E711
:1035E00047F613639C426ED047F643639C42C9D1B1
:1035F0000122394B1A700022384B1A60C2E70023AF
:103600000DF1070101208DF80730FEF7C9FE9DF886
:103610000730042B02D013F0FD0FB3D10122114665
:103620002F4B1878FEF7FEFEACE700230DF10701E3
:1036300001208DF80730FEF7B3FE9DF80730042B0C
:1036400002D013F0FD0F9DD101220221E8E70023F3
:103650000DF1070101208DF80730FEF7A1FE9DF85E
:103660000730042B02D013F0FD0F8BD10122032170
:10367000D6E700230DF1070101208DF80730FEF792
:103680008FFE9DF80730042B03D013F0FD0F7FF45D
:1036900079AF01220521C3E700230DF107010120C5
:1036A0008DF80730FEF77CFE9DF80730DA1E012A00
:1036B00002D9002B7FF466AF01220621B0E7012278
:1036C000084B1A705EE7FFF779FE5BE7FFF722FF12
:1036D00058E7054656E700BF391600203C16002083
:1036E000682F00203716002070B5154CFFF76AF8D8
:1036F000206858B1A37A4BB907F0C6F963689842BD
:1037000004D301212089A172FFF71EFF00250126A5
:103710000C4C206858B1A37A4BB907F0B5F963682F
:10372000984204D3A67201212089FFF70DFF0135CD
:103730000B2D04F10C04ECD100F07AFC70BD00BF3D
:1037400054160020C00C002008B5064B1B780BB99E
:10375000FFF7BEFD4FF0804304229A61BDE80840A8
:1037600007F0FBB83516002008B5074B1B780BB1E6
:10377000FFF7C0FD4FF080434FF480229A61BDE80F
:10378000084007F0E9B800BF351600202DE9F743DF
:103790000D46AD4A49790446136891B1032B00D810
:1037A0000133AA4E1360FEF735FE33899C4204D1E3
:1037B0006F7957B107F022F93060A54B0027984682
:1037C00029E0002BEDD0013BEBE7B37A0BB9336076
:1037D000F3E739462046FFF7B7FEB7723760002897
:1037E000EBD1002095E07E4308EB0607BB7A13B9C6
:1037F00048F806301DE049462046FFF7A5FE87F849
:103800000A9048F806900028EBD012E001370B2F01
:1038100003F10C030DD01A899442F7D195F8059065
:103820000C26B9F1000FDED007F0E8F87E4348F827
:10383000060029462046FFF7C9FD0028D1D02946B9
:10384000204600F055FC0028CBD047F604639C428C
:1038500000F0C1802CD8B4F5FC4F67D009D847F6EA
:1038600020039C4200F0158147F603439C42B8D0E8
:103870002EE047F602639C426B7900F0918074D988
:10388000002BAED0734C2278042AAAD000230DF16D
:10389000070101208DF80730FEF782FD9DF8073003
:1038A000042B02D013F0FD0F9BD10022042158E01D
:1038B00047F640639C421ED015D847F606639C42EB
:1038C00000F0CE80C0F0A38047F607639C422AD068
:1038D0002946204600F054FE002882D02946204682
:1038E000FFF774F815E047F642639C4214D009D301
:1038F00047F64363BAE76B79002B3FF472AFFFF7EB
:1039000083F86EE76879544B10B101221A7068E7AA
:10391000187003B0BDE8F0836B79002B3FF461AF02
:10392000FEF7CEFE5DE76A794C4BEFE76B79002B33
:103930003FF457AF474C2278012A3FF452AF00239F
:103940000DF1070101208DF80730FEF729FD9DF8E4
:103950000730042B03D013F0FD0F7FF442AF002299
:1039600001212078FEF75EFD3BE7002B3FF439AFE5
:10397000384C2278022A3FF434AF00230DF10701BE
:1039800001208DF80730FEF70BFD9DF80730042B62
:1039900003D013F0FD0F7FF424AF00220221E0E7F3
:1039A000002B3FF41EAF2B4C2278032A3FF419AFB3
:1039B00000230DF1070101208DF80730FEF7F0FC20
:1039C0009DF80730042B03D013F0FD0F7FF409AFEF
:1039D00000220321C5E76B79002B3FF402AF1D4C99
:1039E0002278052A3FF4FDAE00230DF107010120E6
:1039F0008DF80730FEF7D4FC9DF80730042B03D078
:103A000013F0FD0F7FF4EDAE00220521A9E76B79DD
:103A1000002B3FF4E6AE0F4C2278062A3FF4E1AECD
:103A200000230DF1070101208DF80730FEF7B8FCE7
:103A30009DF80730DA1E012A02D9002B7FF4D1AE9F
:103A4000002206218DE700BF4016002054160020FA
:103A5000C00C0020682F00203816002034160020EB
:103A60006B79002B3FF4BDAE114C2278002A3FF455
:103A7000B8AE00230DF1070101208DF80730FEF7E5
:103A80008FFC9DF80730012B3FF6ABAE00221146AC
:103A900067E76B79002B7FF41BAF05F047FB4FF016
:103AA000804318B14FF480229A6111E70422FBE7AA
:103AB000682F0020014B1870704700BF441600208B
:103AC000F8B505460C46584E584F2146284600F09A
:103AD0000FFC50B1062C08D8DFE804F004085D9311
:103AE00093A0A0000022504B1A60F8BD32687ABB48
:103AF000A5F14703042B0BD8DFE803F025201B16A4
:103B000003000023FF211A464B20FEF7E3FA0122AF
:103B10004FF4FA712846FEF70BFB2846FEF7BAFA77
:103B200006F06CFF3060E0E7FF22002311464A20D8
:103B3000EBE70022FF2311464920E6E70023FF229E
:103B400019464820E1E7442347201A461946DCE796
:103B5000104606F099FF4EF65F23984203D90524DC
:103B6000334B1C70B1E7334B1B7883B9472D0ED113
:103B7000314B1B78042B3FD103232D4C2846237057
:103B800044231A461946FEF7A5FA24789DE77A7E63
:103B90008AB30324E4E73068F8B9A5F14803032B9E
:103BA000A3D8DFE803F015100B020023FF211A460B
:103BB0004B20FEF78FFA0122C821ABE7FF2200233A
:103BC00011464A20F5E70022FF2311464920F0E77D
:103BD0000023FF2219464820EBE706F055FF4EF67A
:103BE0005F23984201D90624BAE77B7E0BB10424F7
:103BF000B6E7104B1B786BB12846BDE8F840FEF7DE
:103C000049BAFF224FF4FA612846FEF791FA284696
:103C1000FEF740FA0022064B1A7066E70022044BBA
:103C20001A70FEF74DFDE7E748160020640C0020EF
:103C300044160020682F00201833002008B5034BDD
:103C40001978FFF73DFF012008BD00BF4416002092
:103C50000120704770B506460D464B200021FEF747
:103C600051FA10B90024204670BD00214A20FEF709
:103C700049FA0028F6D000214920FEF743FA00282F
:103C8000F0D000214820FEF73DFA0028EAD00021BC
:103C90004720FEF737FA0028E4D029463046FFF7E0
:103CA000D7FF04460028DDD00022044B29461D70B2
:103CB000034B30461A60FFF703FFD4E74416002099
:103CC0004816002070B50D461446FEF738FB064630
:103CD00080B155B3174B5B7E2BBB013D052D09D839
:103CE000DFE805F0030C120808182CB102214B2064
:103CF000FFF7B0FF304670BD0121F8E714B1022193
:103D00004A20F5E70121FBE714B102214920EFE742
:103D10000121FBE714B102214820E9E70121FBE77B
:103D200002214720E4E71E46E4E7002CF8D10121F8
:103D3000F7E700BF640C0020094B1B787BB9094BE7
:103D40001A7832B1084A527E4AB959781046FEF7BD
:103D500069BB064B1B78042B01D01146F6E7704770
:103D600044160020682F0020640C00201833002027
:103D70002DE9FF473F4D06460F4600F0F1FAFFF7E9
:103D8000DBFF2C78002C31D03B4C236813B906F0B4
:103D900035FE2060206806F077FE40F6B733984283
:103DA00005D92B7801332B7006F028FE20602B7884
:103DB000013B032B16D8DFE803F0020B0F130022A0
:103DC0001146442004F0D2FB002004B0BDE8F08787
:103DD000002244211046F5E7002144220846F1E77D
:103DE0004422EDE700232B702360EDE7234B1B7883
:103DF00083B939463046FFF71DFB0028E4D0394629
:103E00003046FEF7AFF93946304604B0BDE8F0471A
:103E100000F0B8BA22462146204604F0A7FBDFF89E
:103E200060A0DFF860900DF104080A2551462A468B
:103E30004046FCF795FB99F81E30E2B2B3FBF5F56E
:103E4000954214F8080011D9312B03D90023FF2221
:103E5000194605E01D2B4FF00003F8D81A46FF2144
:103E6000013403F0D9FC0A2CDFD1C2E700231A4643
:103E7000EEE700BF391600203C1600203416002063
:103E80008CE40008640C0020012804BF014B18706A
:103E900006F03ABD1C110020014807F076BE00BFB5
:103EA000A0860100F8B50023374E5E280446337023
:103EB000364D21D1364A374F1269F97882F4806243
:103EC000C2F3802262F30001CA072B70F97015D586
:103ED000314A927F632A17D9304A19461360442227
:103EE000FEF7F8F8FF22C8215E20FEF721F9012332
:103EF0002B705E20FEF7CEF82878F8BD4FF0804397
:103F00001B6913F040030BD00023244A19461360A9
:103F10005E204422FEF7DEF801224FF49671E3E7BB
:103F20001D4FBA7F0A2A23D81A464421FEF7D2F839
:103F30000122C8212046FEF7FBF801232B703370C5
:103F4000BB7F012BD5D8154C236813B906F056FD5D
:103F5000206020680028CCD006F096FD42F2107355
:103F60009842C6D9002301202360FFF7FFF9C0E77C
:103F70000A4A194613601A46FEF7ACF8FF22C82118
:103F80002046FEF7D5F8B4E74E1600204D16002067
:103F900000080040682F0020640C0020501600200C
:103FA000024B1878C0F34000704700BF6C2F002010
:103FB000034B1A7860F341021A70186801F01BBCB9
:103FC0006C2F0020044A137823F0030343F003030B
:103FD0001370106801F00FBC6C2F002008B5002290
:103FE0004FF48061024808F02FFF012008BD00BF98
:103FF0000008004010B501F0FBFB0A4B186008B93F
:10400000FFF7E0FF4FF080444FF48023A36105F0F9
:104010008DF808B10423A3615E20FEF73BF8012070
:1040200010BD00BF6C2F0020012070470120704799
:1040300070B5002006F028FDB0F57A7F34D34FF03C
:1040400080441D4A23691178C3F3801399421B4DA4
:1040500013D02369C3F38013137023695B060CD557
:10406000174E3378042B08D006F0C8FC4FF4000339
:104070002860A361304607F093F82868A0B106F0E5
:1040800003FDB0F5FA6F0FD300220D4C2A602378A0
:10409000042B0BD04FF08043802220469A6108F019
:1040A00093FE204608F075FA012070BD054B1146BD
:1040B0001878FEF7B7F9F7E76016002064160020BD
:1040C00018330020682F002008B54423FF201A462B
:1040D0001946FDF7FFFF0322FA21FF20FEF728F81B
:1040E000FF20FDF7D7FF012008BD01207047000029
:1040F00045F22123984270B505460C4600F0CD806C
:1041000017D8B0F5A97F00F0B6800AD8E32800F0F0
:10411000A58040F251139D4200F0AD80012420465D
:1041200070BD40F22B43984200F0A78040F62C036C
:10413000F1E747F62303984236D020D845F22323EF
:10414000984200F0AA8047F620039842E6D14C79C5
:10415000002C39D1614D2878C0F3400080F0010077
:1041600000F00100FFF724FF2B789B0740F1A380AC
:1041700004F0B4FF4FF0804304229A61CFE747F682
:10418000146398422ED047F6156398424DD047F6F7
:1041900007639842C2D1524B1B7803B14B79514A05
:1041A00003F0010313700FE004F0E8FF0B28B5D013
:1041B0000CD8072806D80528B0D20138C0B201288B
:1041C00002D8ABE70928A9D00024A8E7282805D8F9
:1041D0002128A3D21C28A1D01F28F4E72B38C0B275
:1041E0000228EDE7404C207800F0BCFA0228EBD022
:1041F000207800F0B7FA88B9022000F018FA0022FF
:1042000044231146FF20FDF765FF0122FA21FF201C
:10421000FDF78EFFFF20FDF73DFFD5E7207800F08A
:10422000A1FA0228EBD10020E7E72F4C207800F01C
:1042300099FA02280546C7D1207800F093FA30B9E0
:10424000284600F0F4F9002344221946DAE72078E2
:1042500000F088FA0228F6D10020F2E7224B187805
:1042600000F080FA02287FF459AF284664798CB1B7
:1042700000F052F9A8E76479F9E74C794CB11B4B8F
:104280001A7822B90122E2201A7000F045F92B2099
:10429000EEE72B2000F056F941E76679002E7FF417
:1042A0003DAF124D2C78002C3FF438AFE22000F0E7
:1042B00049F92E7033E706F0DBF910F0FF0F83D1D8
:1042C0002C78C4F34004002C7FF47EAF04F026FF6A
:1042D0004FF080434FF480224FE700BF6C2F002047
:1042E000682F0020341600206E1600204C16002087
:1042F0000539012910B5044615D80020FFF7DAFB6F
:104300000A4B1B7833B1FEF7DBF92046FDF7C2FEFE
:10431000002010BD4FF080431B695B06F5D40120DF
:10432000FFF736F8F1E70120F3E700BF682F002020
:1043300008B5037C5E2B0DD1074B1B7813B1074BDF
:10434000187830B900235E201A46194603F064FA43
:10435000002008BD0120FCE7682F00204D1600203A
:10436000064B1B789B0702D5054B1B7823B1002217
:104370001146104604F0FAB8704700BF6C2F0020B9
:104380004E16002008B5094B1B78DB060BD5084BF1
:10439000187800F0E7F9022805D044230B201A46CC
:1043A000194603F039FA012008BD00BF702F002024
:1043B0006E16002008B5FEF77DF904280ED00628F9
:1043C00001D003280AD10320FEF73AF90020FEF7B6
:1043D00065F90020FEF7F0FF012008BD0220FEF77E
:1043E0002FF90020F9E7000010B548B14FF08044E4
:1043F0002369590703D404F071FE0423A36110BD9F
:10440000064B1B789A07FAD44FF0804423695B0768
:10441000F5D504F083FE4FF48023EFE76C2F0020E6
:1044200010B50278072A01D0002010BD4278032A77
:10443000FAD18278022AF7D10B4BC4781A7834B9B2
:1044400064F341021A7006F043FF0120EDE742F0E9
:1044500002021A704FF080431869C0F380000028F0
:10446000E2D104229A61E0E76C2F002003280DD8E6
:1044700006290BD8102A09D8772301EB011103FB79
:104480000010034B104433F81000704701207047B0
:10449000B8E70008012070470C22024B02FB0030F5
:1044A000704700BFB80F0020A0F58073B3F5F85F28
:1044B00010B526D210F4805F00F4007400F480730D
:1044C00000F4806100F400620DD0002B0CBF0020CE
:1044D00010200CB140F0200009B140F040000AB1BA
:1044E00040F0800010BD181C18BF01200CB140F036
:1044F000020009B140F00400002AF3D040F00800A7
:10450000F0E70020EEE710B50C46FFF7CDFF23469D
:10451000BDE8104018470000A0F1E003072B10B5DC
:10452000044600D940B920460449FFF7ECFFE0B249
:10453000BDE81040FEF77EBA0149F6E7A52B00085A
:10454000652C000810B50446C0B2FEF7D9FAA4F1F4
:10455000E003072B00D92CB903492046BDE81040E1
:10456000FFF7D1BF0149F8E7052C0008C52C00086A
:104570000120704708B5FFF7FBFF08BD0120704719
:1045800001207047704708B5FFF7FCFF08BD000029
:1045900013B502AB03E903000F4B1B78B3B99DF8C9
:1045A0000530009873B16AB100F0BEFC04460146C4
:1045B000009800F087FC2046009902B0BDE810404A
:1045C00001F030BB00F098FC0446F4E7009800F0DE
:1045D000ABFC0099F1E700BF6D160020034600898F
:1045E00010B40A4638B95C881888998840EA0440B3
:1045F00010BCFFF7CDBF10BC704738B50121044691
:10460000FFF7ECFF21460546FFF7B4FF18B121463E
:10461000284605F07DFC00F0010038BD10B50446C9
:104620000021FFF7DBFF2146FFF7ADFF10BD10B5FE
:1046300001248440E4B2204601F0C8F82046BDE8D9
:10464000104000F0A0BB704708B500F041FBFFF739
:10465000FAFFBDE8084046F2A81007F096BA08B580
:10466000FFF7F2FFBDE8084006F026BA08B5FFF7ED
:10467000EBFFBDE8084006F047BA38B50121054612
:10468000FFF7ACFF2946044604F0EAFF08B9002012
:1046900038BD29462046FFF779F80028F7D029468B
:1046A000204605F03BFF0028F1D02946204605F0C2
:1046B00057F90028EBD02946204605F0ADFE00282A
:1046C000E5D02946204604F095FE0028DFD0294693
:1046D000204605F071FF0028D9D06B795BB147F611
:1046E00003439C421DD00AD8B4F5F84F16D047F6C4
:1046F00001439C4217D02846FFF740FFC8E747F622
:104700005B439C4215D047F65C439C420ED047F673
:104710005A439C42EFD101F035F8ECE7FFF79FFFD9
:10472000B5E701F035F8FFF7A1FFB0E701F01EF89B
:10473000E1E701F02AF8DEE708B5FFF715F804F025
:10474000B3FB00F035F8BDE80840012004F090BC50
:1047500008B500F032F8002004F08AFCBDE80840FB
:10476000FEF7F2BF03091CBF1846042382081EBFD0
:1047700010460233DBB242081CBF0133DBB21846DD
:10478000704701207047704738B50546FFF7F9FFBD
:10479000044610B12846FFF7F6FF204638BD7047A3
:1047A00010B50446FFF720FE2046FFF7EDFF10BDD1
:1047B00008B50020FFF7F4FF08BD08B505F050FF6D
:1047C000FFF7EEFF08BD000010B505F049FF074BED
:1047D00004461A78824207D0187006F00FF9044B8D
:1047E00018602046FFF7DCFF10BD00BF6C160020EC
:1047F0006816002010B586B06C4684E803009DF86A
:1048000005300BB100F0E2FE0023ADF81230ADF838
:10481000143094E8030011F0FF0F0390ADF810106E
:1048200003AC05D194E8070000F012FE06B010BDFD
:104830002046FFF7E2FE0028F4D1F7E70379012BC9
:1048400002D1008800F092BB704708B529B101F091
:10485000FFFCBDE8084001F0CFBD01F057FDF8E7CF
:1048600038B505460C46FEF7E5F81CB92846FEF7B4
:1048700047F938BD6420013C07F087F9A4B2F4E79A
:1048800008B539280CBF50213221FFF7E9FF08BDD8
:104890002DE9F047867981460C46457900F060FEA7
:1048A0003609804600B3A846F5B1C4F3072303F0E8
:1048B000F002402A09D004F12002D2B2072A25D9F9
:1048C0001EB903F0E003202B23D0A84B93F80180FE
:1048D00018F0040808D0022000F018FF00F040FE95
:1048E00080F001005FFA80F8C4F303330B2B3FD84C
:1048F000DFE813F01100110060006000BD00D3007C
:104900003E003E00D8003301450145014FF000084C
:10491000EAE7B046E8E7C4F30723C4F3032613F03D
:10492000F00F18BF3601E7B285B156B107F1200389
:10493000DBB2072B304600D92FB900F021FE00F082
:104940008DFE384658E000F031FEF8E73846FEF7B5
:10495000D7F86EB107F12003DBB2072B304600D940
:1049600017B900F015FE01E000F028FE00F076FE19
:10497000C4F30334083C032C03D805F071FEFFF7A1
:104980000FFFB8F1000F00F0528100F0E1FD10F0D0
:10499000010040F04C8189F8050000F0D3FD00F0E3
:1049A00025FA484600F05EF900F0CCFDBDE8F0477E
:1049B00000F028BAC4F3072303F0F003C4F303277D
:1049C000202B5FFA84FA18BF3F01BAF1000F07D01D
:1049D000BAF1010F32D0002D3AD0CEB150460BE0E3
:1049E000624B5B785A0711D44DB127B1384600F0BD
:1049F000C7FD00F033FE0020FEF71CF8B8E728469C
:104A0000FEF77EF8002FB3D03846AAE755B11EB99D
:104A10003846FEF7C7F8ABE7012EA9D1384600F0BB
:104A2000F5FDA5E7002EA3D13846FEF7EBF8384692
:104A300000F0FAFD384600F0D5FD99E715B1052ED6
:104A400096D8E5E7042E93D83846FEF7DBF88FE7D3
:104A5000002EF9D0BAF1390F0CBF4FF4FA5041F2E1
:104A6000883007F092F85046FEF74AF880E7C4F322
:104A7000812343B1012B7FF47BAF65B1C4F30900FF
:104A800005F038FE74E725B1C4F3090005F016FE01
:104A90006EE72846FAE72846F2E72946E0B2FFF734
:104AA000D4FE65E714F4407F27D1002D7FF460AF7A
:104AB000C4F342108000C3B204F00F009840C2B2A9
:104AC00014F010001EBF0F209840C043C4F3812390
:104AD00018BFC0B2022B40EA020008D00AD8012B4E
:104AE00002D000F05BF943E700F050F940E700F036
:104AF0005DF93DE700F047F93AE7C4F30122D3B28C
:104B000005B302F00103002B3FF432AFC4F34210AF
:104B10008000C3B204F00F009840C2B214F010003D
:104B20001EBF0F209840C043C4F3812318BFC0B2FA
:104B3000022B40EA02000AD00CD8012B04D000F06E
:104B400081F915E75B08DEE700F074F910E700F083
:104B500081F90DE700F038F90AE7E7B2C4F303265C
:104B600035B1304600F042F952E700BF702F002007
:104B70003846FEF747F8304600F044F9F8E6E7B269
:104B8000A7F1F003042B3DD8DFE803F003220E1554
:104B90001E003DB1042E3FF6EBAEC4F3042000F03E
:104BA0003DF9E5E6052EF6E7C4F30420002DE3D138
:104BB00000F01CF9DCE625B1C4F3042000F00FF985
:104BC000D6E600F009F9D3E61A4B5B785B0704D40C
:104BD000C4F30420002DCFD0EAE74DB1C4F304257F
:104BE000284600F003F90321284600F06DFDBFE6DA
:104BF000012000F08BFD012E7FF6BAAE022000F0FE
:104C000085FDB5E62DB1002E7FF49BAEC4F30420E4
:104C1000CEE74EB1392F0CBF4FF4FA5041F2883035
:104C200006F0B3FF38461FE7C4F30420A4E7BDE84D
:104C3000F08700BF702F002038B50446008960B1AE
:104C400000F016FF054600F00DF900F09BF829462C
:104C50002046BDE83840FFF71BBE2188607900F090
:104C600091F9EFE7037910B50446B3B1FFF705FDFD
:104C700068B900F075FC80B1637973B1074B5B785C
:104C80005B070AD5BDE81040022000F03FBD20467A
:104C9000FFF7D2FF2046FFF7C1FC10BD702F0020A8
:104CA00008B5002005F00AFD002005F023FD00F006
:104CB0008DFC00F0D3FC01F0BBFBBDE8084001F027
:104CC0009BBB08B500F038FCBDE80840FFF7E8BF23
:104CD00008B500F065FCBDE80840FFF7F2BFC0F37F
:104CE00003320E3202F00F02092A10B5C4B21BD8EB
:104CF000012101FA02F340F20332134203D113F00F
:104D000010000DD110BDF02C10D004D8E72C8CBFB2
:104D100000200120F6E7F42C14BF00200120F1E769
:104D2000E72C03D9F12CF7E70020EBE70846E9E789
:104D300008B50346007958B1188928B100F098FEEB
:104D4000BDE80840FFF7CBBF188800F00FF9F7E780
:104D500008BD82B002AB03E9030002B0704784B023
:104D600004AB03E9070004B07047704708B5FFF7CC
:104D7000FCFF08BD08B5FFF7F9FF014B187008BD2F
:104D80006E1600207047FFF7F5BF0000024B1B783E
:104D90001843FFF7EFBF00BF6E160020024B1B78D1
:104DA0001840FFF7E7BF00BF6E160020024B1B78CC
:104DB0005840FFF7DFBF00BF6E160020704708B5F0
:104DC000FFF7FCFF08BD000008B5FFF7F8FF014B37
:104DD000187008BD6F1600200020FFF7F5BF0123F3
:104DE00003FA00F0C0B2FFF7EFBF0000012303FA9F
:104DF00000F0034B1B781843C0B2FFF7E5BF00BFBC
:104E00006F160020012303FA00F0034B1B7823EAFE
:104E10000000FFF7D9BF00BF6F160020012303FA7F
:104E200000F0034B1B785840C0B2FFF7CDBF00BF66
:104E30006F160020024B1B781843FFF7C5BF00BF59
:104E40006F160020024B1B781840FFF7BDBF00BF54
:104E50006F160020024B1B785840FFF7B5BF00BF0C
:104E60006F160020704701F00703C90830B501EB49
:104E70004101012401390A4400219C40E4B212F8A6
:104E8000015F20FA01F343F300036B40234001313B
:104E90006B4003291370F2D130BD002210B500F031
:104EA0000704C00800EB4000014410468B5CE3405F
:104EB00003F00103934001321843032AC0B2F5D135
:104EC00010BD000017B40C46C0F307210629ADF849
:104ED00004000CD89DF80430102B08D8204603EBB2
:104EE0000113044A194403B010BCFFF7BCBF03B060
:104EF00010BC70477016002082B0ADF80400C0F3FB
:104F0000072006280AD89DF80430102B06D800EB9D
:104F100000100449184402B0FFF7BFBF002002B0E0
:104F2000704700BF7016002073B503240D4BADF819
:104F300004001E780C4B1B781E4346FA04F3DB0773
:104F4000E5B206D414F1FF34F7D20025284602B0AA
:104F500070BD0199284600F076FE80B20128F1D09C
:104F6000F4E700BF6F1600206E16002007B5ADF8FD
:104F700004000198FFF7D8FF019903B05DF804EB36
:104F800000F061BE13B5104BADF804101B782BB1C7
:104F9000019802B0BDE81040FFF7E8BF70B101987A
:104FA000FFF7C2FF044601460198FFF78BFF20463A
:104FB000019902B0BDE8104000F045BE0198FFF72E
:104FC0009BFF0446F3E700BF6D16002010B50124D7
:104FD00004FA02F204FA01F11143C9B231EA000203
:104FE00004FA03F306BF1843C0B2984310BD000093
:104FF00008B513460A46014603480078FFF7E6FF66
:10500000BDE80840FFF7E0BE6F160020F8B50A279C
:105010000D4B0E4E1C780E4D3378A34200D1F8BDD7
:1050200007FB04F2AB18A85AB3F802C09A88D988D3
:1050300040EA0C4042EA014101341A89FFF78FFE31
:1050400004F00704E8E700BFF9160020F816002076
:10505000A8160020064B10B49A885C881888D98856
:1050600040EA044042EA014110BC1A89FFF777BECA
:105070009E160020F8B51C4B9A7912F0F00F0CD157
:105080005A7952B14FF00A0C184A194912780D7822
:105090001E885F88174CAA4200D1F8BD0CFB02F1B4
:1050A000601890F804E0BEF1000F19D0615AB142C7
:1050B00016D14179A1B94188C91B89B2C7290FD836
:1050C0000122997962F307119971837962F30713C9
:1050D00083710548FFF7C6FDBDE8F840FFF796BFAE
:1050E000013202F00702D6E79E160020F9160020D2
:1050F000F8160020A8160020F0B50A270D4B0E4A1E
:105100001B7816780D4CB34202D100221046F0BD38
:1051100007FB03F5621992F801C08C4505D1655D66
:10512000854202D15279002AF0D1013303F00703FE
:10513000E9E700BFF9160020F8160020A8160020A5
:105140002DE9F04F8BB002AB04460146062218460B
:10515000FBF706FAB34D0346297922796779A84609
:10516000C1B9AAB18FB12046FFF7E2FD064660B192
:105170000A2221462846FBF7F3F92846FFF75EFB93
:10518000FFF778FFFFF766FF69E02046FFF76AFD4B
:10519000012664E0B4F802A068886E79AAEB0000EA
:1051A00094F800B094F8019080B2002E00F0FB80DB
:1051B000C72800F2A380002A51D0AB792A8813F0C7
:1051C000F00F20885CD1904212D129892289914226
:1051D0000ED1002F4DD1012262F30713AB71FFF7FF
:1051E00039FF2846FFF73EFDAB79A371002636E074
:1051F000002F3ED149465846FFF77EFF5846FFF73D
:105200007BFF05460028F1D18DF808B08DF8099094
:105210000298FFF7ABFEC0F303310B2912D801222D
:105220008A4012F4406FC3B21DD112F00C0F0ED1A0
:10523000910707D010F4706F00D07BB12033DBB240
:10524000072B0BD92046FFF70DFD354606E010F47D
:10525000706FF3D0A27912F0F00FEFD12E463046E6
:105260000BB0BDE8F08FEF2BF8D90F33DBB2022B78
:10527000E7E798F8063043F0010388F80630B5E711
:1052800090420ED12889228990420AD14FB92046F6
:10529000A371FFF7E7FC0A2221462846FBF760F9D5
:1052A00070E72046FFF744FD00283FF46EAF002F63
:1052B0003FF46BAF98F806301F2B15D9B8F80020D3
:1052C0008DF81630ADF8102098F80420B8F80830A2
:1052D0008DF814200022ADF812A08DF81520ADF83D
:1052E000183004A8FFF7BEFC0A2221464D48FBF700
:1052F00037F9FFF7BFFEFFF7ADFE49E7A87910F0D9
:10530000F001019118D18DF80C208DF808B08DF8BE
:105310000990ADF80AA08DF80D7093E80300FFF72F
:1053200018FD2846FFF79EFC0A2201992846FBF744
:105330008DF9FFF78FFE59E7002A90D02A8823883D
:105340009A420ED12A8923899A420AD14FB9A07173
:105350002046FFF787FC0A2239462846FBF776F9F4
:105360007DE72046FFF7E4FC00283FF40EAF002F56
:105370003FF40BAF98F806301F2BB5D9B8F80020D2
:105380008DF82230ADF81C2098F80420B8F80830C9
:105390008DF820200022ADF81EA08DF82120ADF858
:1053A000243007A89EE7C7283ED8002A3FF4F0AE75
:1053B0003E46002F3FF4E9AE2A8823889A4220D146
:1053C0002A8923899A421CD1AB79DA0713D413F0C6
:1053D000F00210D0F02AA37106D0DBB2C3F303129F
:1053E000013262F30713A3712046FFF73BFC0A2248
:1053F00021460C4852E70A2221460A48FBF7B0F83A
:105400002DE72046FFF794FC00287FF46DAF98F855
:105410000630204643F0010388F80630FFF722FCEF
:105420001DE700BF9E1600208DF80C208DF808B0F7
:105430008DF80990ADF80AA08DF80D7093E803007F
:10544000FFF787FC0A2231462846FBF7FFF899E66A
:10545000F0B589B001AC84E807002046FFF770FE84
:10546000294E0746294D70B19DF808301BB194E8CC
:105470000700FFF774FC0A24254F2878337883420D
:1054800026D109B0F0BD05AB94E8070003C31A802C
:105490009DF80830002BEED033782A785C1C04F09D
:1054A000070494420AD00A22194805A902FB030006
:1054B000FBF756F83470FFF7A9FDDCE7FFF708FCAF
:1054C0000A223946134837702F70FBF7BFF8D2E72E
:1054D00004FB0070FFF734FE0028D2D02A78624324
:1054E000BB18B85AB3F802C09A88D98840EA0C4071
:1054F00042EA01411A89FFF732FC2B78013303F0AD
:1055000007032B70B9E700BFF8160020F91600203A
:10551000A81600209E160020024B0146186805F0D0
:105520008BB900BFC40F0020024B0146186805F07C
:105530009BB900BFC40F0020014B186805F0ACB93F
:10554000C40F0020014B1878C00870473A1700209C
:10555000024B187800F00700704700BF3A17002090
:10556000034B187810F0070018BF0120704700BFE8
:105570003A170020014B1878704700BF3D170020F4
:10558000024A137818431070704700BF3D1700207F
:10559000024A137823EA0000107070473D1700207C
:1055A0000022014B1A7070473D170020024A137801
:1055B00018431070704700BF3E170020024A13784E
:1055C00023EA0000107070473E1700200022014BB4
:1055D0001A7070473E170020704708B5FFF7FCFFB0
:1055E00008BD000008B5054A1378034204D023EA39
:1055F00000001070FFF7F1FF08BD00BF3B1700204F
:10560000704708B5FFF7FCFF08BD000008B5054A64
:10561000137830EA030C03D003431370FFF7F1FF54
:1056200008BD00BF3C17002008B5054A13780342A7
:1056300004D023EA00001070FFF7E3FF08BD00BFAD
:105640003C17002008B5044B1A781AB100201870D6
:10565000FFF7D7FF08BD00BF3C17002010B5124B65
:1056600012491B780978124C0B43124920680978BB
:10567000037031B10B43037005F058F808B1FFF720
:10568000E1FF246820220C492046FAF739FF48B18F
:10569000214620220848FAF763FF2046BDE8104063
:1056A00004F0EABF10BD00BF3D1700203E170020E8
:1056B000C40F00203C1700201A170020704708B5BF
:1056C000FFF7FCFF08BD0000094A10B552785207E9
:1056D0000AD5084C41EAC0012170FFF787FB20780A
:1056E000C008FFF7ECFF10BDBDE81040FFF77EBB20
:1056F000702F00203A170020002008B5024B1870C8
:10570000FFF7DDFF08BD00BF3A17002008B50A4AC1
:10571000137823EA0000107042070CD198420AD097
:10572000064B5B785B0706D5C008FFF76BFBBDE84F
:105730000840FFF7E1BF08BD3A170020702F002096
:10574000094A08B55378C3F3800181420AD060F357
:1057500082035370108800F040F8BDE80840022032
:10576000FFF7D4BF08BD00BF702F0020044B58784E
:10577000C0F3800080F0010000F00100FFF7E0BFFF
:10578000702F00200120FFF7DBBF0020FFF7D8BFFC
:1057900008B500F0CFFFBDE808404FF6FF710020CC
:1057A00000F0AABF08B5002000F03FFF4FF6E66307
:1057B000984203D1BDE8084003F0F7BE002008BDC1
:1057C000022000F023BF032000F020BF0146032089
:1057D00000F084BF042000F028BF0146042000F040
:1057E0008BBF0F2000F030BF01460F2000F092BFAA
:1057F000132000F029BF0146132000F08BBF0020CA
:10580000FFF7F9BF08B50020FFF7EEFFFFF7F7FF3E
:1058100008BD000013B5002400F08CFF4FF6E661D0
:10582000002000F069FF0021022000F057FF002156
:10583000032000F053FF1C4B4FF4A05104201C70B8
:1058400000F05AFF2146062000F048FFFF21072004
:1058500000F044FF2146082000F05CFF2146242090
:1058600000F03CFF2146172000F038FF21460C20B5
:1058700000F034FF21460D2000F030FF002300220D
:105880006846CDE900231821082200F00DFF2146CB
:10589000202000F03FFF204603F09CFE03F0BFFEF7
:1058A000FFF7B0FF02B010BD6E160020FFF7B2BFC9
:1058B00001460E2000F012BF73B505F0D9F80B4C6D
:1058C0000546238883420ED00026ADF8006005F01F
:1058D000CFF8ADF80460ADF8020002AB13E90300A5
:1058E000FEF788FF258002B070BD00BF481700207A
:1058F00008B505F083F8024B1860024B186008BD2C
:10590000401700204417002070477047012070475F
:1059100008B5054800F090FA00F00AFFFFF7F4FF21
:10592000FCF7FEFC08BD00BF315E00080120704797
:1059300008B5FFF7FBFF08BD08B5FDF7F3F9FDF764
:10594000D3FE08BD08B500F097FAFEF728FFBDE8C2
:10595000084003F035BB000008B505F04DF803F032
:105960006EFE00F059FBFFF7EDFF054B1A7842F091
:1059700080021A701888FFF730FFFDF7A7FD08BDF9
:10598000702F00202DE9F04F85B0FFF7BFFF60B901
:10599000FFF792FF04F070FA03F086FA00F070FD52
:1059A00005B0BDE8F04FFEF70FBF2F4E00F04EFBE5
:1059B00037460024E0B257F8045B00F087FA062C63
:1059C0004FD0854204F10104F4D0284B1B789B078B
:1059D00001D500F081FAFFF7ABFF00254FF0010B76
:1059E00000905FFA85F8404600F070FA56F8043BE4
:1059F000074698422FD000244FF0010943400193FD
:105A0000019B13EA090F1ED0009B17EA090F14BF70
:105A10004FF0010A4FF0000A83B18DF808408DF86D
:105A2000098005F025F88DF80CB0ADF80A008DF866
:105A30000DA002AB93E80300FEF7DCFE52462146C0
:105A4000404602F0EBFE0134E4B2112C4FEA490962
:105A5000D6D146F8047C0135072DC2D1FFF748FFA7
:105A600098E78542B1D193E74C17002068170020D2
:105A700038B500F0F3F8B0F5A04F044622D2B0F5E7
:105A8000804F77D2DF2812D8CD2861D2A7280AD834
:105A9000A5284ED2012804D003B233B1032898BF01
:105AA0000024204638BDC2284AD90024F9E7B0F5C1
:105AB000005F80F0A280B0F5807F4DD2E82828BF3B
:105AC0000024EEE745F25F23984216D845F24023C2
:105AD00098425FD245F21F23984254D8B0F5A44FA4
:105AE0007CD30123C4B2A00804F0030403FA04F435
:105AF00044EA401444F40D442CE045F29F239842BC
:105B000007D8B0F5A54F52D300F01F044AF2F400B5
:105B10003DE045F2BF23984256D945F2DF23984233
:105B2000C3D8040204F4F85444F4204444F0F004CC
:105B3000B7E75B34394BE4B21C5D44F48044B0E712
:105B40005834374BE4B233F8144044F48844A8E79F
:105B500040F4A044A4B2A4E7C0F3072000F006F983
:105B60000546E0B200F07AF82D0205F4F855284316
:105B700084B296E7C0B200F071F804F47064044394
:105B800044F42044E6E700F01F044AF2F10040EA42
:105B9000042486E70123C4B2C4F3820004F00304A2
:105BA00003FA04F444EA401444F40C44D2E7012319
:105BB000C4B2C4F3820004F0030403FA04F444EA18
:105BC000401444F40A44C5E700F01F0000F0CEF88A
:105BD000040204F4F85444F4005462E700F01F0097
:105BE00000F0C4F8C306C4F3431448BF0001240204
:105BF00000B2044344F41044ACE7C0F3042000F0C6
:105C0000B5F80546E0B200F029F82D0205F4F85584
:105C100045EA000444F400549CE700BF70EB000820
:105C200074EB000882B0ADF80410C1F30721062917
:105C300006D89DF80420102A02D802B004F040BB18
:105C4000002002B0704707B5ADF804100199FFF7C6
:105C5000E9FF03B05DF804EBFFF70ABF822825D007
:105C60000CD8312867D004D829285AD02A2869D0DE
:105C70007047352850D0392818D07047E32833D0E2
:105C800004D8E0281CD0E22829D07047E62835D077
:105C9000E72838D0E42835D1334B5A78910731D5ED
:105CA0001B7813F0100F08BFE72015E02E4B1A7871
:105CB000920752D15B7813F0080F18BF2920704764
:105CC000294A1378D90744D4527812F0010F19D019
:105CD00013F0100F08BFE32018BF00207047224BBD
:105CE0001B7813F0040FF2E71F4A1378590732D4D8
:105CF0005278D20731D413F0100FEDE71A4B1B780E
:105D00001A07CED47047184A1378190727D4527847
:105D10009107F0D5E4207047134B1B7813F0200F48
:105D2000CBE7114B1A7892061BD45B7813F0080F5F
:105D300018BF392070470C4B1B7813F0400F18BF69
:105D40002A207047084B1B7813F0400F18BF3120F2
:105D5000704739207047E2207047E0207047E62006
:105D600070473520CEE700BF702F002010B52F4CB4
:105D700021784B0713D500F01402A2F1040C00F0B7
:105D80001803DCF1000242EB0C02A3F1080CDCF179
:105D9000000343EB0C039A4218BF80F00C000B0782
:105DA00013D500F01402A2F1140C00F01803DCF17A
:105DB000000242EB0C02A3F1180CDCF1000343EBF0
:105DC0000C039A4218BF80F00C006478E30713D5E7
:105DD00000F0110202F1FF3C00F01803DCF10002B8
:105DE00042EB0C02A3F1080CDCF1000343EB0C03C3
:105DF0009A4218BF80F00900A30711D500F01102E4
:105E000000F01803A2F111046242A3F1180C6241E0
:105E1000DCF1000343EB0C039A4218BF80F0090049
:105E2000CB0648BF00F0E70010BD00BF702F002078
:105E30000020704700207047014B1860704700BF7A
:105E4000C80F0020FFF7A4BC08B500F0FFF8C82079
:105E500005F09BFE00F0FAF8002000F037F8C307C9
:105E600005D5FFF7EFFFBDE8084004F025BE08BDEB
:105E700008B5FFF7E9FF08BD08B5FFF793FC08B9BF
:105E8000FFF714FDFFF79CFC084B1870FFF7A2FC0E
:105E9000074B1880FFF7ECFFFFF795FCFEF773FF49
:105EA000044B1878BDE80840FEF789BF681700204A
:105EB000702F00206F160020704708B5FFF7FCFF19
:105EC00008BD704708B5FFF7FCFF08BD014B53F84C
:105ED00020007047902F002070474FF4076005F0B6
:105EE0008DBC00BF00BF00BF00BF00BF00BF00BF30
:105EF00000BF00BF00BF00BF00BF00BF00BF00BFAA
:105F000000BF00BF00BF704708B5FFF7E6FF08BD40
:105F100008B5302383F31188012100F00F03994065
:105F2000202220F00F0006F08FFF002383F311885A
:105F300008BD000038B511240B4D55F8040B421C68
:105F400001D0FFF7E5FF013C14F0FF04F5D1072471
:105F5000064D55F8040B431C01D0FFF7D9FF013C57
:105F600014F0FF04F5D138BDACEB0008F0EB0008ED
:105F70002DE9F843264D0E4655F8211080464B1C5E
:105F8000174642D0302383F31188012221F00F09F4
:105F900001F00F0102FA01F421464846240406F0FC
:105FA00053FFC9F81840002484F31188FFF799FFC4
:105FB0006FEA070C1748A8F1040208F1180850F816
:105FC000041B52F8043FB1F1FF3F1AD021F00F0E2D
:105FD000DEF810E001F00F012EFA01F1C90710D42C
:105FE00001243B4313609045E9D155F82600431C3A
:105FF00001D0FFF78DFF21463046BDE8F843FFF79B
:1060000083BF0CEA03031360EDE7BDE8F88300BF2C
:10601000ACEB0008F0EB000810B51C24FFF78AFF7A
:10602000224600210748FAF711FB224600210648C4
:10603000FAF70CFB072000F03FF8BDE81040FFF72F
:106040003CBF00BF902F0020742F002070B588B097
:106050001C22002101A8FAF7F9FA002401252A469A
:10606000E1B201A80134FFF783FF112C4FEA450587
:10607000F5D11C2201A90E48FAF742FA002814BFF4
:106080000126002607D00A4D01AC0FCC0FC594E8BD
:10609000070085E80700334607220649044800F058
:1060A0000DF80446FFF70EFF204608B070BD00BF94
:1060B000742F0020902F0020704700002DE9F04140
:1060C00080460F461546124E2BB10123337004F063
:1060D00095FC104B186034781CB900242046BDE8AC
:1060E000F0810C4B186804F0CFFC0028F5D0AD000F
:1060F0002A4641463846FAF703FA38B12A4641465D
:106100003846FAF72DFA00233370E7E70446FAE73A
:10611000691700206C17002008B505F015F9FFF786
:106120001BFCBDE8084005F025B908B505F028F9C5
:10613000FFF728FCBDE8084005F024B908B504F0D5
:106140001FFC05F0FFF8FFF7E3FBFFF7E5FFFFF7A4
:10615000ECFFFFF7F1FBFAE700EB4003C3EB03139F
:1061600000EB830003B2002B07DAB3F1800001D506
:1061700003F17F0040F30720704703F18000F9E747
:10618000164B1B78D90707D5154B187840007F2888
:106190001FD800B3C0B270479A0703D5104B1878C8
:1061A0008000F4E75B0703D50D4B1878C000EEE7DD
:1061B0000C4B1B785BB10C4A094912780878934262
:1061C000F4D25843C000B0FBF2F080B2DFE7082001
:1061D000E0E77F2070470120704700BF7A1700205A
:1061E000CE0F00207B170020CF0F0020144B1B7810
:1061F000D90705D5134B18788008F8B1C0B270479D
:106200009A0703D50F4B18784008F6E75B0705D5CA
:106210000C4B18787F28F0D97F2070470A4B1B78E9
:1062200053B10A4A074912780878934236BF584357
:1062300080B2B0FBF2F0EDE70120DFE7012070470C
:106240007A170020D20F00207C170020D30F0020E7
:10625000CD2808B505D1FFF793FF4042294BD870F0
:1062600008BDCE2802D1FFF78BFFF7E7CF2805D175
:10627000FFF786FF4042234B9870F1E7D02802D108
:10628000FFF77EFFF7E7D92804D1FFF7AFFF1D4BDB
:106290001871E5E7DA2803D1FFF7A8FF4042F6E7D7
:1062A000DB2805D1FFF7A2FF4042164B5871D7E714
:1062B000DC2802D1FFF79AFFF7E700F12F03DBB2EA
:1062C000072B08D801230F4AD13803FA00F053787E
:1062D00018435070C4E7DD2805D10B4A137843F00A
:1062E00001031370BCE7DE2804D1074A137843F09A
:1062F0000203F6E7DF28B3D1034A137843F004031F
:10630000EFE700BF741700207A170020364BCD2826
:1063100093F902200AD193F9031000290CDA002125
:10632000D97052B90021314A117006E0CE280DD142
:1063300093F903100029F2DC72B11A795B791343E7
:106340005BB2002B4FD12A4A13707047CF2806D179
:10635000002AF1DA00229A7093F90320E1E7D028AD
:1063600002D1002AF6DCE7E7D92893F9041004D11A
:106370000029E1DD00211971DEE7DA2802D10029C8
:10638000DADAF7E7DB2893F9051004D10029D3DA2C
:1063900000215971D0E7DC2802D10029F8DCCBE7D5
:1063A00000F12F01C9B2072907D80121D138814056
:1063B000587820EA01005870BEE7DD2805D10D4865
:1063C000017821F001010170B6E7DE2804D1094807
:1063D000017821F00201F6E7DF28ADD10548017808
:1063E00021F00401EFE77047741700207B170020AD
:1063F0007C1700207A17002008B504F039FB094B00
:10640000DA7899780A431CBF074A10801A795B79B9
:1064100013431CBF054B18800248BDE8084004F038
:1064200043B900BF741700207017002072170020B6
:1064300008B5062200210548FAF708F90023044AA6
:106440001370044A1370044A137008BD74170020B7
:106450007B1700207C1700207A17002090F902306B
:106460005BB990F9033043B990F904302BB990F936
:106470000500003018BF0120704701207047000060
:1064800037B5594C062221466846FAF769F80023C9
:106490009DF80220A370E370237163719DF80330AF
:1064A00013430AD0514B188804F0E7FA504A137886
:1064B0003BB35049097888422CDC9DF804209DF8B4
:1064C000053013430BD04C4B188804F0D6FA4B4AD6
:1064D0001378002B4ED04A490978884253DC69462C
:1064E000414804F0EDF918B93F48FFF7B7FF08B18C
:1064F000FFF782FF062269463B48FAF731F803B0FE
:1065000030BD40490D780A2169438842D5DD013309
:10651000137001E0FF2BFAD19DF902503DB1FFF756
:106520002FFE002DCCBF0123FF235843A0709DF9FF
:1065300003503DB1FFF724FE002DCCBF0123FF2304
:106540005843E07094F902000028B6D094F9032073
:10655000002AB2D0FFF700FE30B1A0701046FFF75E
:10656000FBFD20B1E070A8E70123A370F6E701234B
:10657000E370A2E724490D780A2169438842AEDD21
:106580000133137001E0FF2BFAD19DF904503DB1A6
:10659000FFF72CFE002DCCBF0123FF2358432071B1
:1065A0009DF905503DB1FFF721FE002DCCBF012321
:1065B000FF235843607194F9040000288FD094F9A8
:1065C0000520002A8BD0FFF7C7FD30B1207110469F
:1065D000FFF7C2FD20B1607181E701232371F6E767
:1065E000012363717BE700BF741700207017002040
:1065F0007B170020CD0F0020721700207C17002091
:10660000D10F0020CC0F0020D00F0020002307B5B1
:10661000014601220DF107008DF8073000F08CF8DB
:106620009DF8070003B05DF804FB002307B50146A1
:1066300002220DF10600ADF8063000F07DF8BDF83D
:10664000060003B05DF804FB07B5042200230146F1
:106650000DEB0200019300F06FF8019803B05DF8B4
:1066600004FB07B501228DF8071001460DF1070064
:1066700000F067F803B05DF804FB07B50222ADF83F
:10668000061001460DF1060000F05BF803B05DF85E
:1066900004FB07B50422019101460DEB020000F056
:1066A00050F803B05DF804FBF8B505461446D31D59
:1066B00023F0070300AFADEB030D68460E4600F074
:1066C0003BF8224669462846F9F71AFF20B12246D0
:1066D0003146284600F035F8BD46F8BD38B50C46C1
:1066E0000546FFF793FFA04205D021462846BDE8A6
:1066F0003840FFF7B6BF38BD38B50C460546FFF742
:1067000094FFA04205D021462846BDE83840FFF757
:10671000B4BF38BD38B50C460546FFF795FFA0421B
:1067200005D021462846BDE83840FFF7B2BF38BD46
:1067300000F01EB900F03CB80B460146184600F0C8
:1067400051B80B460146184600F09EB808B5064BF6
:106750004FF4006200211846F9F778FF40F608026E
:10676000C0F8002808BD00BF8017002010B5064CF7
:1067700094F8043833B900F076F910B1012084F8A8
:10678000040810BD0220FCE78017002010B5074C5C
:1067900094F804383BB100F070F918B100230120DF
:1067A00084F8043810BD0220FCE700BF80170020E9
:1067B00038B5FFF7DBFF044618B9FFF7E7FF2046BF
:1067C00038BD00F052F90546FFF7C0FF012C06D195
:1067D000FFF7DCFF00280CBF002505F001052C4663
:1067E000EDE7000008B5034608469918B1F5006FBB
:1067F00005D804491944F9F7B3FE012008BD00206B
:10680000FCE700BF8017002038B5FFF7AFFF4FF45B
:10681000807205461049002000F04CF970B10CA3BD
:10682000D3E900234FF400610B4803F05CF8024603
:106830000B464FF4006000F076F930B90024012DCA
:1068400001D1FFF7A3FF204638BD0224F7E700BFC0
:1068500025232284E49CF2CB8017002010B5094C3C
:10686000D4F80038B3F5805F09D300F0FEF828B102
:10687000FFF7CAFF40F60803C4F8003810BD012036
:10688000FCE700BF801700208318B3F5006F2DE9E7
:10689000F74F06460D46174604D90024204603B09C
:1068A000BDE8F08FDFF8C08008EB000421462846E1
:1068B000F9F726FE002854D03A4629462046F9F733
:1068C0004FFEFFF753FF824628B14FF0000B2FB960
:1068D000FFF7C4FF29E0FFF759FFDEE7052FB946B0
:1068E00028BF4FF00509C6F3024343EAC9038DF8F8
:1068F0000030330AADF802B08DF80130ADF804B0C5
:10690000ADF806B08DF802600DF1030305EB090246
:1069100015F8011B954203F8011BF9D1DDE90023AD
:10692000D8F8000800F0FFF808B9044611E0D8F8DC
:1069300000380833C8F80038FFF790FF01280446F4
:1069400003D1A7EB09074E44C1E710B1022818BFD5
:106950000024BAF1010FA1D1FFF718FF00289CD045
:106960009CE701249AE700BF801700200000000088
:10697000F0B585B0FFF7EAFE00F070F820B9FFF738
:10698000E5FE002005B0F0BD4FF4807232490020D2
:1069900000F075F8304E10B9FFF7D8FEEFE72CA3E2
:1069A000D3E900234FF40061304602F09CFF0D460E
:1069B000044602A94FF4006000F079F8DDE90223F3
:1069C0009D4208BF944201D0FFF7C0FE40F6080781
:1069D0006946384600F06BF810B3DDE9004554EA2B
:1069E00005031CD0E2B2930907F10807CDE902457F
:1069F00026D104F47F431004C4F307441C4300F47D
:106A0000E0202043D2088318B3F5006F18D80DF1A9
:106A10000B013044F9F7A4FDB7F5805FD8D1012010
:106A2000C6F8007870B900F020F80028A7D0FFF76A
:106A3000EBFE40F60803C6F800380028A2D19EE716
:106A40000020EDE7FFF70AFFF7E700BFAFF3008094
:106A500025232284E49CF2CB8017002008B500F0A7
:106A6000D1F8012008BD0120704708B5002000F0D2
:106A7000CBF8B0FA80F0400908BD0120704738B566
:106A8000D5002A460C4600F0DCF818B9214625440A
:106A9000A94203D1B0FA80F0400938BDD1E9002302
:106AA000D243DB4341F8082B41F8043CF0E70122D4
:106AB000FFF7E5BF2DE9F043074688461546002657
:106AC000C1B06B46202DAE4628BF4FF0200E1C46AD
:106AD0009C4608EBC602764408EBC6094A4511D12C
:106AE0000024744513D14FEAC4094A46614638462A
:106AF00000F0C5F8A8B92D1B4F44E2D1012041B0E8
:106B0000BDE8F083F2E80201E4E80201E6E7D3E938
:106B10000002C043D24343F8080B43F8042C01346D
:106B2000DFE70020EBE707B5CDE900236946012246
:106B3000FFF7C0FF03B05DF804FB0000002208234C
:106B40001146014804F06EB80C08004008B5FFF784
:106B5000F5FF30B1062004F0A3F804F0D9F80020C6
:106B600008BD4FF0FF30FBE738B503F047FF00F5F5
:106B70007A75FFF7E3FF78B1052004F091F804F08F
:106B8000A1F8C4B204F0C4F803F038FFA84206D25A
:106B900014F00100EDD138BD4FF0FF30FBE76FF08E
:106BA0000100F8E7F7B51F464BBA090C0646154633
:106BB0008DF80400ADF806308DF80510FFF7BEFF24
:106BC000E8B104210DEB010004F08EF8044648B949
:106BD00045B1022E0BD0032E0ED1B9B2284604F0D7
:106BE0008DF8044604F094F8204603B0F0BDB9B225
:106BF000284604F079F8F4E74FF0FF34F2E74FF05D
:106C0000FF34F1E703F0D2BF00F58033B3F5002F76
:106C100010B5044612D283B283B9FFF7A5FF78B945
:106C2000FFF794FF60B9034602462146D820FFF7DC
:106C3000B9FF28B9BDE81040FFF796BF4FF0FF300D
:106C400010BD2DE9F04180460D461646FFF78CFF3A
:106C50000446074638B1324600212846F9F7F6FCCB
:106C60002046BDE8F08133462A4641460320FFF71F
:106C700099FF04460028F3D032463946EDE72DE966
:106C8000F04107468846164676B9FFF76DFF044681
:106C900038B9FFF753FF20B3042004F001F804F0E3
:106CA00037F82046BDE8F081FDB2C5F58075B542E4
:106CB00028BF3546FFF758FF04460028F1D1FFF7FB
:106CC00045FF04460028ECD12B46424639460220B7
:106CD000FFF768FF04460028E3D1A8442F44761B41
:106CE000D2E74FF0FF34DCE730B5C0F3072285B0C0
:106CF0000190C0F30740BAB909B1304B185C8DF868
:106D00000C008DF80D008DF80E0000209DF80C3061
:106D100063F307009DF80D3063F30F209DF80E30EC
:106D200063F3174005B030BD9DF8043061B32349CB
:106D3000085C0625FF215D436FF05404B5FBF1F5B7
:106D40006C4304EB430404EB4404E4B204FB02F39D
:106D5000C4F1FF04891A62431B121212C3F1FF032C
:106D6000C2F1FF02414343434243C1F30721C3F34E
:106D70000723C2F30722C0B2062D19D8DFE805F0B9
:106D80000608110F1418060080B2D2E70346104619
:106D90008DF80C008DF80D308DF80E10B5E7024619
:106DA00018460B461146F3E7134602460846F9E734
:106DB0000246084619461346EAE700BF24EC0008DD
:106DC000012184B004B0FFF78FBF012830B501D88E
:106DD000C0B230BDB0F5F75F88BFFF224FF00101B0
:106DE0009EBF42090832D2B28B185B1003FB03F539
:106DF000ADB28542DCB205D9621ED2B29142F3D95E
:106E0000481EE5E7FF2B02D0611CC9B2F6E7184621
:106E1000DFE70000074B188800EB402200EB820000
:106E200000F55850193080B2188000EB1020C0B225
:106E3000704700BFDA0F002010F0400116BFC343B7
:106E40000346DBB210B503F00F0201B1013209496C
:106E5000C3F301135B00CC186478CB5C624303EB93
:106E60002213DBB2020644BF5B42DBB283F0800038
:106E700010BD00BF0CEC0008144B84B003EB4101C3
:106E8000E423019091F87710C0F307204B43C2EB45
:106E900013231C33002BB8BF5B42A0EBC3031BB210
:106EA00023EAE373584300128DF805000020019B8C
:106EB000DAB262F30700C3F3072262F30F20C3F3D1
:106EC000074363F3174004B0704700BF440D002030
:106ED000144B84B003EB4101E423019091F8771047
:106EE000C0F307404B43C2EB13231C33002BB8BF46
:106EF0005B42A0EBC3031BB223EAE37358430012C7
:106F00008DF806000020019BDAB262F30700C3F39C
:106F1000072262F30F20C3F3074363F3174004B063
:106F2000704700BF440D002084B0019000208DF810
:106F30000420019BDAB262F30700C3F3072262F375
:106F40000F20C3F3074363F3174004B070470000FA
:106F500084B0019000200B4B03EB410191F8773096
:106F60009A1A8DF80420019BDAB262F30700C3F38A
:106F7000072262F30F20C3F3074363F3174004B003
:106F8000704700BF440D002084B0019000200B4BDF
:106F900003EB410191F878309A1A8DF80420019B97
:106FA000DAB262F30700C3F3072262F30F20C3F3E0
:106FB000074363F3174004B0704700BF440D00203F
:106FC00030B5134B85B03831019003EB4104257A7D
:106FD00003EB4103A5F1200464B2002CDB79BCBFB4
:106FE000C5F1200464B29B1AC0B2234403440020BC
:106FF0008DF80430019BDAB262F30700C3F3072275
:1070000062F30F20C3F3074363F3174005B030BDAD
:10701000440D002084B0019000209DF8102003EB67
:10702000430302EB53028DF80420019BDAB262F3B2
:107030000700C3F3072262F30F20C3F3074363F390
:10704000174004B070471FB592B2019048B20028B3
:1070500002FB02F2BCBF484240B2C0F1380000FB64
:10706000002080B21C46FFF7B0FE00EB4000044455
:1070700000208DF80440019BDAB262F30700C3F3ED
:10708000072262F30F20C3F3074363F3174004B0F2
:1070900010BD000084B0019003F13800104B03EBE9
:1070A0004003187ADB792038703B594302FB001209
:1070B0000020002A9DF80410B8BF7F3201EBE212D5
:1070C0008DF80420019BDAB262F30700C3F30722B4
:1070D00062F30F20C3F3074363F3174004B0704714
:1070E000440D002084B0019003F13800104B03EBF5
:1070F0004003187ADB792038703B594302FB0012B9
:107100000020002A9DF80410B8BF3F3201EBA21204
:107110008DF80420019BDAB262F30700C3F3072263
:1071200062F30F20C3F3074363F3174004B07047C3
:10713000440D00201FB503F13804164B019003EBFA
:1071400044031C7AC0B2203C6243DC79A4F1700392
:107150005BB2002BBCBFC4F170035BB2C3F1380358
:1071600001FB032111EB410148BF7F3100EBE1112D
:1071700000208DF80410019BDAB262F30700C3F31C
:10718000072262F30F20C3F3074363F3174004B0F1
:1071900010BD00BF440D002030B50D4685B00190F4
:1071A000C4B21046FFF748FE124B0C2203EB450316
:1071B00093F877301844C0B2A0F180035BB2002B83
:1071C000BCBFC0F1800043B200205B00DBB2534380
:1071D00004EB13248DF80440019BDAB262F307003C
:1071E000C3F3072262F30F20C3F3074363F317408F
:1071F00005B030BD440D0020114B84B0019003EB6D
:10720000410191F87710C0B28B1A5BB2002BBCBF62
:10721000521A53B21822DBB2534300EB13208DF8FD
:1072200004000020019BDAB262F30700C3F30722D7
:1072300062F30F20C3F3074363F3174004B07047B2
:10724000440D0020054B40F6B8301B791033FF2B5E
:1072500028BFFF231B09B0FBF3F07047B02F0020BD
:10726000C94384B00190C9B2C0F30740484300123B
:107270008DF806000020019BDAB262F30700C3F329
:10728000072262F30F20C3F3074363F3174004B0F0
:10729000704784B0C9B20190C1F18201C0B2002927
:1072A000A8BF40188DF804000020019BDAB262F3F9
:1072B0000700C3F3072262F30F20C3F3074363F30E
:1072C000174004B0704784B0BDF8102003EB83036F
:1072D00013449BB2FF2B28BFFF23DB430190DBB29B
:1072E000C0F307400344FF2B28BFFF2300208DF885
:1072F0000630019BDAB262F30700C3F3072262F3A0
:107300000F20C3F3074363F3174004B0704700290D
:107310001FB5B8BF4942002AB8BF524209B209019D
:1073200012B2FF294FEA0212A8BFFF21FF2AA8BF0D
:10733000FF22BDF8184009B2234412B29BB2914219
:10734000D4BF5B189B189BB2FF2B28BFFF23DB43E6
:107350000190DBB2C0F307400344FF2B28BFFF239B
:1073600000208DF80630019BDAB262F30700C3F308
:10737000072262F30F20C3F3074363F3174004B0FF
:1073800010BD00001FB5482B0190C0F3074030D856
:10739000BDF81840E31A9BB2FF2B28BFFF2308312A
:1073A00089B2102905D902F1080189B2112928BF33
:1073B000FF23DB43DBB20344002AB8BF0332FF2BB9
:1073C00028BFFF2300200C498DF80630497801EBD7
:1073D000A2028DF80420019BDAB262F30700C3F326
:1073E000072262F30F20C3F3074363F3174004B08F
:1073F00010BDFF23D3E700BFB02F002084B0BDF83D
:1074000010200190D31A9BB2FF2B28BFFF23DBB2C1
:10741000D943C0F30742C9B20A44FF2A28BFFF225A
:1074200018448DF8040000208DF80620019BDAB284
:1074300062F30700C3F3072262F30F20C3F307438D
:1074400063F3174004B0704784B0BDF8102001907A
:10745000D31A9BB2FF2B28BFFF23DB43C0F30740A7
:10746000DBB20344FF2B28BFFF2300208DF806303A
:10747000019BDAB262F30700C3F3072262F30F2025
:10748000C3F3074363F3174004B07047024A13780D
:1074900018431070704700BF8A1F0020012310B5E9
:1074A000044C0822182104482370FFF745F90023F3
:1074B000237010BD8A1F0020B02F002028B900299A
:1074C000ACBF002380231846704780EAE072A2EB2D
:1074D000E072002912B201EB0203ABBF891A5B0113
:1074E0004901511AABBF91FBF3F393FBF1F3C3F1E5
:1074F0002003C3F160035BB2DBB20028BCBF5B4278
:10750000DBB2E0E730B5C0F3072585B0EB1A019098
:107510001046DCB2FFF7D2FFC0EB801300EB830014
:1075200004440020E4B26C4324128DF80540019B12
:10753000DAB262F30700C3F3072262F30F20C3F34A
:10754000074363F3174005B030BD30B5C0F30745BE
:1075500085B0EB1A01901046DCB2FFF7AFFFC0EB2D
:10756000801300EB830004440020E4B26C43241237
:107570008DF80640019BDAB262F30700C3F30722DD
:1075800062F30F20C3F3074363F3174005B030BD28
:1075900030B585B09DF82040C0F307250190104616
:1075A0001C1BFFF78BFF2C44E4B2201AC0B26843C7
:1075B00000128DF805000020019BDAB262F307008B
:1075C000C3F3072262F30F20C3F3074363F31740AB
:1075D00005B030BD30B585B09DF82040C0F30745FB
:1075E000019010461C1BFFF769FF2C44E4B2201ADF
:1075F000C0B2684300128DF806000020019BDAB289
:1076000062F30700C3F3072262F30F20C3F30743BB
:1076100063F3174005B030BD1FB5019010461C46FE
:10762000FFF74CFF20448DF804000020019BDAB2E4
:1076300062F30700C3F3072262F30F20C3F307438B
:1076400063F3174004B010BD1FB59DF818400190BA
:1076500010461C1BFFF732FFE4B2201A8DF804001D
:107660000020019BDAB262F30700C3F3072262F342
:107670000F20C3F3074363F3174004B010BD0000AD
:1076800008B5082218210348FFF70EF80022024B24
:107690001A7008BDB02F00208A1F002084B004B0EB
:1076A000FFF78EBB2DE9F74F334D00EB0017EB19B9
:1076B0005B5C8346FF2B8A462AD000262F4A17445C
:1076C0004FF0000906EB061403F13808291905EB01
:1076D0004808144411F801EBBEF1FF0F0ED0F0B2D0
:1076E000834518D15FFA89F0824514D117F80A0052
:1076F0002030FF2828BFFF2007F80A0009F1010900
:10770000B9F1110F04F10104E4D10136072ED7D1EC
:1077100003B0BDE8F08F0EF1380E05EB4E0E9EF86B
:1077200007C098F807009EF808E0A0EB0C0098F856
:1077300008C00191ACEB0E0C1FFA8CFC0CFB0CFC8E
:1077400000FB00C080B20093FFF73FFB2828009B9E
:1077500001990A4AD2D8C0F128001FFA80FC20788B
:10776000BCF1100F94BF6044103080B2FF2828BFD6
:10777000FF202070C2E700BF440D00208C1F0020B6
:10778000FFF77EBF10B5084C35232046032200F8D2
:10779000013B0649F8F7E4FE4FF68073A380BDE88D
:1077A0001040FFF76DBF00BFB02F002096E4000827
:1077B0000020704770B504460E461546FFF7F8FFE7
:1077C000054B04EB04141C44A35DFF2B1EBF2B547C
:1077D0000130C0B270BD00BF440D0020014BDB681A
:1077E000184700BF14EC000808B5074B074A18708B
:1077F000074B1B78C3F301031370FFF7EFFF03225E
:10780000044B1A7008BD00BFD70F0020D80F00200E
:10781000B02F0020D90F00205E2817B406DC054CDD
:107820006468A446019403B010BC604703B010BC68
:10783000704700BF14EC00082DE9F04F0478824631
:1078400004EBC40304EB4304E4B204F11307FFB2F6
:107850005F2FBB4628BF4FF05F0B2E4D2E4A2E796F
:1078600089B07308168803915E43C6F30723029319
:107870002A4B03EB440803F23519E3B29B4506D8C3
:107880005E2F8CBF0020012009B0BDE8F08F14F8F6
:1078900009209AF801301A4237D098F8782098F8E1
:1078A0007710203A92B202FB02F0703989B201FBE4
:1078B000010080B205920491FFF787FA029B95F8C8
:1078C00001C00093AB7895F803E0059A04994CEA5F
:1078D000032C12B2034609B24CEA0E40039EB04795
:1078E000C0F307238DF81C00C0F307408DF81D304E
:1078F0008DF81E000798FFF7D1FEC0F30743C2B210
:10790000C0F307212046FFF787FF08F10208013482
:10791000B3E700BFB02F0020B82F0020440D002097
:107920000149FFF789BF00BF917500080149FFF7C2
:1079300083BF00BFD57500080149FFF77DBF00BFB9
:10794000157000080149FFF777BF00BF49760008AE
:107950002DE9F04F0478824604EBC40304EB4304A2
:10796000E4B204F11307FFB25F2FBB4628BF4FF00C
:107970005F0B254D254A2E7985B073081688019135
:107980005E43C6F307230093214B03EB440803F245
:107990003519E3B29B4506D85E2F8CBF002001202D
:1079A00005B0BDE8F08F14F809209AF801301A42AA
:1079B00025D0AB78687895F803C098F8782098F8C7
:1079C000771040EA0320203A7039009B40EA0C40CF
:1079D000019EB047C0F307238DF80C00C0F30740A9
:1079E0008DF80D308DF80E000398FFF757FEC0F3A9
:1079F0000743C2B2C0F307212046FFF70DFF08F18D
:107A000002080134C5E700BFB02F0020B82F0020C6
:107A1000440D00200149FFF79BBF00BF057500081A
:107A20000149FFF795BF00BF4B7500080149FFF7FB
:107A30008FBF00BF477000080149FFF789BF00BF33
:107A4000197600082DE9F74F0478074604EBC403C4
:107A500004EB4304E4B204F113095FFA89F9B9F1C4
:107A60005F0FCA46884628BF4FF05F0A1D4E1E4A68
:107A70003579DFF878B0AB08158803FB0555C5F3F9
:107A80000725E1B28A4507D8B9F15E0F8CBF002007
:107A9000012003B0BDE8F08F14F80B207B781A4268
:107AA0001DD0B07873782A4643EA0023F07843EA81
:107AB0000040C047C0F307238DF80400C0F307401F
:107AC0008DF805308DF806000198FFF7E7FDC0F34B
:107AD0000743C2B2C0F307212046FFF79DFE0134E1
:107AE000CFE700BFB02F0020B82F0020790E002074
:107AF0000149FFF7A7BF00BF796E00080149FFF7F2
:107B0000A1BF00BFD16E00080149FFF79BBF00BFB6
:107B1000296F00080149FFF795BF00BF516F0008AA
:107B20000149FFF78FBF00BF896F00080149FFF7C8
:107B300089BF00BFC16F00080149FFF783BF00BFC5
:107B4000997100080149FFF77DBF00BFF971000876
:107B50002DE9F04F2E4E04782E4A357904EBC403FC
:107B600004EB4304AB081588E4B25D4304F113074A
:107B7000C5F30725FFB2814605F1400087B05F2FAE
:107B8000C0B20391BA4628BF4FF05F0AFFF754F91D
:107B900080384FFA80FB2846FFF74EF980384FFABD
:107BA00080F80296E3B29A4506D85E2F8CBF00207B
:107BB000012007B0BDE8F08F174AA15C99F80120B9
:107BC000114223D0029A009550789278594640EAA3
:107BD0000220029A039E92F803C0424640EA0C40FB
:107BE000B047C0F307238DF81400C0F307408DF8A9
:107BF00015308DF816000598FFF750FDC0F30743C8
:107C0000C2B2C0F307212046FFF706FE0134C9E7E0
:107C1000B02F0020B82F0020790E00200149FFF777
:107C200097BF00BF957000080149FFF791BF00BFE3
:107C3000E57000080149FFF78BBF00BF35710008F0
:107C40002DE9F04F0478384D04EBC40304EB4304F2
:107C5000E4B22F7904F11306F6B27B1C5F2EB24614
:107C600028BF4FF05F0AB3F5807F08BFFF234FF6B0
:107C7000FF778046B7FBF3F785B0DFF8B0B0DFF8E9
:107C8000B0900191E0B2824506D85E2E8CBF0020F4
:107C9000012005B0BDE8F08F14F80B2098F80130F2
:107CA0001A422FD099F80030DFF888C0013B5BB250
:107CB0001A0629D53A462979A8780131B1F5807F8D
:107CC00008BFFF216B78514343EA0023E878C1F3F2
:107CD0000F2143EA0040019B9847C0F307238DF82A
:107CE0000C00C0F307408DF80D308DF80E0003989E
:107CF000FFF7D4FCC0F30743C2B2C0F3072120460C
:107D0000FFF78AFD0134BDE713F80C20824209D148
:107D100003F10C0209EB42025178927841EA022207
:107D2000BA42C8D3013BC3E7B02F0020790E002030
:107D3000BC2F0020CD2F00200149FFF781BF00BFDD
:107D4000617200080149FFF77BBF00BF9372000812
:107D50002DE9F04F0C78824604EBC40304EB430496
:107D6000E4B204F11307FFB25F2F3B4628BF5F2345
:107D70008B46454D8DB004932B7805920393434B6E
:107D8000029503EB440803F235130693049AE3B219
:107D90009A4206D85E2F8CBF002001200DB0BDE8AE
:107DA000F08F069BE25C9BF801301A4220D0032240
:107DB00037490AA8F8F7D4FB029B0AF101061E44D2
:107DC000D146002303995FFA89F2914214D8314ACF
:107DD000D07843431B128DF82A300A98FFF75EFCD7
:107DE000C0F30743C2B2C0F307212046FFF714FDDA
:107DF000013408F10208C9E716F8012B98F877005A
:107E000098F878C0801AF27980B2ACEB020C1FFAB5
:107E10008CFC0FFA8CF20CFB0CFC01B200FB00C0D6
:107E200080B2099308910792FEF7CFFF029B09F1F8
:107E30000C0E03EB4E0E9EF801C0164B9EF802E0AE
:107E4000079A4CEA0E2C93F804E0099B0EF1010E00
:107E5000BEF5807F08BF4FF0FF0E0CFB0EFC8DF8C7
:107E60002A30CCF30F23009308990346059D0A9806
:107E7000A847C0F307238DF829308DF8280009F1B1
:107E80000109C0F307439DE7BC2F0020440D0020EB
:107E9000B12F0020B02F0020054B01461B78054A6A
:107EA000013BB3F1FF3F08BF0023D8B2FFF750BF3B
:107EB000BC2F0020C77200080146024A0020FFF7CD
:107EC00047BF00BFC7720008054B01461B78054A33
:107ED000013BB3F1FF3F08BF0023D8B2FFF738BF23
:107EE000BC2F00200F7300080146024A0020FFF754
:107EF0002FBF00BF0F730008054B01461B78054AD2
:107F0000013BB3F1FF3F08BF0023D8B2FFF720BF0A
:107F1000BC2F0020857300080146024A0020FFF7AD
:107F200017BF00BF85730008054B01461B78054A43
:107F3000013BB3F1FF3F08BF0023D8B2FFF708BFF2
:107F4000BC2F0020FD7300080146024A0020FFF705
:107F5000FFBE00BFFD730008054B01461B78054AB4
:107F6000013BB3F1FF3F08BF0023D8B2FFF7F0BEDB
:107F7000BC2F0020497400080146024A0020FFF788
:107F8000E7BE00BF497400082DE9F34104781E4A9A
:107F900004EBC40304EB4304064653789078E4B240
:107FA00043EA002304F11305D078EDB25F2D43EAD4
:107FB00000402F4628BF5F27FFF770FBDFF84C809B
:107FC000C0F307238DF80400C0F307408DF8053097
:107FD0008DF80600E3B29F4206D85E2D8CBF0020CC
:107FE000012002B0BDE8F08114F8082073781A422D
:107FF00008D09DF806309DF804209DF80510204615
:10800000FFF70AFC0134E5E7B02F0020790E0020CD
:108010002DE9F0430478DFF8BC9004EBC40304EBD3
:108020004304E4B204F1130585B0EDB25F2D4FF0C7
:10803000030209F10101064601A82F4628BF5F2768
:10804000F8F78EFA99F801808DF804800198FFF70F
:1080500025FBC0F307238DF8093099F804308DF81B
:10806000080098448DF80480C0F307408DF80A009A
:108070000198FFF713FBDFF86080C0F307238DF84A
:108080000C00C0F307408DF80D308DF80E00E3B200
:108090009F4206D85E2D8CBF0020012005B0BDE8B0
:1080A000F08314F808307278134211D0DB0743BF15
:1080B0009DF80E309DF80C209DF80D109DF80A30AB
:1080C0005CBF9DF808209DF809102046FFF7A4FB2F
:1080D0000134DCE7B02F0020790E00202DE9F74FA6
:1080E0000478204D04EBC40304EB4304E4B204F130
:1080F0001306F6B25F2E80464FF0030205F1010130
:108100006846B246DFF8609028BF4FF05F0AF8F784
:1081100027FA2F79A9F1BD0BBF08E3B29A4506D81B
:108120005E2E8CBF0020012003B0BDE8F08F14F854
:10813000092098F801301A4212D01BF814306A78DE
:108140001B0903FB07238DF800300098FFF7A6FA00
:10815000C0F30743C2B2C0F307212046FFF75CFB20
:108160000134DAE7B02F0020790E00202DE9F74F17
:108170000478214D04EBC40304EB4304E4B204F19E
:108180001306F6B25F2E80464FF0030205F101019F
:108190006846B246DFF8649028BF4FF05F0AF8F7F0
:1081A000DFF92F79A9F1BE0BBF08E3B29A4506D8D3
:1081B0005E2E8CBF0020012003B0BDE8F08F14F8C4
:1081C000092098F801301A4213D01BF8143007FB2D
:1081D00003F26B7803EB52138DF800300098FFF731
:1081E0005DFAC0F30743C2B2C0F307212046FFF790
:1081F00013FB0134D9E700BFB02F0020790E002017
:108200002DE9F7430478DFF8B89004EBC40304EBDE
:108210004304E4B204F11305EDB25F2D4FF0030205
:1082200009F10101064668462F4628BF5F27F8F787
:1082300097F9224B99F804001B88C0085843C0F3F3
:108240000720FEF7F9FDA0F180035BB2002BBCBF55
:10825000C0F1800043B299F803805B00DBB208FBF9
:1082600003F31B128DF802300098FFF717FADFF8BE
:108270005480C0F307238DF80400C0F307408DF845
:1082800005308DF80600E3B29F4206D85E2D8CBF04
:108290000020012003B0BDE8F08314F808207378B3
:1082A0001A4208D09DF806309DF804209DF805106C
:1082B0002046FFF7B1FA0134E5E700BFB82F0020F0
:1082C000B02F0020790E002037B5154B04469A7860
:1082D00059788DF80120DA788DF80220FEF79AFDA2
:1082E0004FF4B47201F1B405B5FBF2F302FB135382
:1082F0005B1A48BF033300F003009B1003FB00131D
:108300008DF800300098FFF7C9F9C0F30743C2B2F7
:10831000C0F30721204603B0BDE83040FFF77CBA28
:10832000B02F00202DE9F0410478064604EBC40389
:1083300004EB4304E4B2837804F11305EDB22BBBE4
:108340001B4B0A211B791B4A1033FF2B28BFFF232D
:1083500012885343C3F30F23B3FBF1F201FB123333
:108360009BB26BB9FEF756FD5F235843124B0012C8
:108370000344727893F835311A4201D0FFF7A4FF15
:108380005E2D8CBF00200120BDE8F0815F2D2F46BF
:1083900028BF5F27DFF82480A742F1DD727814F848
:1083A00008301A4202D02046FFF78EFF0134F3E76F
:1083B000B02F0020B82F0020440D0020790E00209F
:1083C00013B50446FEF726FD8DF80000FEF722FDEA
:1083D0000B4B40F35700DB787F308DF802308DF87F
:1083E00001000098FFF75AF9C0F30743C2B2C0F387
:1083F0000721204602B0BDE81040FFF70DBA00BFCC
:10840000B02F00202DE9F0410478064604EBC403A8
:1084100004EB4304E4B2837804F11305EDB233BBFB
:108420001C4B1D4A1B7912881033FF2B28BFFF23DA
:1084300053430522C3F30F23B3FBF2F202EB820294
:108440009B1A9BB26BB9FEF7E5FC5F235843134BB5
:1084500000120344727893F835311A4201D0FFF7C5
:10846000AFFF5E2D8CBF00200120BDE8F0815F2DA5
:108470002F4628BF5F27DFF82880A742F1DD7278FA
:1084800014F808301A4202D02046FFF799FF013451
:10849000F3E700BFB02F0020B82F0020440D0020CC
:1084A000790E00202DE9F7430478DFF8B89004EB4B
:1084B000C40304EB4304E4B204F11305EDB25F2DF1
:1084C0004FF0030209F10101064668462F4628BF16
:1084D0005F27F8F745F8224B99F804001B88C0087D
:1084E0005843C0F30720FEF7A7FC0C22A0F180033D
:1084F0005BB2002BBCBFC0F1800043B25B00DBB2BB
:10850000534399F8018008EB13288DF800800098F8
:10851000FEF756FCDFF85080C0F307238DF8040007
:10852000C0F307408DF805308DF80600E3B29F4296
:1085300006D85E2D8CBF0020012003B0BDE8F0837B
:1085400014F8082073781A4208D09DF806309DF878
:1085500004209DF805102046FFF75EF90134E5E799
:10856000B82F0020B02F0020790E0020014B9B680F
:10857000184700BF14EC00082DE9F04F037885B0D0
:1085800003EBC30203EB42035FFA83FB0BF1130916
:108590005FFA89F94B465F2B28BF5F2300938378EE
:1085A00082464BB1002211461046FFF7DFFF7722CB
:1085B00000213A48F8F74AF89AF800306BB9384C7D
:1085C000208802F05AFA18288CBF01220022354B6D
:1085D0001A7002D902F04CFA208000252C462F4652
:1085E00002E0122F52D800242F4A05EB051802EBA7
:1085F000080319191B5D01915B453FD300998B421C
:108600003CD2134493F835219AF8013001371A42CD
:10861000FFB233D0214B254A984418F80460A6F1E4
:10862000550323EAE373C3F1AA038DF80830937866
:10863000D2788DF8093006F1AA03FF2B28BFFF235B
:1086400003EB43030233DBB253431B128DF80A30B2
:108650000298FFF723F8C0F30743C2B2C0F3072123
:1086600001980078FFF7D8F80E4B1B7833B1013E24
:10867000B6F1FF3F08BF002608F804600134E4B2F9
:10868000112CB1D10135EDB2072DAAD1B9F15E0F90
:108690008CBF0020012005B0BDE8F08F8C1F0020AA
:1086A00004200020891F0020440D0020B02F00204E
:1086B000544B2DE9F04FDC7887B004EB4406B6103C
:1086C000F3B20293FF23B3FBF4F301938378DFF853
:1086D000488163B1002211461046FFF747FF772219
:1086E00000214948F7F7B2FF002388F8003000273F
:1086F000464DDFF814B12B7801332B70D9464FF07B
:10870000000A98F800205FFA8AF31A4362D10393B3
:10871000F8F71EF83E4B9842039B5BDC8BF8004059
:1087200004AA39461846FFF745F880B199F80020A9
:10873000029B9DF810009A425BD9931B7343A21BC6
:1087400093FBF2F32246DBB21946FFF765F80AF114
:10875000010ABAF1070F09F11109D2D10137FFB2AD
:10876000112F0BF1010BC9D12B78019A934204BF51
:1087700000232B7098F800300133DBB21C2B3ED95C
:10878000002388F800300623224D661E2946112258
:108790001D48062B05D190F86670BC4208BF80F8D2
:1087A000666011F8117C013AA74224BF01F8116CF0
:1087B0000C7012F0FF0201F1010100F10100E8D19B
:1087C000013B13F0FF03A5F11105DFD1002007B035
:1087D000BDE8F08F99F80020002AA1D094429FD9DB
:1087E00029780198814204BF02F1FF3289F8002004
:1087F00096E76243B2FBF6F20023D2B2A4E788F810
:108800000030E3E7B02F00208C1F0020881F0020DD
:1088100054555505F21F00208B1F00202DE9F04F05
:1088200085B0074688461646FDF780F88146002841
:108830004AD0002E4BD002AA41463846FEF7BAFF76
:108840000546324C23782B44082B22DDC5F1080A5B
:10885000691C52462144601CF7F782FE05F10901AC
:108860005246214404F10900F7F77AFE04EB450172
:108870004FEA4A02193104F11900F7F771FE05F1C8
:1088800011015246214404F11100F7F769FE84F802
:1088900000A000221146964694F800C0D0B200EB2A
:1088A0000C03DBB28542019313D86544EDB201B1EC
:1088B00025704EB1164B1B7803F0FC037C2B03D1C3
:1088C00041463846FEF7EEFE05B0BDE8F08F35466E
:1088D000B7E702AB13F802A0019B0AF13801E018D8
:1088E0000C4B80F811A003EB4101019B91F807B0FC
:1088F0000C33097A04EB4303417280F801B0013272
:1089000083F801E083F802E04946C7E7062000202B
:10891000B02F0020440D00202DE9F04F924B89B07C
:108920001B7801908342914F45D1914A3B78127850
:1089300003F003039B1A18BF01238E4DAB706A78B6
:108940007B799A4205D00022114610466B70FFF7E2
:108950000DFE019B2C2B37D8DFE813F02F003800D9
:108960004C005000540058005C0060006400680037
:108970006C007000740078007C0080008400880027
:108980008C009000940098009C00A000A400A80017
:10899000AC00B000B4001601C201430247024B0212
:1089A0004F02530257025B025F02630267026B02CF
:1089B0006F02730277020123BFE7A87848B1002253
:1089C00011461046FFF7D2FD002002E06948FFF78C
:1089D000DBFA684B1A7801321A7040B90221664AF4
:1089E0009B7811701BB9019B0BB90323137009B05D
:1089F000BDE8F08F5F48FFF70BFBEAE75D48FFF744
:108A00006DFBE6E75B48FFF7B1FBE2E75948FFF78C
:108A1000F7FBDEE75748FFF76BF8DAE75548FFF753
:108A20006DF8D6E75348FEF7F5FFD2E75148FEF759
:108A3000F7FFCEE74F48FEF773FFCAE74D48FEF752
:108A400075FFC6E74B48FFF75FF8C2E74948FFF7F5
:108A500061F8BEE74748FFF763F8BAE74548FFF714
:108A600065F8B6E74348FEF767FFB2E74148FEF70F
:108A7000DDFFAEE73F48FEF7DFFFAAE73D48FEF720
:108A800061FFA6E73B48FFF7C9F8A2E73948FFF7BF
:108A9000CBF89EE73748FFF7CDF89AE73548FFF760
:108AA00041FC96E73348FFF7ADFC92E73148FFF70A
:108AB000F9FC8EE72F48FFF73FF88AE72D48FFF7CC
:108AC00041F886E72D4B28782D4E01301968326821
:108AD00000EBC00400EB44009142C4B2984630D988
:108AE000FEF798F94FF05F0909FB00F9254B4FEAB3
:108AF00029294B4493F835216B781A4221D0FEF78F
:108B000089F9810722D50023ADF818308DF81A3085
:108B10000698FEF7C3FDC0F30743C2B2C0F30721B6
:108B20004846FEF779FE3B794FF4FA721033FF2B7B
:108B300028BFFF231B09B2FBF3F3D8F8002013442E
:108B400033605E2C8CBF0020012042E7FEF762F903
:108B50008DF81800FEF75EF940F357007F308DF86E
:108B60001900FB78D2E700BFD70F0020B02F0020FC
:108B7000D80F0020D40F0020D90F0020B82F0020DC
:108B80008C210020440D0020B34BB44A18681168B2
:108B90000092884202933FF617AFAB78B04E9BBB72
:108BA0002C78DFF8D4B204EBC40304EB4304E4B242
:108BB00004F113095FFA89F9B9F15F0FCA4628BFBA
:108BC0004FF05F0A04EB4408B044E3B29A4553D82F
:108BD000B9F15E0F40F23D815F24A14D013C05F1EA
:108BE00003055BD1FEF716F983075DD586F81A41B8
:108BF00086F81B4186F81C41FEF724FB009B1B688E
:108C00001844029B1860DFE600220024114610463B
:108C1000FFF7ACFCB046A146FEF7FCF882070BD587
:108C200088F8009088F8019088F8029001345F2C51
:108C300008F10308F0D1B3E7FEF7ECF88DF8140063
:108C4000FEF7E8F8FB7840F357007F308DF81630D8
:108C50008DF815000598FEF7B3F804EB440B06F801
:108C60000B0006EB0B0AC0F30723C0F307408AF89A
:108C700001308AF80200D9E714F80B206B781A4209
:108C800008D098F8023098F8002098F80110204693
:108C9000FEF7C2FD08F10308013496E703222946D6
:108CA000E81EF7F75DFC99E7FEF7B4F88DF81800B9
:108CB000FEF7B0F8FB7840F357007F308DF81A309C
:108CC0008DF819000698FEF77BF8C0F3072386F8A5
:108CD0001A01C0F3074086F81B3186F81C018BE7A8
:108CE000AB7823B1002211461046FFF73FFC2878ED
:108CF000013000EBC00300EB4300C3B20393574BBA
:108D00001A68584B1B689A4256D9B8787B78564DEA
:108D100043EA0023F878554F43EA0040FEF7BEFCD3
:108D2000C3B20093C0F3072BC0F30746AA46B94667
:108D300007240295029B19F8018B13F8010B02938B
:108D4000B8F1000F3BD03346009A5946FEF764FD58
:108D500033465946009A9AF81000FEF75DFD013C33
:108D600099F8003014F0FF0409F8013C0AF1FF3AC9
:108D7000E0D1FB79E8795BB33346009A5946FEF7B8
:108D80004BFD33465946009A687AFEF745FDFEF7DB
:108D900041F810F0030F0CBF01230023FB71344B8B
:108DA0001135AB4207F10807C0D1FEF74BFA2B4B48
:108DB0001B6818442B4B1860039B5E2BC2E643468E
:108DC00042464146FEF728FD434642464146C2E739
:108DD000234622462146FEF71FFD23462246214612
:108DE000D2E72448FFF7C8FBF3E52248FFF760FC11
:108DF000EFE52048FEF7A0FFEBE51E48FEF7A2FFD7
:108E0000E7E51C48FFF748F8E3E51A48FFF754F890
:108E1000DFE51848FFF758F8DBE51648FFF764F878
:108E2000D7E51448FFF768F8D3E51248FFF774F860
:108E3000CFE51048FFF778F8CBE50E48FFF784F848
:108E4000C7E50C48FFF788F8C3E50A48FFF794F830
:108E5000BFE50120BDE500BF90210020B82F002014
:108E60002F20002094210020440D00204C210020C0
:108E7000BB0D0020D40F0020790E00200120704788
:108E800008B5FFF7FBFF08BD08B5017801EBC1038A
:108E900001EB4301C9B2A1F113005F2928BF5F2193
:108EA000C0B2FAF765FF08BD2DE9F8433B4E3378B1
:108EB00003F00303012B4DD1394C0025206801F04C
:108EC000E3FD804601F09AFD3649206091F800E00C
:108ED000AC467446C8F57F47FF37EBB29E4513D8C2
:108EE000BCF1000F00D00C702F4B1B7823BB3378E4
:108EF00013F0030500D09D082C4C2378032B29D8B0
:108F0000DFE803F01C2A3A3F05F10C0201EB4202B4
:108F1000537892F80290013543EA09239F4225BF16
:108F200043449BB204F1FF3453702DBF1B0AE4B2DB
:108F30004FF0010C9370D0E70025DDE700221C4BB9
:108F400018491A701B4B292218601B48F7F708FBB9
:108F500001232370BDE8F8832846FFF7DDFC002DD0
:108F6000F8D0134B1B78052B01D1FFF789FFBDE823
:108F7000F8430F48FFF788BF2846BDE8F843FEF7DF
:108F800033BC0E4B1B780BB1FEF77AFB094B18680C
:108F900001F07AFD0F28DDD90023DAE7B02F002099
:108FA000842100200620002088210020D90F0020E5
:108FB000D40F0020B82F0020BC2F00208A1F0020D3
:108FC00008B5274B1B6898474FF0FF330021254A0F
:108FD000117053769376D376137753779377D3774D
:108FE00082F8203082F8213082F8223082F8233053
:108FF00082F8243082F8253082F8263082F8273033
:1090000082F82830184A117053769376D376137706
:1090100053779377D37782F8203082F8213082F823
:10902000223082F8233082F8243082F8253082F80A
:10903000263082F8273082F82830FCF7B3FB18B9C5
:10904000FCF734FCFEF79EFBFEF728FA074B1B7873
:1090500013F0FC0F03D1BDE80840FEF793BB08BD39
:1090600014EC0008BC2F002006200020B02F0020A8
:1090700070B50646054D38B12C782CB92046FFF75F
:109080004BFC2046FEF7B0FB2E7070BD88210020FF
:10909000044A137883F0010313700022024B1A7004
:1090A000FEF7F4B9B02F0020D90F00200020FFF701
:1090B000EFBF0120FFF7ECBF064B1A7812F0030256
:1090C00004BF05490A7001211A7861F301021A7080
:1090D000704700BFB02F0020D90F002008B5FFF760
:1090E000EBFFBDE808400120FEF7D0B908B5094BF9
:1090F00000201A7892071EBF0021074A11701A78C3
:109100006FF301021A70FFF707FCBDE8084000206A
:10911000FEF76ABBB02F0020D90F002008B5FFF77B
:10912000E5FFBDE808400120FEF7B0B9024B187812
:1091300000F00300704700BFB02F00200A4A1378E8
:1091400013F0030F0ED048B9012060F387031370AA
:109150000022064B08461A70FEF798B92C2888BFE3
:109160002C20F2E7704700BFB02F0020D90F00205D
:109170000021FFF7E3BF0121FFF7E0BF014B1878A3
:1091800080087047B02F0020054B01461B789B08D4
:1091900001332D2B34BF18460120FFF7CFBF00BF8E
:1091A000B02F00200120FFF7EFBF0000064B014663
:1091B0001B78C3F38503013B13F0FF0314BF18466C
:1091C0002C20FFF7BBBF00BFB02F00200120FFF70E
:1091D000EDBF000030B4084C2578AD0709D0442A13
:1091E00028BF44226070A170E270184630BCFEF7C0
:1091F0004DB930BC704700BFB02F00200023FFF7EF
:10920000E9BF0000014B5878704700BFB02F002025
:10921000014B9878704700BFB02F0020014BD878E1
:10922000704700BFB02F0020054910B44C780346AA
:10923000CA7804F10800897810BCFFF7CBBF00BFE3
:10924000B02F00200120FFF7EFBF0000054910B448
:109250004C780346083CCA78A0B2897810BCFFF766
:10926000B9BF00BFB02F00200120FFF7EFBF000003
:1092700010B4064C0346A178E2781031FF2928BFCC
:10928000FF216078C9B210BCFFF7A4BFB02F002047
:109290000120FFF7EDBF000010B4064C0346A17893
:1092A000E278103921EAE1716078C9B210BCFFF7A9
:1092B00091BF00BFB02F00200120FFF7EDBF0000DD
:1092C00010B4064C0346E278A1781132FF2A28BF79
:1092D000FF226078D2B210BCFFF77CBFB02F002015
:1092E0000120FFF7EDBF000010B4064C0346E27802
:1092F000A178113A22EAE2726078D2B210BCFFF78C
:1093000069BF00BFB02F00200120FFF7EDBF0000B4
:10931000024B18710020FEF7B9B800BFB02F002033
:10932000014B1879704700BFB02F0020044A137911
:109330004033FF2B28BFFF231371FEF7A7B800BFF0
:10934000B02F00200120FFF7F1BF0000034A13797E
:10935000403B23EAE3731371FEF798B8B02F002067
:109360000120FFF7F3BF00000022014B1A70704785
:1093700098210020F0B50B4C45002F18E61996F8FF
:1093800001C08C4505D1E75D974202D1B6789E4277
:1093900007D001270544044E6019377041706255AB
:1093A0008370F0BDE52F002098210020F8B5054618
:1093B0000E461746002420463B46324629460134D5
:1093C000FFF7D8FF5F2CF6D1F8BD000010B5054CB3
:1093D00023782BB15F21044800F0B2F800232370FA
:1093E00010BD00BF98210020E52F002000B11047DC
:1093F0000847000038B54D790446BDB9FCF7BAF806
:10940000A4F5F043203B00F02200142B3AD8DFE80B
:1094100003F00B0F14171A1D202326292C2F333588
:10942000370D0D0D0D0D0D00FFF743FE284638BD1D
:10943000154A1649FFF7DAFFF8E7144A1249F9E727
:10944000134A1449F6E7134A1149F3E7124A13493C
:10945000F0E7124A1049EDE7114A1249EAE7114ACA
:109460000F49E7E7104A1149E4E7104A0E49E1E7DE
:109470000120FFF780FED9E70520FAE70D20F8E785
:109480001220F6E70125D1E7CD910008A59100084B
:109490006992000845920008B9920008919200086C
:1094A00009930008E19200086193000845930008C1
:1094B00070B5072301264FF400444FF000451B4AC6
:1094C00006FA03F10142946119D0052100BF00BFE3
:1094D00000BF00BF00BF00BF0139F7D1956100BFD9
:1094E00000BF00BF00BF00BF00BF00BF00BF00BF84
:1094F00000BF00BF00BF13F1FF33E1D270BD00BF5A
:1095000000BF00BF00BF00BF00BF00BF00BF00BF63
:1095100000BF00BF00BF0521956100BF00BF00BFB5
:1095200000BF00BF00BF0139F7D1E4E700040040ED
:1095300001224FF40041014803F086BC00040040C2
:10954000F8B5164D04462B780E461BB9FFF7F0FF11
:1095500001232B70302383F3118800235F1CDBB2BF
:10956000B3420CD34FF4A86300BF00BF00BF00BFDD
:1095700000BF00BF013BF7D183F31188F8BD03EBB7
:109580004303E518E05CFFF793FF6878FFF790FF6F
:10959000A878FFF78DFF3B46E0E700BF9921002048
:1095A00008B52820FDF732F808BD08B52520FDF7DD
:1095B0002DF8252801D0002008BD2620FDF726F82B
:1095C0001028F8D12720FDF721F8A0F131035842E7
:1095D0005841F1E710B5041E14BF2521FF212520B5
:1095E000FDF77CF8002C14BF1021FF212620FDF789
:1095F00075F8002C18BF3121BDE8104008BFFF21CD
:109600002720FDF76BB87047704710B50446FFF789
:10961000FBFFE1B22820BDE81040FDF75FB808B5B8
:109620000020FFF7D7FF0020FFF7EFFF00F0FAFD63
:1096300000F08EFEBDE808400120FFF7CBBF08B563
:10964000FFF7E1FFFFF7ACFFFFF7DEFFFFF7ADFF2E
:1096500018B9BDE80840FFF7E2BF08BDFFF726BD17
:1096600008B54B794BB1A0F5EE427F2A03D8C0B2C2
:1096700000F07AFE0023184608BD0123FBE7FF2314
:109680000370704710B503780446013B032B0BD8D9
:10969000DFE803F0020B1215FFF7C0FD4423C0EB17
:1096A0000020B0FBF3F0607010BDFFF73FFD002815
:1096B000F9D0FFF763FDF6E7FFF732FEF3E7FFF7B8
:1096C000A1FD6070FFF7A4FDA070EDE738B5037849
:1096D0000446013B032B2CD8DFE803F002111E23C4
:1096E000FFF790FD0546FFF793FD4422637801469E
:1096F0005A43A8B2120ABDE83840FFF77FBD43784D
:109700001BB9BDE83840FFF7F1BCFFF7D5FC607826
:10971000BDE83840FFF72CBD4078BDE83840FFF782
:10972000F7BD45788478FFF779FD21460246284643
:10973000E1E738BD024610F8023B082B05D0092BA3
:1097400005D0072B05D1FFF7C1BFFFF79BBFFEF781
:1097500017B8FF231370704708B54378032B03D164
:10976000BDE80840FFF7E6BFFFF789FF08BD2DE918
:10977000F04104460F46FAF753FE002840F0B1804E
:109780002378013B122B4BD8DFE803F00A14455F26
:10979000656F7272724A4A777B818A939699A200AA
:1097A000002363700C23A37039462046BDE8F041C6
:1097B00001F08EBD6378013B032B31D8DFE803F065
:1097C000020C0F2301F01AF9030EA370030CE370CF
:1097D000030A23716071E7E7FFF7E2FEF4E725462D
:1097E000A67804F11B08062EDED8F0B2FCF76EFB5B
:1097F000030CEB70030A2B7168710335454506F1C4
:109800000106F0D1D0E70023A370E3700423237195
:1098100005236371C8E76378022B04D0052B10D0B1
:10982000FF232370C0E7E378A07840EA0320237980
:1098300040EA0340637940EA036000BAFFF7E5FEBF
:10984000B2E7A078FFF70AFFAEE7E278A178607888
:1098500000F0BDFCBCE722796379A17843EA0223DA
:109860006078E27800F0C9FC9EE700F0DBFC9BE743
:1098700039462046FFF770FF96E700F02EFD607036
:1098800092E700F02CFD030A6370A0708CE760780B
:10989000A378221DE17843EA002000F023FD83E74E
:1098A0006078A378221DE17843EA002000F037FDBC
:1098B0007AE700F04DFD77E700F07EFCDFE76078A7
:1098C000A378221DE17843EA002000F0CDFC6BE78D
:1098D0006078A378221DE17843EA002000F0DBFCE9
:1098E00062E7BDE8F081F0B50144884202D310463A
:1098F0001946F0BD002710F8014B4FEA031C6240E7
:1099000094184FEA021E43EB03054CEA127C14EB59
:109910000E0445EB0C054FEA421EA4184FEA431C07
:1099200043EB05054CEAD26C14EB0E0445EB0C0539
:109930004FEAC21E4FEAC31C4CEA526C14EB0E04F1
:109940004FEA022645EB0C054FEA032C4CEA126C59
:10995000A41945EB0C033A19B64646EB0303C4E7DA
:1099600038B505464879002800F0DC80A5F5E045CB
:10997000ABB2222B00F2BB80FBF72CFF6A4C013DFF
:109980002080212D12D8DFE805F04DBD551B1F5951
:10999000235D692FB5336D3771973B759F417B838D
:1099A00027612B65477F8EA9B31651C5237843F0F5
:1099B0000103237095E0637843F00803637090E03F
:1099C000237843F00203F4E7237843F00403F0E73D
:1099D000237843F00803ECE7637843F00103EDE7F5
:1099E000637843F00203E9E7237843F01003E0E7EC
:1099F000237843F02003DCE7237843F04003D8E7E3
:109A0000FBF766F9237843F08003D2E7237823F04D
:109A10000C0343F00C03CCE7637823F0030343F01B
:109A20000303CBE723786FF30003C2E763786FF398
:109A3000C303C3E723786FF34103BAE723786FF3D7
:109A40008203B6E723786FF3C303B2E763786FF35B
:109A50000003B3E763786FF34103AFE723786FF355
:109A60000413A6E723786FF34513A2E723786FF377
:109A700086139EE7FBF72CF923786FF3C71398E75B
:109A8000237823F00C0394E7637823F0030395E72E
:109A90002378C3F3800282F00102D2B262F3820320
:109AA00062F3C30385E76378DA4302F0010262F3ED
:109AB000000362F3410381E72378C3F3801282F04D
:109AC000010262F3861374E7FBF702F92378C3F30C
:109AD000C01282F0010262F3C7136AE70120FBF7AC
:109AE000E7FE2088FBF779FEFBF7F2F8002038BD8F
:109AF0000020F4E72378C3F3001282F0010262F33E
:109B0000041356E72378C3F3000282F0010262F3E4
:109B100000034EE76378C3F3C00282F0010262F3F0
:109B2000C3034BE70120E2E7702F0020F8B5174B85
:109B30001749C2081F5C174B8D5C17499B5C00F0EE
:109B400007008E5C0341054113F0010446FA00F062
:109B500005F0010500F0010602D0E120F8F76AFFE8
:109B600015B1E620F8F766FF3846FAF789FE15B119
:109B7000E620F8F7C5FF14B1E120F8F7C1FF26B1E0
:109B8000BDE8F8402C20FAF77BBEF8BD44ED000894
:109B900024ED0008C4ED000834ED00082DE9F04183
:109BA00004460E464FF00A08214F207800283DD089
:109BB000012838D16378012B0ED1A078A51CFAF7C3
:109BC0005FFE2C4635460134013DEDB2FF2DECD051
:109BD000642001F0DAFFF7E7022B04D1A078A51C7E
:109BE000F8F728FFEDE7032B04D1A078A51CF8F7C0
:109BF00087FFE6E7042B01D00134E3E72246002586
:109C000012F8023FD95D1446490706D415F1FF3515
:109C1000D8D3642001F0B9FFF8E7303B08FB0535E5
:109C200012F8013FEEE7FFF781FFCBE7BDE8F081D7
:109C30009DE400080021FFF7B1BF70472DE9F84F00
:109C4000254F3B786BB14FF0000A4FF00E0B234EBF
:109C5000DFF88C9035783B78AB4204D800233B701A
:109C60003370BDE8F88F0BFB05F309EB030405F136
:109C7000010822795FFA88F886F80080E2B122892B
:109C8000E2B94FF6FF726089904217D00121FFF7C9
:109C9000D4FF00230BFB05952B71FBF797FCBAF162
:109CA000000F09D12046FBF743F828B941F288306C
:109CB00001F06BFF4FF0010A4546CCE739F803206D
:109CC0006088A388E18842EA004043EA0141228992
:109CD000FBF7BEFBDDE700BF1522002014220020A9
:109CE000A42100207047000038B50024084B1C80D8
:109CF000FAF7D0FBA5B2A84200D838BD2846FAF73B
:109D0000CBFBC3790BB9837103720134F0E700BF59
:109D10001622002038B50D4D0D4B2C781B780D4ABE
:109D2000A3420ED032F8141081420BD1FAF7B4FBE3
:109D3000012383712B78A34203D1013404F003047F
:109D40002C7038BD013404F00304E9E7A22100209F
:109D5000A32100209A2100208B792DE9F74F002BB9
:109D600040D1224D9C46A8464FF6FF794FF0010E98
:109D70001F4A92F800B0DAB293452AD900264FF66E
:109D8000FF740A68B5F80CA00192019FF2B237F88F
:109D900012700136BA4508BF94B2002FF5D14C4578
:109DA0001DD00EFA04F444EA0C0C0EFA02F25FFA2B
:109DB0008CFC013A624511D10E2253438C8808EB8A
:109DC000030214810424147128F80370508181F86F
:109DD00007E003B0BDE8F04FFFF79CBF2F710133E0
:109DE0000E35C8E703B0BDE8F08F00BFA421002006
:109DF0001522002070B50D4B0D4E1C780D4D33789B
:109E0000A34205D1FFF71AFFBDE87040FFF76CBF12
:109E100035F81400FAF740FB014635F81400013418
:109E2000FFF79AFF04F00304E9E700BFA221002036
:109E3000A32100209A2100200023F0B51A461C46D9
:109E4000D0F800E0DDB23EF8156076B1D1F800C080
:109E5000002503E0BE4208BF01220135ECB23CF808
:109E60001470002FF6D10133ECE71AB1AC4238BFC1
:109E70000846F0BD1046FCE70F4B70B51B789BB150
:109E80000E4C208880B100F0F8FD0D4E33888342DF
:109E90000AD20C4B00251A780B4B1B789A4204D03F
:109EA000FFF7A8FF3580258070BDFFF7C7FE25802E
:109EB000BDE87040FFF718BFDC0F0020182200201B
:109EC00016220020A2210020A321002008B5002393
:109ED000064A1380064A1370064B1A78064B1A700E
:109EE000FFF702FFBDE80840FFF7A8BE18220020D8
:109EF000DC0F0020A3210020A2210020034B1A78B0
:109F00000AB1FFF7E3BF01221A707047DC0F00208F
:109F100047F650432DE9F04F984287B007460E466A
:109F200008D14D79C5B10122994B1A70284607B066
:109F3000BDE8F08F47F65143984204D14D795DB1A9
:109F4000FFF7C4FFF2E747F65243984204D14D7938
:109F500015B1FFF7D3FFE9E78E4B18788E4B1B78CE
:109F60001843FAF7FFFB0446FFF7BCFE844203D018
:109F70003188FBF757FE07464FF0000A5546FAF7BF
:109F800089FA1FFA8AF8404525D87379002B00F02A
:109F9000ED80002D00F0EA8000F06AFD7F4B188014
:109FA0007F4B1C78072C13D8621C1A7031460A228A
:109FB00003A8F6F7D5FA0E227A4B03A902FB043365
:109FC0000A221846F6F7CCFA4FF6FF7287814281D3
:109FD00085F00105AAE74046FAF75EFA4FF6FF7BE7
:109FE0004FF0000C044600685FFA8CF130F8112045
:109FF0000CF1010C974208BF1FFA81FB002AF3D134
:10A000004FF6FF70834530D0A379002B32D1604AE0
:10A010001078727994F8079094F808C0002A64D0F8
:10A02000002862D0B9F1000F0CD1012000FA0BF327
:10A0300043EA0C0C5C4B84F808C0188831289CBF9C
:10A04000322018804FF00109237A09FA01F1013911
:10A0500099420AD1514B188870B1009200F00DFD61
:10A060003228009A08D984F806901543EDB20AF117
:10A07000010A84E71046CCE700204C4BDFF834B1EE
:10A0800093F800909BF8001089450BD18442ECD0E6
:10A09000474921F8198009F1010909F003098BF8F2
:10A0A0000090E2E7424B019233F81900FAF7F4F915
:10A0B00021460090FFF7C0FE019A88B14FF00103DE
:10A0C00084428371D1D0394B1978894508D1009BDE
:10A0D000834201BF09F10101344B01F00301197002
:10A0E00009F1010909F00309CCE7B9F1000F15D115
:10A0F000012202FA01F10139614502D153B900EAA6
:10A1000002090122237A02FA0BF223EA02032372E4
:10A110004A46AAE74046FFF7FDFDF2E70CF1FF32A1
:10A120004CFA0BF112EA0C0201F001011BD1D1B182
:10A13000A188A1B10392049200F09AFC04228DF848
:10A140001020A2880DF10C08ADF80E00ADF8142017
:10A1500098E80700FBF77CF90022E271D1E740465E
:10A16000FFF76BFDF8E75FFA81F9CAE70F4B1A7842
:10A17000104B1B789A4202D0FFF73CFE28E7FFF70E
:10A180005DFD0022054B1A80FFF7AEFD20E700BF02
:10A19000DC0F00206F1600206E1600201822002011
:10A1A00015220020A421002016220020A221002038
:10A1B0009A210020A321002004207047222352006E
:10A1C00003FB0121EE2303FB001029307047032815
:10A1D00038B510D806290ED8102A0CD8FFF7EEFF94
:10A1E0000546FCF713FA000284B2681CFCF70EFA6D
:10A1F000204380B238BD0020FCE7032870B51C4620
:10A200000FD806290DD8102A0BD8FFF7D7FF05461F
:10A21000210AFCF763FAE1B2681CBDE87040FCF764
:10A220005DBA70BD2DE9F84300240025E7B212E0C5
:10A230005FFA86F94A4641463846FAF717F9013679
:10A2400003464A4641463846FFF7D7FF112EEFD165
:10A250000135072D03D000265FFA85F8E8E70134C1
:10A26000042CE2D1BDE8F883F8B51446002700F1CC
:10A2700029055618B44200D1F8BDA5F12903B3F55C
:10A280006E7F06DA2846FCF7C1F9207001350134EB
:10A29000F0E72770FAE7F8B50E461746002400F1FC
:10A2A0002905B44200D1F8BDA5F12903B3F56E7FAD
:10A2B00003DA395D2846FCF711FA01350134F0E77D
:10A2C000032810B406D8062904D8102A02D810BCD6
:10A2D000FFF77DBF002010BC70471020704740F290
:10A2E0001F4070472DE9F041144640F21E474FF0E1
:10A2F000000800F2E1355618B44201D1BDE8F08102
:10A300006FF47873EB18BB4206DC2846FCF77EF945
:10A31000207001350134EFE784F80080F9E72DE97A
:10A32000F0410E461746002440F21E4800F2E13587
:10A33000B44201D1BDE8F0816FF47873EB18434566
:10A3400003DC395D2846FCF7C9F901350134EFE734
:10A3500010B540F2E134204600210134FCF7BEF98B
:10A36000B4F5006FF7D110BD0F28F7B505464ED8EC
:10A3700040F2FF70FCF74AF9002848D140F2E1347E
:10A380002DBBCDE900552046FCF740F9661C8DF841
:10A3900000008DF80150D0B3012812D13046FCF7EF
:10A3A00035F9A71C8DF8010088B3431E022B19D87C
:10A3B0003846FCF72BF9E61C8DF8020038B38DF80F
:10A3C000035032216846FFF7E9FB3446DBE7B4F57A
:10A3D000006F1CD02046FCF719F908B9013DEDB219
:10A3E0000134CDE7042814D102243846FCF70EF9D5
:10A3F0007E1C0DF8040050B17C2804D102AB1C4433
:10A4000004F8075CDDE70134072C3746EDD103B0D3
:10A41000F0BD3E46D5E7000047F61643984210B51A
:10A420000C461BD1FBF7A6F862790D4B72B100F018
:10A43000AA00002815BF01220022352029201A7009
:10A44000FBF76AF8FBF70AF9002010BD1B78002B18
:10A4500014BF35202920FBF767F8F3E70120F4E764
:10A460001A220020F8B5144642791D469DF818704E
:10A47000284B92B11C7000F0FBFA274B188004F1B6
:10A480002003DBB2072B44D8012004F00704A040CE
:10A49000C0B2BDE8F840F8F785BB1E78A6422ED1C1
:10A4A0001D4B188800F0E9FAC72828D8AE4205F1FC
:10A4B000200415D006F12003DBB2072B06D80120BB
:10A4C00006F00706B040C0B2F8F79CFBE3B2072BDA
:10A4D00006D8012005F007039840C0B2F8F762FBE8
:10A4E0003846E4B2FAF7CCF9072C12D8012005F06F
:10A4F0000705A840C0B2BDE8F840F8F783BB04F1F7
:10A500002003DBB2072B04D8012004F00704A0408D
:10A51000F0E7F8BD1B2200201C22002013B5A0F597
:10A52000F84018380C4606283BD8DFE800F0171E24
:10A530000410252C330026230093E12347F61A410B
:10A540001A462046FFF78EFF002002B010BD2723D9
:10A550000093E52347F61B411A46F2E72623E02243
:10A56000009347F61841E123EBE72723E422009309
:10A5700047F61941E523E4E72623E222009347F654
:10A580001C41E123DDE72723E622009347F61D4126
:10A59000E523D6E72823E522009347F61E41012351
:10A5A000CFE7487918B10022024B1A70CDE701209D
:10A5B000CBE700BF1B22002047F67743984270B5D7
:10A5C00006D047F67843984229D00124204670BD32
:10A5D0004C7994B100F02CF8FAF708FC00F028F858
:10A5E000044600F02BF8054600F02EF829460246F6
:10A5F0002046FAF7FDFC0024E8E700F019F8FAF726
:10A6000001FC00F015F8054600F018F8064600F0C9
:10A610001BF8314602462846FAF7EAFCD6E74C79A1
:10A6200014B100F00BF8D7E700F008F8E7E70000F6
:10A63000014B1878704700BFDE0F0020014B1878DF
:10A64000704700BFDF0F0020014B1878704700BF34
:10A65000DD0F0020014B1860704700BF2022002052
:10A66000024B186808B10368184770472022002081
:10A6700008B5FFF7F5FF08BD084B1B686BB1084A2A
:10A68000127842B1074A92F90020002ABFBF02782F
:10A690004270062202705B68184770472022002033
:10A6A0001C110020702F0020034B1B681BB10221DE
:10A6B00001709B6818477047202200200B4B07B59C
:10A6C0001A8882420ED01880094B1B6853B10322AE
:10A6D0008DF80500000A8DF806008DF80420DB686F
:10A6E00001A8984703B05DF804FB00BF26220020B4
:10A6F000202200200B4B07B51A8882420FD0188009
:10A70000094B1B685BB104228DF80500000A8DF827
:10A7100006008DF80420DB680DEB0200984703B0BB
:10A720005DF804FB24220020202200200C4B821C18
:10A730001B7863B10B4B93F90030002BACBF0623A1
:10A740001E230020013BDBB2FF2B02D17047062302
:10A75000F7E712F8011B0029F4D00130C0B2F1E78D
:10A760001C110020702F0020F1B1114B1B789BB100
:10A77000104B93F90030002B0EDACA081D2A13D8AB
:10A780000123104401F0070103FA01F18378194213
:10A7900014BF012000207047831C083013F8012BE0
:10A7A0008A4203D08342F9D10020704701207047CC
:10A7B0001C110020702F00204FF0FF33002230B515
:10A7C000851C15F8014B8C420ED0B3F1FF3F02D12E
:10A7D000002C08BF13460132D4B2062C62B2F0D16D
:10A7E0005A1C01D01844817030BD002210B5831C62
:10A7F000083013F8014B8C4208BF03F8012C834248
:10A80000F7D110BDCB081D2B07D8184401F0070362
:10A81000012199408378194381707047CB081D2B23
:10A8200008D81844012301F007018B40817821EA00
:10A83000030181707047000010B4094C034624786E
:10A840000A463CB1074C94F90040002C02DA10BCD7
:10A85000FFF7D8BF1146184610BCFFF7ADBF00BFC9
:10A860001C110020702F002010B4094C03462478DE
:10A870000A463CB1074C94F90040002C02DA10BCA7
:10A88000FFF7CCBF1146184610BCFFF7AEBF00BFA4
:10A890001C110020702F0020074B02301B7843B1A1
:10A8A000064B93F90030002B03DA1E220021F5F746
:10A8B000CDBE0622FAE700BF1C110020702F002039
:10A8C00042784B789A421DD190F902301BB191F930
:10A8D00002209A4216D190F903301BB191F903205E
:10A8E0009A420FD190F905301BB191F905209A4297
:10A8F00008D190F9040030B191F90430181A18BF4A
:10A90000012070470120704770470000002814BFE5
:10A910000220012008B5024B1870F9F7B5FA08BDFE
:10A9200028220020032008B5024B1870F9F7ACFA72
:10A9300008BD00BF28220020FFF7E8BF012008B5AE
:10A94000024B1870F9F7A0FA08BD00BF28220020BA
:10A95000FFF7F4BF704770477047704710B5FFF7B7
:10A96000F9FF0024FBF772FBFFF7F5FFE0B2FBF7FE
:10A97000ADFA18B90134072CF8D110BD0120FCE75D
:10A9800008B501F0CDF9BDE8084000F011BF08B5E9
:10A99000F9F7D2FEBDE8084040F2A46001F0F5B836
:10A9A00008B5FAF7FDFDFAF711FEFAF7C5FDFBF75A
:10A9B0003FFD0020FFF782FE0020FFF79BFEBDE871
:10A9C0000840F9F7C5BE0000302383F31188064B19
:10A9D000DA69064B1A600023054A1360054A1360C2
:10A9E00083F31188704700BF2831002034220020F3
:10A9F0002C22002030220020FFF7E6BFD0B5302304
:10AA000083F31188134B144C144AD96923681068D6
:10AA1000C91A884212480AD9A3F58333E03B236060
:10AA20000468104B01F583312344E0310360116069
:10AA30000468002383F311884FF47A7000270A4ECC
:10AA40000A4AE0FB0167002330463946F5F7CEFBA2
:10AA50002044D0BD28310020342200202C220020A8
:10AA60003022002088598F029F860100A0860100B5
:10AA700008B5FFF7C3FF80B208BD10B50446FFF765
:10AA8000BDFF001B80B210BD10B50446FFF7B6FF36
:10AA9000001B10BDBFF34F8F0549064BCA6802F477
:10AAA000E0621343CB60BFF34F8F00BFFDE700BFF1
:10AAB00000ED00E00400FA0508B5024A024B1A60F6
:10AAC000FFF7E8FFEFBEADDEFC6F00200A4A08B5D5
:10AAD00052F8041C094B99420DD1002342F8043C62
:10AAE00083F31488064B1B6883F3088862B6054B12
:10AAF0001B689847FEE708BD00700020EFBEADDE82
:10AB000000E0FF1F04E0FF1F08B5FFF7C3FF0000D0
:10AB10000F4B10B51A78CAB901220E4C1A7020607A
:10AB200040F282324FF400714FF0804002F08CF915
:10AB30004FF480614FF0804040F2823202F084F99D
:10AB40002146BDE81040044801F058BC10BD00BFCC
:10AB500038220020E00F00208831002008B54FF097
:10AB6000FF31024801F02AFBC0B208BD9431002039
:10AB70000A464FF0FF330146014801F0C4BB00BF55
:10AB8000B83100200A464FF0FF330146014801F07A
:10AB90003BBB00BF9431002008B5034801F053FCD3
:10ABA00080F00100C0B208BD88310020194B10B5FB
:10ABB0001C786CBB012208211A701748224602F04B
:10ABC00043F922462021144802F03EF92246102182
:10ABD000114802F039F94FF47A7000F0D6FF41F6CF
:10ABE000822208210C4802F02FF940F28222202113
:10ABF000094802F029F940F282221021064802F0A9
:10AC000023F9064801F048FC4FF0FF32044B1A606C
:10AC100010BD00BF3922002000040040E4320020B3
:10AC2000E80F002001461A4810B5046801342BD102
:10AC30004C1C29D053B3174C9B0023822346032A74
:10AC400005D8DFE802F0021A1D1F0022DA60012495
:10AC5000016021F00F0001F00F019960224604FA13
:10AC600001F1586002F0F0F80A490B4801F006FCC7
:10AC7000094801F01FFC204610BD4FF48002E5E7B3
:10AC80008022E3E7054AE1E70020F5E71846F3E70D
:10AC9000E80F00203C220020E43200208000400029
:10ACA0001FB501218DF807000DF10F030DF107020B
:10ACB000034801F01AFC9DF80F0005B05DF804FB95
:10ACC000E4320020002307B501210DF107020548F9
:10ACD0008DF8073001F02BFC9DF8070003B05DF8FC
:10ACE00004FB00BFE432002008B50246024801F030
:10ACF0000DFC002008BD00BFE432002008B502466C
:10AD0000024801F014FC002008BD00BFE43200201E
:10AD100010B5074C2368013308D0064801F0D8FB72
:10AD2000044801F0B9FB4FF0FF33236010BD00BFB2
:10AD3000E80F0020E43200207047000010B5084AF8
:10AD4000084C117824784B1C03F00F039C421DBF64
:10AD5000054C13706054002018BF012010BD00BFC7
:10AD6000123100201331002002310020F8B50B4CC5
:10AD700090F84B7090F84A601D460020234643F837
:10AD8000040F42EA012046EA0722294600F0FCFAB5
:10AD900020606068002818BF2046F8BD702300209E
:10ADA00090F84A10054B02291A7804D1012A01D0E3
:10ADB000062A02D15A78024B1A707047D02300201D
:10ADC000A823002008B5302383F31188034800F03E
:10ADD00017FC002383F3118808BD00BF9C100020DE
:10ADE00038B5044605293DD8DFE801F0303C033092
:10ADF000303D302383F31188204D214A012101F099
:10AE0000F2FB204A0321204601F0EDFB95F890105B
:10AE100005F14402204601F0E6FB95F8921021B1BD
:10AE200005F16802204601F0DEFB174800F0B1FB97
:10AE3000002383F31188154B1B7813B10520FFF70E
:10AE40007DFF0220BDE83840FFF778BF0846FFF7D6
:10AE500075FF302383F311880B4800F077FB002344
:10AE600083F3118838BD302383F31188064800F03E
:10AE700085FB002383F311880520E3E7EC0F002016
:10AE8000D4ED0008F8ED00089C100020C923002034
:10AE900070B5044606480D4603680BB100F0D8FCB7
:10AEA0002B462146BDE87040024A014800F0C8BC6C
:10AEB00090230020B9AE000870B530230E4683F30E
:10AEC00011880B78042B03D0002383F3118870BD05
:10AED000144B1B78DB09F7D1134C2278002AF3D0EE
:10AEE000124B1B78002BEFD00B899B0705D408234E
:10AEF0000F4A0121304601F0C8FB40F2E730002143
:10AF00000C4B24784FF47A72A4FB034520184FF0C1
:10AF1000000345EB0101F5F769F931468000FFF7C1
:10AF2000B7FFD1E7702F00208C2300201C110020D8
:10AF3000A9230020A0860100F8B590F8443004460B
:10AF400003F07F02212A40F0828013F0800334D086
:10AF5000002B7CD090F84500022829D003281ED071
:10AF6000012874D194F848305BB1022B94F8462044
:10AF70000DD0494B1A70A36394F84A30E363002361
:10AF80002DE0464AA2630822E2632364F8BD022A48
:10AF9000EFD1434BA3630623E3630023F5E7B4F843
:10AFA0004830002B53D101203E4AE063A263ECE716
:10AFB00001203D4BE063A363EFE790F845300A2B97
:10AFC0003CD00B2B0ED0092B41D190F848300BB15F
:10AFD000022B3CD1354BA3630223E363344B236440
:10AFE0000120D3E7B0F8483023BB90F846502D4BF2
:10AFF000002D14BF012200221A701BD12A4B1A788F
:10B00000C2B1302282F3118840F2E73000211E786D
:10B01000284B4FF47A72A6FB036730184FF00003F9
:10B0200047EB0101F5F7E2F821468000FFF730FF1A
:10B0300085F311880023A363E363D0E71E4990F8EA
:10B0400047200D78184BED091A70F3D1D8E740F27C
:10B050008163B4F844209A4214D194F8492061687D
:10B0600094F848304D6843EA022394F8471094F866
:10B0700046202046A84708B9002087E74368A36315
:10B0800003687BE70D4B93F89230002BF4D02046F9
:10B09000BDE8F84000F094BAE8230020A92300207E
:10B0A000CA2300201C1100208C230020D023002064
:10B0B000A1AD0008A0860100702F0020EC0F002039
:10B0C00008B5102200210448F5F7C0FA0023034A0E
:10B0D0001370034A137008BD0231002012310020A2
:10B0E00013310020F8B5294D294E2C460021307827
:10B0F0002B78284F984230D101B12070F8BD012241
:10B100002370254B1A70254B93F84F10081C18BF5D
:10B110000120FFF707FCE9E7002223701E4B1A709D
:10B12000FFF73EFC1D4B93F84F10081C18BF012081
:10B13000FFF702FCDAE72370184B93F84F10081C56
:10B1400018BF0120FFF7E2FBD0E70021237008467B
:10B15000F8E72370FFF7F2FBC8E71A46BA5C013341
:10B1600003F00F030121052AC4D80FF2080C5CF884
:10B1700022F000BF53B10008F5B0000837B1000855
:10B180004BB10008FFB0000819B1000813310020CE
:10B190001231002002310020C92300201833002082
:10B1A00070B50546144C04F10803A36504F11C03B3
:10B1B000E36504F13003E36704F18C06B0343146F3
:10B1C000204600F081F93146204600F0A7F92846D4
:10B1D00001F0FAFD284601F0DCF941F2883000F078
:10B1E000D4FC0649284601F0C1F9284601F0CAFD01
:10B1F0000022034B1A6070BDEC0F00201CEE00080B
:10B2000090230020014B1878704700BFA82300202E
:10B2100070B5302304460D46164683F311880F4956
:10B220000B78042B03D0002383F3118870BD012019
:10B230000B89A04018420AD001EB8401CB684FF47F
:10B240007A7158690C3000F0ADFC0130EBD0334618
:10B250002A462146014801F018FAE4E71833002095
:10B2600010B50D4B04461B7853B901460822012046
:10B27000FFF7CEFF202221460848F5F771F910BDEF
:10B28000074B014693F90030002BABBF0822202268
:10B2900001200320ECE700BF1C110020A92300209F
:10B2A000702F002010B50446014606220320FFF748
:10B2B000AFFF062221460248F5F752F910BD00BF44
:10B2C000CA230020032201461046FFF7A1BF000059
:10B2D000202910B40A46044606D10448214650F8F5
:10B2E000B03F10BC5B68184710BC7047EC0F0020E3
:10B2F00070B50A4C88B004F1B005D4F8B030202203
:10B300001E6A694600232846B04720B1C1B268468C
:10B31000FEF72DFAF1E708B070BD00BFEC0F00207A
:10B32000FFF7D4BB7047704708B5FFF7F9FF01F08E
:10B33000A7FBFFF7F7FF08BD08B501F0BDFBFFF75E
:10B34000F2FF08BDFFF704BB08B5FFF7B9FE0648DA
:10B35000FFF726FF054B064A41F288301A60BDE828
:10B36000084000F012BC00BF183300200824002061
:10B3700020110020014B1868FFF76CB90824002049
:10B38000FFF7B0BEFFF7B4BF020A032A12D006D8F7
:10B39000012A20D0022A21D00020024619E0212AC9
:10B3A00011D0222AF8D10229F6D80E4A0E4852F8B6
:10B3B000212006E0C0B20228EED80C4A0C4952F80F
:10B3C0002020405C05E00229E6D80920094A52F80D
:10B3D00021201A6070471220074AFAE75B20074ACB
:10B3E000F7E700BF48EE000854EE00082CEE000816
:10B3F00038EE00083CEE0008B2EE000857EE0008F8
:10B4000013B5446BE36F1A681178042915D1217ABA
:10B41000022912D11979012312898B4013420CD1D0
:10B4200001A904F1440000F078FD024628B1E46F60
:10B43000019B2179206801F028F902B010BD0C3081
:10B4400000F005BD4FF0FF330C3000F000BD44307C
:10B4500000F0CCBD4FF0FF33443000F0C7BD0C30DE
:10B4600000F0D8BC4FF0FF310C3000F0D3BC4430BA
:10B4700000F09CBD4FF0FF32443000F097BDC26F2A
:10B4800070B5136805461978042901D0012070BDF4
:10B49000017A0229FAD1012052795C899040044056
:10B4A000F4D105F10C0000F070FC02460028EDD04C
:10B4B000EE6FAB6A3068043B717901F0D4F8204636
:10B4C000E5E7406BFFF7DBBF7FB5034601260D467E
:10B4D00004460F4A43F8042B43600E4B0672029059
:10B4E0000193CB680C3000934B690A6A314600F037
:10B4F0002AFC094B02940193AB68EA690093314638
:10B500002B6904F1440000F0E5FC04B070BD00BFFD
:10B51000F8EF0008C3B4000801B400080B6830223B
:10B5200082F311880A7903EB820290614A79093229
:10B5300043F822008A7912B103EB82039861022357
:10B54000C1670372002383F31188704738B504463E
:10B5500001250221043000F07FFB04F10C00257569
:10B560006FF0010100F051FB84F84C5004F14400ED
:10B570006FF00101BDE8384000F047BB10B5012174
:10B580000446043000F068FB0023237584F84C3037
:10B5900010BD38B5044600250C3000F0EBFB04F17B
:10B5A0004400257500F0ADFC201D84F84C500121AD
:10B5B00000F052FB2046BDE83840FFF760BF0000B6
:10B5C00090F8443003F06003202B09D190F8453007
:10B5D000202B05D3212B05D9222B4FF0000309D0B6
:10B5E00000207047054B83630723C3630023036474
:10B5F000012070478363C363F9E700BF3011002067
:10B60000C36F73B51A6804461178042927D1017AEB
:10B61000022924D11979012315898B401D401ED19F
:10B6200000F14406304600F026FDC0B1304601A9C5
:10B6300000F073FCE36F06461A7E4AB101981A695E
:10B640002946121A3044F5F701F8E36F1B6901939C
:10B65000E06F019B01793246006801F016F802B0F4
:10B6600070BD00EB81032DE9F3419E6904460D4650
:10B67000FEB1302383F311880821301D04EB8507C8
:10B6800000F0EAFAFB6806F144085B691B6813B135
:10B69000404600F050FC01A9404600F03EFC024646
:10B6A00050B1019B2946204600F0EFFF002383F3B1
:10B6B000118802B0BDE8F081FB685A691268002A5F
:10B6C000F4D01B8A013B1342F0D1F36F1B7E002B99
:10B6D000ECD104F14402E5E7093110B550F82140FE
:10B6E000C4B1302383F311880421601800F0B4FA48
:10B6F000E26F04F10C001368527903EB8203DB68FC
:10B700009B69596800F04BFB2046FFF7B8FE002309
:10B7100083F3118810BD7047024B034A1A60034A35
:10B720005A607047143100209833002000700020C8
:10B73000094B30B51C684D1E224449422A440A4038
:10B7400059681044884204D8A04202D318601046B9
:10B7500030BD0022FBE700BF1431002008B53023C4
:10B7600083F31188FFF7E4FF002383F3118808BDFA
:10B7700070477047FEE7000070B5082000240B4BAF
:10B7800093E826000439954207D8D968914209D830
:10B79000013803F11003F3D170BD51F8046F42F882
:10B7A000046BF0E742F8044BF0E700BF20F000081C
:10B7B00038B501230025074C23706560FFF7ACFF07
:10B7C0000549064800F034F90223237085F31188F7
:10B7D00038BD00BF20310020A0F000082831002033
:10B7E00072B60322024BD865024B1A70FEE700BF07
:10B7F000283100202031002000F03CB8034B59686C
:10B800005A68521A9042FBD8704700BF001000E0FF
:10B8100010B50A4A13699C68A1420CD85C68816023
:10B8200003604460206058609868411A99604FF046
:10B83000FF33936110BD091B1B68ECE72831002022
:10B840000361002310B4C260436110BCFFF7E0BF86
:10B85000036881689A680A449A60426813605A6073
:10B8600000234FF0FF320360014B9A61704700BF25
:10B870002831002070B5124D2946EA690132EA618B
:10B8800051F8102F8A4206D030269368013B93600E
:10B890002C69A36803B170BD226861680A605160B9
:10B8A000236083F31188E36821692046984786F373
:10B8B000118861690029EBD02046FFF7A9FFE7E76F
:10B8C0002831002000238268037503691B6899688A
:10B8D0009142FBD25A680360426010605860704722
:10B8E00000238268037503691B6899689142FBD83D
:10B8F0005A680360426010605860704708B5302392
:10B9000083F311880A7D0023052A06D8DFE802F0B8
:10B910000C050503130F8A6913604FF0FF330846C7
:10B920008B61FFF7CFFF002383F3118808BD8A697D
:10B930009368013393604A680B6813605A60ECE7C0
:10B94000FFF7C0BF054BD9680875186802685360D7
:10B950001A6001220275D860F4F732BC2831002049
:10B9600030B50C4B87B0DC684B1C05460FD0234626
:10B97000094A6846FFF764FF2846FFF7E3FF009B8C
:10B9800013B16846FFF764FFA06907B030BDFFF749
:10B99000D9FFF9E728310020FDB8000838B50C4D73
:10B9A0008161EB6881689A680446914203D8BDE8DA
:10B9B0003840FFF787BF1846FFF792FF0123EC607E
:10B9C000237501462046BDE83840F4F7F9BB00BFB7
:10B9D00028310020044B1A68DB6890689B68984205
:10B9E00094BF00200120704728310020084B10B57B
:10B9F0001C68D868226853601A6001222275DC60D6
:10BA0000FFF76EFF01462046BDE81040F4F7D8BBB3
:10BA100028310020044B1A68DB6892689B689A42C0
:10BA200001D9FFF7E3BF70472831002030BFFDE7A1
:10BA300070B504460025194B86B0856221630E4619
:10BA4000586000F027F904F11003236163614FF09F
:10BA5000FF33A361124BE561DA69002304F134017D
:10BA6000C4E9082324606460A560E562E56580237D
:10BA70000C4A204600F01CF801230B4AE0600375D5
:10BA80000092726868460192B268CDE90223074BC2
:10BA9000CDE9043500F03EF806B070BD203100203D
:10BAA00028310020AFF00008B4F000082DBA0008DB
:10BAB0008B6002224B62002308618A820B62CB6199
:10BAC000084670478368C168A3F14C0243F81C2CF8
:10BAD000026943F84C2C42690C4843F8482C0C4A44
:10BAE00043F8180C43F82C2C022203F8142C0022E3
:10BAF00043F8201C03F8132C43F8041C43F8082CCB
:10BB000043F80C2CA3F12800704700BF2831002017
:10BB1000D101000808B5FFF7D5FFBDE80840FFF7E1
:10BB20000FBF000038B5302484F311882839441839
:10BB300044F8243C049B002544F8203C0A4BA4F123
:10BB4000240144F8043C0223A382084BE160A26074
:10BB5000236162622562E56129462046FFF71EFFE8
:10BB600085F31188204638BDD10100082831002016
:10BB7000024BDB6898610F20FFF7E4BE28310020FC
:10BB8000302383F31188FFF7F3BF08B50146302354
:10BB900083F311880820FFF7E3FE002383F3118865
:10BBA00008BD0000054BDB6821B1036098610320EC
:10BBB000FFF7D6BE4FF0FF30704700BF283100209E
:10BBC00003682BB10022026099611846FFF7B8BEE6
:10BBD00070470000064BDB6839B1426818605A6054
:10BBE000136043600420FFF7BBBE4FF0FF30704787
:10BBF000283100200368984206D01A68026050601D
:10BC000099611846FFF79CBE704738B504460D464B
:10BC10002068844200D138BD036823605C60856180
:10BC2000FFF78EFEF4E700230060406083607047FA
:10BC3000C3691943037DC1610A2B03D1836919428A
:10BC400005D170470B2B06D183698B4303D10023A9
:10BC50008361FFF775BE704770B506460D460468F0
:10BC6000B44200D170BDE3682B43E36015B1236992
:10BC70001D4203D0A1686068FFF7DAFF2468EFE790
:10BC8000EFF30983203383F30988002383F31188BA
:10BC900070470000302080F3118862B60B4B0C4ACD
:10BCA000D96821F4E0610904090C0A430949DA6002
:10BCB000CA6842F08072CA6007490A6842F001020D
:10BCC0000A602022DA7783F82200704700ED00E056
:10BCD0000003FA05F0ED00E0001000E010B530239D
:10BCE00083F311880B4B5B6813F400630FD0EFF301
:10BCF00009844FF08073203CE36184F30988FFF7E7
:10BD000069FE10B1044BA36110BD044BFBE783F344
:10BD10001188F9E700ED00E0E3010008E601000802
:10BD200008B500F077FF01F08EF800F044FB00F05A
:10BD300099FB00F00DFCFFF7FFFABDE8084000F0AA
:10BD400000B801F0A1B80172002130B5039C0433A2
:10BD500004FB0325C361049B00600363059B4060F3
:10BD6000C160426102618561046242628162C162B6
:10BD7000436330BD0022416AC26041610161826259
:10BD8000C2626FF00101FFF740BF0369426993424D
:10BD900001D1C2680AB9181D7047002070470369B5
:10BDA0001960C26800210132C260C269134482690D
:10BDB0000361934224BF436A0361FFF71BBF38B599
:10BDC00004460D46E3683BB162690020131D12680A
:10BDD000A3621344E36207E0237A33B9294620467D
:10BDE000FFF7F8FE0028EDDA38BD6FF00100FBE741
:10BDF000C368C269013BC3604369134482694361FC
:10BE0000934224BF436A436100238362036B03B1FF
:10BE10001847704770B53023044683F31188866A4B
:10BE20003EB9FFF7CCFF054618B186F311882846C6
:10BE300070BDA36AE26A13F8015B9342A36202D366
:10BE40002046FFF7D5FF002383F31188EFE72DE9A4
:10BE5000F84F04460F4691469A464FF0300888F353
:10BE600011880025AB46A66A4EB951462046FFF719
:10BE7000A6FF20B186F311882846BDE8F88FA16A95
:10BE8000E66AA9EB0503761A9E4228BF1E46402E9D
:10BE900016D938464022F4F763FBA36A4037403393
:10BEA000A3624035A26AE36A9A4202D32046FFF7B2
:10BEB0009FFF8BF311884D45DED288F31188D2E7BE
:10BEC00038463246F4F74CFBA36A37443344A36246
:10BED0003544E7E710B5029C04330172C36103FBEC
:10BEE000042100238362C362039B00600363049BFD
:10BEF0004060C460426102618161046242624363E6
:10BF000010BD026A6FF00101C260426A42610261C3
:10BF100000228262C262FFF778BE436902699A42D8
:10BF200001D1C26822B9184650F8043B0B60704733
:10BF300000231846FAE7C368C2690133C360436946
:10BF40000021134482694361934224BF436A4361E1
:10BF5000FFF750BE38B504460D46E3683BB1236990
:10BF600000201A1DA262E2691344E36207E0237A0B
:10BF700033B929462046FFF72DFE0028EDDA38BDFB
:10BF80006FF00100FBE703691960C268013AC26003
:10BF9000C269134482690361934224BF436A036107
:10BFA00000238362036B03B11847704770B53023D9
:10BFB00004460E4683F31188856A35B91146FFF7AA
:10BFC000C9FF10B185F3118870BDA36A1E70A36A02
:10BFD000E26A01339342A36204D3E1692046043943
:10BFE000FFF7D1FF002080F31188EDE72DE9F84F2E
:10BFF00004460F4691469A464FF0300888F3118860
:10C000000025AB46A66A4EB951462046FFF7A2FF6F
:10C0100020B186F311882846BDE8F88FA06AE66A49
:10C02000A9EB0503361A9E4228BF1E46402E18D99A
:10C0300039464022F4F794FAA36A40374033A362AA
:10C040004035A26AE36A9A4204D3E1692046043982
:10C05000FFF799FF8BF311884D45DCD288F31188E7
:10C06000D0E739463246F4F77BFAA36A37443344C3
:10C07000A3623544E5E7026943699A4217D1C36870
:10C080009BB1836A8BB1043B9B1A0ED01360C368CB
:10C09000013BC360C3691A44836902619A4224BFA9
:10C0A000436A03610023836201231846704700231B
:10C0B000FBE7F8B5154682680B46AA428169066916
:10C0C00038BF8568761AB542044607D218462A4614
:10C0D000F4F746FAA3692B44A3610DE011D9324667
:10C0E0001846F4F73DFAAF1B3A46E1683044F4F7DE
:10C0F00037FAE2683A44A261A36828465B1BA36052
:10C10000F8BD18462A46F4F72BFAE368E4E72DE970
:10C11000F0410446154683682669934238BF856816
:10C1200040690F46361AB54206D22A46F4F718FA85
:10C1300063692B4463610DE012D93246A5EB060812
:10C14000F4F70EFA4246B919E068F4F709FAE26822
:10C1500042446261A36828465B1BA360BDE8F0818E
:10C160002A46F4F7FDF9E368E4E710B50024C3615B
:10C17000029B0A44006040608460C160816141614B
:10C180000261036210BD08B582694369934201D11F
:10C19000826882B98268013282605A1C42611970D9
:10C1A0000369426900219A4224BFC3684361FFF7D3
:10C1B00021FD002008BD4FF0FF30FBE770B53023B4
:10C1C00004460E4683F31188A568A5B1A368A26949
:10C1D000013BA360531CA36115782269934224BFDD
:10C1E000E368A361E3690BB120469847002383F31A
:10C1F0001188284607E031462046FFF7EBFC00286F
:10C20000E2DA85F3118870BD2DE9F74F05460F4638
:10C2100090469A46D0F81C90302686F311884FF04D
:10C22000000B144664B1224639462846FFF741FF09
:10C23000034668B951462846FFF7CCFC0028F1D0E8
:10C24000002383F31188A8EB040003B0BDE8F08F4E
:10C25000B9F1000F03D001902846C847019B8BF32A
:10C260001188E41A1F4486F31188DBE7C361009B41
:10C27000C160816141611144006040608260016180
:10C2800003627047F8B504460E461746302383F321
:10C290001188A568A5B1A368013BA36063695A1C16
:10C2A00062611E70236962699A4224BFE368636118
:10C2B000E3690BB120469847002080F3118807E01E
:10C2C00039462046FFF786FC0028E2DA85F311881C
:10C2D000F8BD8369426910B59A4201D182687AB982
:10C2E00082680021013282605A1C82611C780369D5
:10C2F0009A4224BFC3688361FFF77CFC204610BDCF
:10C300004FF0FF30FBE72DE9F74F05460F4690460B
:10C310009A46D0F81C90302686F311884FF0000B17
:10C32000144664B1224639462846FFF7F0FE03461C
:10C3300068B951462846FFF74DFC0028F1D000238C
:10C3400083F31188A8EB040003B0BDE8F08FB9F1C6
:10C35000000F03D001902846C847019B8BF311883A
:10C36000E41A1F4486F31188DBE70C30FFF74CBF5B
:10C370004FF0FF330C30FFF747BF3030FFF7C3BF3C
:10C380004FF0FF333030FFF7BEBF0C30FFF716BF62
:10C390004FF0FF310C30FFF711BF3030FFF772BFA5
:10C3A0004FF0FF323030FFF76DBF012914BF6FF03F
:10C3B00013000020704700F009BE0000034637B5A7
:10C3C00015460D4A044643F8042B4360012380229E
:10C3D000037200900B4600F154010C30FFF7C5FECC
:10C3E00000942B46802204F1D40104F13000FFF7C1
:10C3F0003DFF03B030BD00BFBCF0000810B53023D6
:10C40000044683F3118800F0F3FD02230020237219
:10C4100080F3118810BD38B5436904460D461BB939
:10C4200004210844FFF718FC294604F10C00FFF72B
:10C43000AAFE002806DA201D4FF40061BDE838404E
:10C44000FFF70ABC38BD302383F31188002340690D
:10C4500083F31188B0FA80F0400970474FF0FF3144
:10C46000FFF7A0BB00F08CBE0123037000230C304B
:10C4700040F8083C40F8043CFFF7D5BB10B530232A
:10C48000044683F31188416000F086FE02230020F9
:10C49000237080F3118810BD10B53023044683F358
:10C4A000118800F0C7FE002301226360227083F32D
:10C4B000118810BD302383F31188436899685A6846
:10C4C0004FF480338B409361002383F311887047CE
:10C4D000302383F31188436899685A6801238B409D
:10C4E0009361002383F31188704738B504463025E3
:10C4F00085F31188032504F8085B00F0B9FE204697
:10C50000FFF7ACFF002383F3118838BD10B530234B
:10C51000044683F31188032304F8083B00F0BDFEB2
:10C520002046FFF79BFF002383F3118810BD10B551
:10C530003023044683F31188032304F8083B00F0FA
:10C54000C2FE2046FFF78AFF002383F3118810BD47
:10C5500001F0DEB8012303700023C361836203622C
:10C56000C3624362036343608360704738B5054626
:10C57000302383F3118800244160C4600461446166
:10C58000846101F0CBF802232B7084F311882046DC
:10C5900038BD70B53023064683F3118801F0D6F814
:10C5A000344600250123756004F80C3B1C3654F812
:10C5B000043B7BB1586920B16FF001010C30FFF7EB
:10C5C000FFFA54F8043C986920B16FF001010C3077
:10C5D000FFF7F6FAB44244F8045CE8D1FFF71AFA20
:10C5E00085F3118870BD70B500EB81030546506975
:10C5F0000E461446DA6018B114220021F4F726F82A
:10C60000A06918B114220021F4F720F83146284619
:10C61000BDE8704001F0B8B8F8B50446002783685B
:10C6200000F1100503F00113836000F11C0655F8BA
:10C63000043B7BB1586920B16FF001010C30FFF76A
:10C64000BFFA55F8043C986920B16FF001010C3035
:10C65000FFF7B6FAB54245F8047CE8D12046BDE8BC
:10C66000F84001F01DB9F0B4012500EB8104E46845
:10C670004789A4698D403D43458123600023A26022
:10C680006360E360F0BC01F07DB9F0B4012500EB1C
:10C690008104E468078964698D403D430581236016
:10C6A0000023A2606360E360F0BC01F08BB900007E
:10C6B000037810B5052B10D1084C4FF47A70E37A4B
:10C6C00043F00803E372637843F004036370FFF7F9
:10C6D0005CFA637803F0FB03637010BD0040014017
:10C6E0002DE9F0410223002504464FF03008037085
:10C6F000C564856000F10C0600F11C0756F8043B88
:10C70000ABB188F3118856F8043C586920B16FF03A
:10C7100001010C30FFF754FA56F8043C986920B137
:10C720006FF001010C30FFF74BFA85F31188BE4220
:10C7300046F8045CE2D184F83450204601F092F8C7
:10C7400063681B6823B12046BDE8F041002118470B
:10C75000BDE8F081F8B503780446052B29D080F8B0
:10C7600050300523037043681B680BB104219847C0
:10C7700000263027A66004F10C051C3455F8043B54
:10C78000ABB187F3118855F8043C586920B16FF0BC
:10C7900001010C30FFF714FA55F8043C986920B1F8
:10C7A0006FF001010C30FFF70BFA86F31188A542F8
:10C7B000E4D1F8BD0178052906D1436890F85020EE
:10C7C0001B68027003B1184770470000F8B590F875
:10C7D000343004460E4613B1002380F8343004F19F
:10C7E00044023146204601F0B1F863689B68B3B952
:10C7F00094F8443013F0600538D00021204601F051
:10C8000021F90021204601F00FF963681B6813B17C
:10C81000062120469847062384F83430F8BD204688
:10C8200098470028E4D094F84B2094F84A3043EA23
:10C830000223E26B9A4294F9442088BFE363002A02
:10C84000E36B80F20781002B00F0FB80092384F862
:10C850003430302383F311880021E36BA26B204630
:10C86000FFF713FF002383F31188D7E794F84520DF
:10C8700003F07F0343EA022340F20232934200F0C6
:10C88000CC8025D8022B00F0A08009D8002B51D0F5
:10C89000012BB2D1774BA3630223E36300234EE065
:10C8A000B3F5817F00F0A680B3F5407F49D0B3F5A2
:10C8B000807FA2D194F84630012B9ED1B4F84C3041
:10C8C00023F00203A4F84C30A563E5632564AAE7CE
:10C8D00040F2016293421DD8B3F5C06F3BD2B3F56D
:10C8E000A06F8AD1B4F84430B3F5A06F0ED194F89C
:10C8F0004630204684F84E3000F03EFF63681B68E7
:10C9000013B1012120469847032323700023A3631A
:10C91000E36314E0B3F5106F33D040F60242934264
:10C92000B8D0B3F5006F7FF468AF04F14F03A36391
:10C93000012324E004F14C02A2630222E263236497
:10C9400071E794F84630012B7FF457AFB4F84C30C0
:10C9500043F00203B6E794F84920616894F8483040
:10C960004F6843EA022394F8471094F84620204683
:10C97000B84700283FF441AF4368A3630368E3630B
:10C98000A4E72378042B10D1302383F311882046A9
:10C99000FFF742FE85F311880321636884F84F5046
:10C9A0001B6821700BB12046984794F84630002B45
:10C9B000ACD084F84F300423237063681B68002BCD
:10C9C000A4D0022120469847A0E794F8483020469A
:10C9D0001D0603F00F010AD500F09CFF012804D0CA
:10C9E00002287FF40AAF244B55E7244B53E700F0AD
:10C9F00075FFF3E794F84630002B7FF4FEAE94F811
:10CA0000483013F00F0181D01A06204602D501F0FC
:10CA100031F87BE701F022F878E794F84630002BF4
:10CA20007FF4EBAE94F8483013F00F013FF46EAF93
:10CA30001B06204602D501F005F867E700F0F4FF79
:10CA400064E7142384F8343031462046BDE8F840CA
:10CA500000F08CBF63B1152384F83430302383F3A6
:10CA600011880021E36BA26B2046FFF7FCFDF9E67D
:10CA70000B23E7E7E8F00008E4F00008E6F0000820
:10CA800008B500F0C9F80B4B9A6C42F020029A648A
:10CA90009A6C9A6C42F040029A649A6C9A6C42F0DA
:10CAA00080029A649A6C9A6C42F480729A649B6CCD
:10CAB00008BD00BF000C01407047162303604FF013
:10CAC000FF307047002070471846704700207047BD
:10CAD00010B50022044608460121FEF73FFE18B9B2
:10CAE0000C234FF0FF30236010BD08B51346002122
:10CAF00058221846F3F7AAFD4FF400524260002076
:10CB000008BD01207047000008B50248FEF768FE26
:10CB1000F3F7EEFCEAF0000808B50248FEF760FE05
:10CB2000F3F7E6FCEFF0000801207047704700F1D2
:10CB30006043090103F56143C9B283F8001301237F
:10CB400000F01F024009800000F16040934000F5B2
:10CB50006140C0F8803103607047012200F01F037C
:10CB60009A4043099B0003F1604303F56143C3F816
:10CB70008020C3F88021002300F1604000F561406F
:10CB800080F800337047090100F16040C9B200F538
:10CB90006D4001767047000017498A68022A12D05A
:10CBA000032A26D0154B1649012A18BF0B46124AF4
:10CBB000926902F07F02013252080132B3FBF2F3B4
:10CBC000104A13607047104A0B68526F49686FEA49
:10CBD0009212012902F003020CBF08490B490332EB
:10CBE00003F01F034A4301335B080133B2FBF3F345
:10CBF000DDE7074BDBE700BF000C0140006CDC0207
:10CC000000127A0038110020000401400048E801B9
:10CC1000001BB700FFF7C0BF13B50C20032440F280
:10CC2000BE71314B314A9C62D862C2F89410002127
:10CC30009962D9629C62D8628020C3F81C0CD3F838
:10CC40001C0CC3F81C0C009101914FF40141C3F876
:10CC5000481C4FF6FC71A3F5744319630F2119604A
:10CC60000223136501234BF68031D364936D03F0E7
:10CC700001030193009B01330093019B13B9009BB7
:10CC80008B42F3D1019B03B9FEE7194B19490120EF
:10CC900019600021A3F59043996180211962196AF6
:10CCA00019622021586019601968196019680143D8
:10CCB0001960C02151679067D16F0329FCD102220E
:10CCC0009A6001220021DA60074A9162D1629A6C6F
:10CCD00042F400429A649A6CDA6C42F40062DA64BC
:10CCE000DB6C02B010BD00BF000001400004014039
:10CCF0000054014012000003144B834225D1144B11
:10CD000002201A6C134942F480721A641A6C42F0C1
:10CD100002021A64D3F8882042F00202C3F8882085
:10CD2000D3F8882022F00202C3F8882001225A6337
:10CD3000DA670864DA6608225A615A6942F0040226
:10CD40005A615A6942F001025A6170471833002053
:10CD5000000C0140004C0140084B83420CD1084BB1
:10CD60005A6902F008025A6100225A61DA66DA67EB
:10CD70001A6C22F002021A64704700BF18330020B8
:10CD8000000C01400F4A936C43F4004343F020032E
:10CD900093644FF080436FF4C0521A634FF0707287
:10CDA000DA624FF020721A6000225A609A60DA60EC
:10CDB0004FF44C325A62012203F5A0335A70072215
:10CDC000DA727047000C01400E4A6FF48051936C88
:10CDD00043F4004343F0200393644FF080436FF427
:10CDE000C0521A6300221A609A60DA6019634FF029
:10CDF000807119604FF4805159605A624FF080522F
:10CE00009A617047000C0140062108B50846FFF7FB
:10CE10008EFE06210720FFF78AFE06210820FFF775
:10CE200086FE06210920FFF782FE06210A20FFF771
:10CE30007EFE06211020FFF77AFEBDE8084006219D
:10CE40002120FFF774BE7047C9434FF0553301638B
:10CE500002F003015943016042F380014160C2F3D3
:10CE6000C10159438160C2F341115943C160C2F30A
:10CE7000C1214B43C3624FF01133C2F3C3125A4373
:10CE8000026242627047000040F2CF22044B082148
:10CE90005A6000229A6007220B201A60FFF773BEC7
:10CEA00010E000E008B5302383F31188FEF7A4FCFE
:10CEB000002383F3118808BD08B5FFF7F3FFBDE831
:10CEC0000840FEF70BBF0000024A536843F002031C
:10CED00053607047003800402DE9F041384DD5F8D7
:10CEE00054717B69D806DCB20AD5302383F31188EC
:10CEF0004FF48061281DFEF7AFFE002383F31188F5
:10CF0000302383F311882F4EA6F1040814F00F0389
:10CF100032D183F311887B68980714D5A10612D506
:10CF2000302383F311882848FFF7D3F9002844DA27
:10CF300008212448FEF790FE7B6823F002037B6003
:10CF4000002383F311887B689A0711D563060FD5F8
:10CF5000302383F311886A6CAB6C9A4205D1AB6BBA
:10CF60001BB110211748FEF777FE002383F31188C9
:10CF7000BDE8F041FEF7B2BE14F0020F14BF4FF44B
:10CF800080710021620748BF41F02001230748BF9C
:10CF900041F0400114F0010418BF41F08001304617
:10CFA000FEF75AFE3B682CB195F8581140461940DF
:10CFB000FFF731FA7C69E4B2A8E73860C0E700BF48
:10CFC000883100208C310020B831002010B5054C8C
:10CFD000054A00212046FFF7F1F9044BC4F854310B
:10CFE00010BD00BF88310020C9CE000800380040C5
:10CFF00038B5294C037A002918BF0C46012B054689
:10D000001AD1264B984217D1254B0C219A6C1E2021
:10D0100042F480429A649A6CD3F8902042F48042A1
:10D02000C3F89020D3F8902022F48042C3F89020D7
:10D03000D3F89030FFF77BFDD5F85431E1791A69C8
:10D0400002F050020A431A612168164A02EB5102AB
:10D05000B2FBF1F202F00F01C3F8C0108021D960D9
:10D06000C2F3071119600021C2F307325A60D96078
:10D07000607922790243A0790243DA600122C3F881
:10D080009C10C3F898205A6842F005025A60FF23AA
:10D0900085F8583138BD00BFF4F000088831002011
:10D0A000000C014000A24A0470B5334CE5692E6BB8
:10D0B000E26A6B6A9A4234BFE36A6B6A13F1FF3328
:10D0C00038D2E36A002B41D1EB6263681B6833B14D
:10D0D00004222948227098472378042B01D1022387
:10D0E0002370302383F3118800212448FEF768FD64
:10D0F000002383F31188F30718D5286A228E666A05
:10D10000E36A616AD31A3344121A934228BF134662
:10D1100099424FF6FF7138BF636A13F1FF331ED295
:10D12000636A1BB9EB6A23F00103EB62BDE8704050
:10D13000FEF7D4BD296EE26A013AE262A26A002AD1
:10D14000BCD01170A26A0132A262B7E7E26AEB6951
:10D150009A429EBFE36A03F1FF33EB61CBE7626A59
:10D16000013A6262226A0AB92966D6E712F8010B0F
:10D1700028662262D1E700BFE4320020EC320020B2
:10D1800010B5034C2046FFF76FF9024BE36110BD69
:10D19000E432002000300040037810B5012B044633
:10D1A00022D1224B98421FD1214B0A219A6C1A207E
:10D1B00042F480529A649A6CD3F8902042F48052E0
:10D1C000C3F89020D3F8902022F48052C3F8902026
:10D1D000D3F89030FFF7ABFC6268E369128A5A61BA
:10D1E0001A6942F001021A616168E369CA89898992
:10D1F0000A4342F00702218E92B21A6069B90122F5
:10D200009A619869904205D10132B2F5807FF7D1D9
:10D2100091B201E0012AFBD1218600229A61DA61F4
:10D22000DA6A22F0FF02DA629B6C10BDE432002061
:10D23000000C014008B50378022B13D10022C3690A
:10D240009A60DA6A22F0FF02DA629B6C064B98421F
:10D2500008D11A20FFF781FC044B9A6C22F480520B
:10D260009A649B6C08BD00BFE4320020000C0140B2
:10D2700091B18362038E41625B089942C16228BF0B
:10D280001946C369026299610139D961DA6A42F0CB
:10D290001102DA6201229A60704799B10023836219
:10D2A000038E41625B089942C16228BF1946C36977
:10D2B000026299610139D961DA6A42F01102DA62D7
:10D2C00001229A60704799B100230362038E416284
:10D2D0005B089942C16228BF1946C369826299619D
:10D2E0000139D961DA6A42F01102DA6201229A60E8
:10D2F000704700000A4A0B4B10B502EB800298738E
:10D3000038B1DC7D987D40EA04200B18994203D1A6
:10D3100010BD987DC0B2F8E7147801F8014BF5E72D
:10D32000204001400040014090F8342010B5152AFB
:10D3300004460CD8012393400C4A134208D19B02A7
:10D3400005D5036C03B19847002384F8343010BD31
:10D3500000216022064B99735A7499735A7443687A
:10D360001B680BB1062198470623EEE7410E10001B
:10D37000004001402DE9F843244C00F1020804EB81
:10D380008803D3F80490224ED9F81850B073337D37
:10D390000746DB0733D5A968FFF7ACFFAB68B9F8E0
:10D3A00012200344AB606B68904203446B602B68AF
:10D3B000A3EB00032B602B8A03F1FF339BB22B827C
:10D3C00000D3F3B9012303FA07F2638923EA0203C6
:10D3D000638104EB88035B68DB6813B139460B4853
:10D3E0009847302383F3118804EB880463689869B5
:10D3F00041680C30FEF7E4FB002383F31188BDE89D
:10D40000F883337D03F0FE033375F8E7183300200B
:10D4100000400140F8B5214C871C04EB87035E688F
:10D420000146726950681568A84219D3012303FAAE
:10D4300001F2238923EA02032381B3680BB120465A
:10D440009847302383F3118804EB87046368002135
:10D4500058690C30FEF7B4FB002383F3118817E002
:10D460000F4B9973136918445060281ADED0348A20
:10D47000844228BF044690681461034409489360BD
:10D4800000EB81011C449C4203D10122044B5A74DD
:10D49000F8BD13F8012B0A70F5E700BF1833002020
:10D4A000004001402040014090F8342010B5152A7A
:10D4B00004460CD8012393400C4A134208D19B0523
:10D4C00005D5036C03B19847002384F8343010BDB0
:10D4D00000216022064B99735A7499735A744368F9
:10D4E0001B680BB1062198470623EEE7410C30007C
:10D4F000004001402DE9F047824B9E79F6B2B70714
:10D5000002D58148FFF756F9750702D57E48FFF727
:10D51000E7F8340713D57C4C6368DB6823B9794A94
:10D52000D37A03F0F703D3722378052B02D1764820
:10D53000FFF740F96368DB680BB173489847714A9D
:10D540009378177903F0FF08FFB253B9002F3DD14C
:10D55000F30702D56C48FFF7FDF8BDE8F047FEF78A
:10D56000BDBB18F0010F1FD00021674CD4F80C9000
:10D570009173537CDBB2580744BF517484F8341064
:10D58000DA0605D580215F4A5174002284F83420E0
:10D5900094F834200AB1062A28D1DB0704D5D9F83B
:10D5A000043000215848984718F0020F02D001209B
:10D5B000FFF730FF18F0040F02D00220FFF72AFF18
:10D5C00018F0080F02D00320FFF724FFB80702D598
:10D5D0000120FFF7CFFE790702D50220FFF7CAFE30
:10D5E0003A07B5D50320FFF7C5FEB1E7092A49D1AF
:10D5F000444D6B7CDBB213F00201D5D103F0110373
:10D60000112BD1D0D9F81420A9735168136910686F
:10D6100019445160411AB9F810E017D0714528BF7C
:10D620007146906811610344384893605A189342D8
:10D6300008D1B9F810308B4294BF02210A21314B36
:10D640005974B1E713F8014B0470F0E7734503D147
:10D650000A236B741161A7E7238923F00103238157
:10D66000D9F808300BB128489847302383F3118844
:10D670000021E36858690C30FEF7A2FA002383F317
:10D68000118891E7152A8FD1DFF878A09AF8113028
:10D69000DD0789D5D9F818500020A968FFF72AFEC0
:10D6A000AB68B9F812200344AB606B689042034446
:10D6B0006B602B684FF00002A3EB00032B602B8AFA
:10D6C00003F1FF339BB22B8200D3A3B90D4B9A73A6
:10D6D00048225A74638923F001036381E368DB689D
:10D6E00013B1002108489847302383F31188E36879
:10D6F00098694168BFE740238AF80E208AF8113004
:10D7000052E700BF00400140183300202040014094
:10D710000148FEF71FBF00BF1833002010B5047882
:10D72000012C0ED1074AC260FFF7E6FA0022064B31
:10D730000D21DA72DC715A720E20BDE81040FFF73D
:10D74000F6B910BDFCF0000800400140037810B5A8
:10D75000012B04460CD00E20FFF7FFF90022054BE9
:10D760002046DA72DA715A72BDE81040FFF7F4BA57
:10D7700010BD00BF0040014090F84E20014B1A70D0
:10D78000704700BF0040014000EB8100344BC2688D
:10D7900001F00F0110B59973106800F00300002923
:10D7A00056D002282CD003282AD0012827D153692B
:10D7B0000BB993691BB3E020294B9874108AC0F30E
:10D7C000C7001874402058740820587458740120F9
:10D7D000DC7900FA01F149B241EA0400C0B2D87123
:10D7E000C0205875528AC2F3C702DA7480221A75B3
:10D7F00010221A751A755A7A1143C9B2597210BD9E
:10D80000506980B100209874108AC0F3C700187462
:10D81000402058740820587458740120DC798840DE
:10D820002043C0B2D8719369002BE8D000200C4B84
:10D830005875528AC2F3C702DA7480221A75102210
:10D840001A751A750122587A02FA01F10143D4E7D8
:10D850000028D4D1DA7942F00102DA71CFE700BFB3
:10D8600000400140002208B50B4BDA715A72426841
:10D87000D2681AB1DA7A42F00802DA72074B002154
:10D88000C360FFF781FF0122034B5A70DA7A42F03E
:10D890000102DA7208BD00BF00400140FCF0000840
:10D8A00070B50D4B0021DA79402602F00102DA71E1
:10D8B000082401228025102059729A730132D2B2B5
:10D8C000042A99745E745C745C7459751D751875BE
:10D8D0001875F2D170BD00BF004001400C4B01F043
:10D8E0000F029A7341B95A7C52070ED4D87910F0BE
:10D8F000010018BF02207047187D10F0200004D1ED
:10D900005B7A134113F0010FF3E70120704700BF6A
:10D91000004001400C4B01F00F029A7341B95A7C50
:10D9200052070ED4D87910F0010018BF02207047BA
:10D93000587C10F0100004D1DB79134113F0010F73
:10D94000F3E70120704700BF00400140064B01F0A3
:10D950000F0103EB810302F10801187802F8010BB3
:10D960009142FAD1704700BF204001404822044B49
:10D9700001F00F0199735A74002380F83430704716
:10D980000040014010B501F00F0400EB8101CB68AD
:10D9900099690A6872B1588A1318013BB3FBF0F316
:10D9A0009BB20B82064B9C7334B11A7D02F0FE02CF
:10D9B0001A7510BD0123F4E740225A74F9E700BF3D
:10D9C0000040014000EB810311F00F0170B508BF6A
:10D9D0004025DC6808BF124A636904BF917355741F
:10D9E000228A1D680F4CAA4228BF2A461A619B68EA
:10D9F00004EB81049D189D4205D1094B997331B107
:10DA000001225A7470BD13F8016B2670F3E7597C3C
:10DA1000C168098A914294BF02220A22F1E700BF3D
:10DA20000040014020400140054B01F00F01997377
:10DA300011B120221A75704760225A74704700BFD6
:10DA400000400140044B01F00F01997311B1102205
:10DA50005A7470476022FBE700400140044B01F01C
:10DA60000F01997311B180221A757047597470476C
:10DA700000400140044B01F00F01997311B14022A5
:10DA80005A7470475974704700400140074BD3E9FE
:10DA900002128A4208D0596801F59C70824201D175
:10DAA000D96070470832DA60704700BFA42D0020AB
:10DAB0000023074930B51A460C46834201D1E2548F
:10DAC00030BD11F8015B01332A44D2B2F5E700BF43
:10DAD000702500202DE9F843034616461A481B4CD2
:10DAE00000F8013BF2F73CFDD4E9018708F59C7989
:10DAF0004F4506F10106E36804D1984506D10020A0
:10DB0000BDE8F88307F108029342F7E7104A21695C
:10DB100002F2CF735B1A312B98BF2261322EEED8FE
:10DB20002569324628460849F2F71AFD4F453D60FF
:10DB300035447D6018BF083725610CBFC4F80880E4
:10DB4000A7600120DCE700BF2C2F0020A42D0020BF
:10DB5000D42500200368044905220B6003790720BF
:10DB60000B71FFF7B7BF00BFB825002070B50546A1
:10DB70001F4C003044F0010418BF0120A047286A60
:10DB80001C4E003018BF0120A0470120A047686B41
:10DB9000003018BF0120A0470024174B174A18492E
:10DBA0005A601961C2E90011C3E902221C704FF4E6
:10DBB000E1302B6A35609847012233682146C3E97A
:10DBC0000544DA751A766422DC619A770D4B0E22D1
:10DBD0001C700D4B0D481C605C60F2F737FD0C4B60
:10DBE0001C800C4B1C601C710B4B1C7070BD00BF6B
:10DBF0005CF10008A8250020A42D0020EC2D0020B9
:10DC0000D4250020AE250020B0250020BD25002011
:10DC1000AC250020B8250020642F00200048704764
:10DC200080F10008034BD8689B68C01A18BF012018
:10DC3000704700BFA42D002038B5184C002523786C
:10DC4000032B29D8DFE803F0020C16200A2314481E
:10DC500043708570FFF77EFF08B10123237038BD44
:10DC6000F6230F4845708370FFF774FF0028F6D045
:10DC70000223F3E7F6230A4843708570FFF76AFF33
:10DC80000028ECD00323E9E70A2305484570837098
:10DC9000FFF760FF0028E2D02570E0E7AF25002005
:10DCA000B825002007B501228DF807000DF1070106
:10DCB0000620FFF70FFF03B05DF804FB38B50446FC
:10DCC0000E4D0F4B286843F00103003018BF0120B0
:10DCD0009847601EC0B204280ED80A4A2B68125C0E
:10DCE00053F822402046F2F739FE2146BDE838407D
:10DCF00002460820FFF7EEBE002038BDA825002010
:10DD00005CF1000856F1000808B1FFF723BF704727
:10DD1000082202490120FFF7DDBE00BFB025002028
:10DD20000E2202490220FFF7D5BE00BFBD2500200C
:10DD30002DE9F74F984C80462068984E003046F009
:10DD4000010618BF01200F46B0472068944D0030EF
:10DD500018BF0120B0472368DFF86092186B0030CD
:10DD600018BF0120B0472368586A003018BF01204F
:10DD7000B04723681B6B984700283FD023685B6A35
:10DD8000984795F83220012A52D0002A47D0022A1B
:10DD900057D099F80030002B6FD0A854013B0132C6
:10DDA000D2B2DBB285F8322089F80030002BE0D106
:10DDB00019467B48013A914261D3AA5C9A425CD1F0
:10DDC0004AF66623ADF80430BB238DF8063023688D
:10DDD00003219B6A01A8984700226B7885F83220BE
:10DDE0005B2B52D05C2B00F089805A2B40F08A804C
:10DDF000EB7813F0F80F01D12268D3772068003058
:10DE000018BF0120B047674A13789146032B00F2F0
:10DE10009080DFE813F0DC007B00B100D5006628BD
:10DE200001D0AC28A5D10123287085F83230A0E7B5
:10DE30005A2822D35C2801D9AA281ED1687002234F
:10DE4000F3E7BB284FF0030310D12A782168662A34
:10DE5000A87085F832308CD16A78AA2A89D100223C
:10DE600085F832200A754F4A137082E7A870013096
:10DE700085F8323089F800007BE70023D5E710F8F9
:10DE800001CB01316344DBB295E7E978236832299D
:10DE900027D00FD822291DD004D82129AED10122A4
:10DEA0005A75ABE7232918D03129A7D1012119834D
:10DEB000DA77A3E735291AD006D8332915D03429C3
:10DEC0009CD101221A7799E7362914D0422995D19D
:10DED0001A7593E70122DA8290E75A754FF480723F
:10DEE000F9E74FF480721A8388E71A83E0E701218B
:10DEF00099765A76DCE70121D976FAE72368EA7841
:10DF00009A777BE70322274B1A7077E72368264D21
:10DF10005B6B98472B68984223685B6B27D39847C5
:10DF20002B68C01A214B1B78834202D2022389F846
:10DF30000030B8F1000F00F06881B8F1060F40F032
:10DF40006C81002F00F05381194C2378D90704D538
:10DF500023F001032370FFF7DBFE23789A0740F1DB
:10DF6000548123F002032370FFF7DAFE4DE1984756
:10DF70002B68DB431844D5E70E4A0F49137809781C
:10DF80000133DBB29942137003D200231370FFF701
:10DF90007DFD0023CBE700BFA82500205CF1000831
:10DFA0003C250020A42D0020602F00203C110020E3
:10DFB000AE250020CC2500203D110020CB250020DF
:10DFC000FFF764FD0023A24A89F800301370D9E9F5
:10DFD00002239342ADD0D3E900159E4B6D1A2A4619
:10DFE0001846F2F7BDFA8246002DA2D0206805F14E
:10DFF000FF3B003018BF0120B0471E229649974BC7
:10E000000A701A709AF800200C2A1DD8DFE812F066
:10E010000D00140044005C006C007A008200930044
:10E02000A500BC00C400CC00DB0005228C4B5A6369
:10E030008C4A1A6004201BE023681B7D33B1002248
:10E0400011461046FFF746FD032370E703230C2219
:10E050000B70834B0B205A6345F2AC121A800822D6
:10E0600081499A700A68C3F803204A68C3F80720F8
:10E07000FFF71EFD2368986A003018BF0120B047E3
:10E0800077482368818E9B6A984723685B6B984723
:10E09000764B186001234AE7032312220B70704B62
:10E0A0005A6345F2AC221A800E229A706E4A0333EC
:10E0B00002F10C0152F8040B8A4243F8040BF9D127
:10E0C000128811201A80D3E7032306220B70644BB9
:10E0D00005205A6345F2AC321A8002229A70BAF8CF
:10E0E0000120A3F80320C3E7032305220B705C4B38
:10E0F0005A6345F2AC421A8001229A709AF80120C4
:10E10000DA7097E7032305220B70554B5A6345F2EB
:10E11000AC52F0E70521524A9AF80100516345F2EA
:10E12000AC611180012153289170D07016BF10226C
:10E1300019701A707EE7032309220B70484B0820E0
:10E140005A6345F6AC021A8005229A70464A116855
:10E150001279C3F80310DA718AE745F6AC12DFF8DA
:10E1600000A10335CAF83450AAF8002010221A7012
:10E170005A463D498AF802B00AF10300F2F7F0F975
:10E18000DAF83400013873E7DFF8D4A00335CAF8B1
:10E19000345045F6AC32E7E7DFF8C4A00335CAF8DF
:10E1A000345045F6AC42DFE7DFF8B4A045F6AC5298
:10E1B000504620F8022B102202351A70CAF834504B
:10E1C0005A462949DAE70323254D6B634AF666234D
:10E1D0002B80BB23AB702368986A003018BF0120E6
:10E1E000B0472368A98E9B6A284698472CE7236886
:10E1F0001F4D5B6B98472B68984223685B6B07D376
:10E2000098472B6898427FF49FAE03B0BDE8F08F2B
:10E2100098472B68C01A0128F5E7154D27B12368E8
:10E220005B6B984728608FE623685B6B98472B6889
:10E23000984223685B6B05D398472B68C01A072860
:10E24000EDD8E2E798472B68DB430344072BF7E759
:10E25000CC250020B82D00203C1100203D110020CD
:10E2600070250020AC560100B92D0020602F002041
:10E27000D0250020022202490320FFF72BBC00BF5B
:10E28000AC250020012202490420FFF723BC00BF77
:10E29000642F0020244B08201A4610B513F8011BE8
:10E2A00091B3002313605360FFF732FD0120002378
:10E2B0001E4A12F8011B61B30E2200211B48F2F71F
:10E2C000C5F9FFF72DFD0120194B19785A780A433B
:10E2D00004D000221A80FFF7CDFF0120154A002349
:10E2E000114612F8014BCCB1002312480B600B71A0
:10E2F000FFF70AFD0120104B1A7822B100221A7094
:10E30000FFF7C0FF012010BD013810F0FF00C5D19C
:10E31000CDE70133DBB20E2BCBD1D5E70133DBB236
:10E32000052BDED1E7E700BFB0250020BD2500208A
:10E33000AC250020B8250020642F0020F8B5044645
:10E340001F464A4B4A4A186842F00102003018BF83
:10E3500001200D469DF818609047231FA02B43D83D
:10E36000444A022315B3D55CA5421AD03DB9D45412
:10E37000414A137843F0010313702846F8BD013376
:10E38000082BF0D16EB1E30804F0070101243B4AE9
:10E390008C40D15C0C43D454374A137843F00203C9
:10E3A00013700025E9E70133082B09D0D15CA142A5
:10E3B000F9D10021D154304A137843F0010313708E
:10E3C0002E48E108435C04F0070443FA04F2D20744
:10E3D000E7D5012202FA04F4274A23EA040343544E
:10E3E000137843F00203C7E7A4F1E00293B2072BCE
:10E3F00016D86DB10FB1E32C05D001231D49934010
:10E400000A7813430B701C4A137843F00103C7E7E3
:10E410000123184903FA02F20B7823EA0203F1E719
:10E42000A4F1A50083B2022B0FD801221449824027
:10E4300091F9003052B22DB11343DBB20B70FFF7EC
:10E4400021FFAEE723EA0203F7E7A4F1A8031A2BA2
:10E450000AD825B158340B4BE4B233F814500A4BA8
:10E460001D80FFF707FF9CE7012586E7A825002010
:10E470005CF10008B0250020AE250020BD2500205D
:0CE48000642F002020F10008AC250020D3
:10E48C004B4A494847464544434200FF440000007C
:10E49C000020202020202020202028282828282068
:10E4AC002020202020202020202020202020202060
:10E4BC0020881010101010101010101010101010C8
:10E4CC0010040404040404040404041010101010B8
:10E4DC001010414141414141010101010101010182
:10E4EC0001010101010101010101010110101010D4
:10E4FC001010424242424242020202020202020254
:10E50C0002020202020202020202020210101010A7
:10E51C0020000000000000000000000000000000CF
:10E52C0000000000000000000000000000000000DF
:10E53C0000000000000000000000000000000000CF
:10E54C0000000000000000000000000000000000BF
:10E55C0000000000000000000000000000000000AF
:10E56C00000000000000000000000000000000009F
:10E57C00000000000000000000000000000000008F
:10E58C00000000000000000000000000000000007F
:10E59C0000000000040C002000000000000000003F
:10E5AC00000000000000000000000000000000005F
:10E5BC00000000000000000000000000000000004F
:10E5CC00000000000000000000000000000000003F
:10E5DC00000000000000000000000000000000002F
:10E5EC00000000000000000000000000000000001F
:10E5FC00000000000000000081828300E200E900BE
:10E60C00EA00B500B600B700CD008301CC008A014A
:10E61C0092019401210223022402250226022702E0
:10E62C002A02B300B4006F0070009F01CB019F025F
:10E63C00A002000000000000C0D40100E093040020
:10E64C00C0270900804F120040771B0080EE360077
:10E65C0060EA00000D0A6B6579626F617264207666
:10E66C0065723A204B425F56455253494F4E000D4E
:10E67C000A636F7265207665723A20302E32322E24
:10E68C0031342D31372D676231326662662D646903
:10E69C007274790D0A000D0A6275696C64206461EC
:10E6AC0074653A20323032352D31302D33312D31E5
:10E6BC00363A30333A3030004A616E652042542D80
:10E6CC0031004A616E652042542D32004A616E65FC
:10E6DC002042542D33005742204B422034005742E5
:10E6EC00204B42203500000000080040010800408B
:10E6FC0002080040030800400500004004080040E8
:10E70C000508004000040040010400400A040040D9
:10E71C000B0400400C0400400D0400400E040040AB
:10E72C000708004008080040090800400948032178
:10E73C0081620C21C162084890F81003074900F06F
:10E74C000F000A68824200D008600020401C232879
:10E75C00FCDB70470000014000F0FF1F0404014087
:10E76C000748032181620C21C1620648016801F04F
:10E77C000F01082901D90821016000BF00BF7047B3
:10E78C000000014004040140030000400000004070
:10E79C000100004004000040020C00400F0000404B
:10E7AC000608004021522C00E200000029003A002B
:10E7BC003B003C003D003E003F0040004100420059
:10E7CC00430044004500137E4600470048003500D6
:10E7DC001E001F0020002100220023002400250021
:10E7EC00260027002D002E002A0049004A004B006D
:10E7FC002B0014001A000800150017001C0018004C
:10E80C000C00120013002F00300031004C004D00A2
:10E81C004E00390004001600070009000A000B0026
:10E82C000D000E000F0033003400320028000000F1
:10E83C0000000000E10064001D001B000600190030
:10E84C00050011001000360037003800E500870085
:10E85C00000052000000E000E300E20000000000B5
:10E86C002C002C0000000000E400E700E600215220
:10E87C000000500051004F0000000000000000009C
:10E88C00000000000000000000000000000000007C
:10E89C0089002800000000000000037CBD00BE00C1
:10E8AC00B100B300B500B200AC00AE00AB00A800E4
:10E8BC00AA00A90001000100010001000100007E76
:10E8CC00017E027E057E067E010001000100010032
:10E8DC00010001000100010001002378010001008A
:10E8EC0001000100010001000100010001004900CC
:10E8FC000100460001000100217801000100010027
:10E90C0001000100010001000100010001000100F3
:10E91C00010020780100010001000100000000004E
:10E92C0000000100010001000100010001000100D4
:10E93C000100147E01000100010001000100000033
:10E94C002778000001000B70010000000000077E1A
:10E95C00077E000000000100010001000100000022
:10E96C002A782878297800000000000000000000B8
:10E97C00000000000000000000000000000001008A
:10E98C0001000000000000002900BD00BE00520183
:10E99C002C082C085101AC00AE00AB00A800AA005A
:10E9AC00A900137E46004700480035001E001F00DA
:10E9BC00200021002200230024002500260027002F
:10E9CC002D002E002A0049004A004B002B00140099
:10E9DC001A000800150017001C0018000C0012008B
:10E9EC0013002F00300031004C004D004E00390058
:10E9FC0004001600070009000A000B000D000E00B1
:10EA0C000F0033003400320028000000000000002A
:10EA1C00E10064001D001B00060019000500110038
:10EA2C001000360037003800E50087000000520067
:10EA3C000000E000E200E300000000002C002C00CD
:10EA4C0000000000E400E700E60023520000500044
:10EA5C0051004F000000000000000000000000000A
:10EA6C0000000000000000000000000089002800E9
:10EA7C00000000000000037C3A003B003C003D001D
:10EA8C003E003F004000410042004300440045006E
:10EA9C0001000100010001000100007E017E027EE8
:10EAAC00057E067E0100010001000100010001004D
:10EABC000100010001002378010001000100157E16
:10EACC0001000100010001000100490001004600A5
:10EADC00010001002178010001000100010001008A
:10EAEC00010001000100010001000100010020787B
:10EAFC000100010001000100000000000000010005
:10EB0C0001000100010001000100010001000000F2
:10EB1C000100010001000100010000002778000045
:10EB2C0001000100010000000000077E077E0000CC
:10EB3C000000010001000100010000002A78287883
:10EB4C002978000000000000000000000000000018
:10EB5C0000000000000000000000010001000000A7
:10EB6C000000000081828300E200E900EA00B500A9
:10EB7C00B600B700CD008301CC008A01920194014C
:10EB8C002102230224022502260227022A02B300B4
:10EB9C00B4006F0070009F01CB019F02A002000027
:10EBAC000008004001080040020800400308004033
:10EBBC000500004004080040050800400004004027
:10EBCC00010400400A0400400B0400400C04004007
:10EBDC000D0400400E0400400708004008080040E7
:10EBEC000908004003000040000000400100004004
:10EBFC0004000040020C00400F00004006080040DA
:10EC0C00003131295A1B750A699300087593000865
:10EC1C00AD930008CD930008000101010101010131
:10EC2C0001010202020202020202020303030303B5
:10EC3C000303030404040404040405050505050684
:10EC4C000606060607070707070808080809090942
:10EC5C00090A0A0A0B0B0B0C0C0C0D0D0D0E0E0EEB
:10EC6C000F0F0F101011111112121313141415157C
:10EC7C0016161717181819191A1A1B1B1C1D1D1EEE
:10EC8C001E1F202021222223242425262627282942
:10EC9C00292A2B2C2D2D2E2F303132323334353670
:10ECAC003738393A3B3C3D3E3F4041424344454670
:10ECBC004748494A4C4D4E4F50515354555658594C
:10ECCC005A5B5D5E5F616264656668696B6C6D6FF3
:10ECDC007072737577787A7B7D7E80828385878866
:10ECEC008A8C8E8F91939596989A9C9EA0A2A3A5A0
:10ECFC00A7A9ABADAFB1B3B5B7BABCBEC0C2C4C6A1
:10ED0C00C9CBCDCFD1D4D6D8DBDDDFE2E4E7E9EB5C
:10ED1C00EEF0F3F5F8FAFDFF000000000000000033
:10ED2C0000000000000000000000000000000000D7
:10ED3C0000000000000000000000000000000000C7
:10ED4C002A2B28000000000000000000000000003A
:10ED5C0000000029000000002C1E34202122243445
:10ED6C002627252E362D3738271E1F202122232417
:10ED7C0025263333362E37381F0405060708090AB3
:10ED8C000B0C0D0E0F101112131415161718191A4F
:10ED9C001B1C1D2F3130232D350405060708090ACD
:10EDAC000B0C0D0E0F101112131415161718191A2F
:10EDBC001B1C1D2F3130354C000000007E0F00D481
:10EDCC00FFFFFFC7000000780300000000000000F8
:10EDDC0039AD000800000000080000007823002076
:10EDEC000000000002000000000000000300000012
:10EDFC000000000039AD00080000000020000000F9
:10EE0C00D4230020000000000200000000000000DD
:10EE1C00E1AD00086DAD000839AF0008C5AD0008C4
:10EE2C0008EF00080CEF000812EF000804040A00B9
:10EE3C0069EE000882EE0008A2EE0008C4EE00089D
:10EE4C001EEF000840EF00084422B609025B0003E5
:10EE5C000100A0FA090400000103010100092111BD
:10EE6C000100012244000705810308000109040187
:10EE7C0000020300000009211101000122220007F9
:10EE8C00058203200001070502032000010904028A
:10EE9C0000010300000009211101000122B6000746
:10EEAC0005830320000112010002000000401361E1
:10EEBC00011000010102000105010906A10105076D
:10EECC0019E029E7150025019508750181029501C6
:10EEDC00750881010507190029FF150026FF00950B
:10EEEC0006750881000508190129051500250195ED
:10EEFC000575019102950175039101C00403090484
:10EF0C000403200000000A034A0061006E00650043
:10EF1C0000000660FF0961A1010962150026FF00CF
:10EF2C009520750881020963150026FF0095207550
:10EF3C00089102C005010902A10185020901A10085
:10EF4C00050919012908150025019508750181028B
:10EF5C000501093009311581257F95027508810657
:10EF6C0009381581257F950175088106050C0A382D
:10EF7C00021581257F950175088106C0C005010920
:10EF8C0080A101850319012AB700150126B7009548
:10EF9C000175108100C0050C0901A101850419013E
:10EFAC002AA002150126A002950175108100C0054A
:10EFBC00010906A1018506050719E029E7150025B9
:10EFCC00019508750181020507190029EF15002527
:10EFDC000195F07501810205081901290595057542
:10EFEC00019102950175039101C000000000000021
:10EFFC0055B4000845B4000875B4000865B40008A1
:10F00C006FB400085FB400084FB400083FB40008A8
:10F01C0000000000ACF7000894330020943300206B
:10F02C0094330020ACF70008000000000000000042
:10F03C0000000000ACF70008000000000000000019
:10F04C0000000000ACF70008000000000000000009
:10F05C0000000000ACF700080000000000000000F9
:10F06C0000000000ACF700080000000000000000E9
:10F07C0000000000ACF700080000000000000000D9
:10F08C0000000000ACF700080000000000000000C9
:10F09C0000000000ACF00008102400202025002007
:10F0AC006330006D61696E0069646C65000000007E
:10F0BC000000000081C3000871C30008A1C3000850
:10F0CC0091C300089BC300088BC300087BC30008D6
:10F0DC006BC30008ABC3000800000100000065789A
:10F0EC006974006B696C6C000096000003000000F2
:10F0FC0000000000CDC70008A9D4000829D30008DF
:10F10C0040004000202500202025002001000000A8
:10F11C0034250020E200E900EA00B500B600B70093
:10F12C00CD008301CC008A019201940121022302BB
:10F13C0024022502260227022A02B300B4006F0023
:10F14C0070009F01CB019F02A0020001020304008A
:10F15C000549D1F80012054A114010B1044881420A
:10F16C0000D0FEE77047000000F0FF1FFF3F00F0EB
:10F17C0080290030627473206C69622078746B2073
:10F18C0076657273696F6E3A2076312E352E3400A7
:10F19C005245454E54206D616C6C6F6320737563E2
:10F1AC0063656564656400002E2E2F2E2E2F2E2E87
:10F1BC002F2E2E2F2E2E2F2E2E2F2E2E2F2E2E2F5D
:10F1CC006E65776C69622F6C6962632F7374646C03
:10F1DC0069622F72616E642E630000002C206675CC
:10F1EC006E6374696F6E3A20000000006173736582
:10F1FC007274696F6E2022257322206661696C65BA
:10F20C00643A2066696C6520222573222C206C6977
:10F21C006E65202564257325730A0000232D302B81
:10F22C0020000000686C4C0065666745464700008E
:10F23C003031323334353637383941424344454620
:10F24C0000000000303132333435363738396162E2
:08F25C00636465660000000018
:08F26400B80FFF7F010000005C
:10F26C00040C002000000000E4E50008C4E50008E0
:10F27C00A4E50008000000000000000000000000F1
:10F28C000000000000000000000000000000000072
:10F29C000000000000000000000000000000000062
:10F2AC000000000000000000000000000000000052
:10F2BC000000000000000000000000000000000042
:10F2CC0000000000C4E60008CEE60008D8E60008FE
:10F2DC00E2E60008EAE6000800000000000000007A
:10F2EC000000000011AB00085DAB000871AB00081A
:10F2FC0085AB000899AB0008FDA9000800000000D0
:10F30C000000000000000000CD260008613300085A
:10F31C0085330008F92300083D27000869220008FE
:10F32C0000000000B80B0000007E00000000000090
:10F33C00B80B0000017E000000000000B80B0000BC
:10F34C00027E000000000000B80B0000037E0000ED
:10F35C0000000000B80B0000047E0000000000005C
:10F36C00B80B0000057E000000000000B80B000088
:10F37C00437E000000000000B80B0000037C00007E
:10F38C0000000000B80B0000117E0000000000001F
:10F39C00B80B0000127E000000000000B80B00004B
:10F3AC00137E00004D4E4F505152535455565758E2
:10F3BC00595A5B5C5D4C4B4A49484746454443426D
:10F3CC0041403E3D3C3B292A2B2C2D2E2F303132F7
:10F3DC003334353638393A28272625242322212060
:10F3EC001F1E1D1C1BFFFFFF0D0E0F1011121314FF
:10F3FC0015161718191AFF00FF0C0B0AFFFF090846
:10F40C00FFFF07060504FF030201FFFFFFFFFFFFDD
:10F41C00FFFFFFFFFFFF3F37FFFFFFC734D440C79D
:10F42C0040BB40AA409B408C407C4050403C40201C
:10F43C004011400240083410341C34283434344019
:10F44C00344D345934653472347E348A34A134A446
:10F45C0034A4289E289028842878286B285F285369
:10F46C002847283A282E28222815280528031B125D
:10F47C001B1F1B2B1B371B441B501B5C1B681B755A
:10F48C001B811B8D1B991BA91BA91BBB1BC71BD449
:10F49C001BD40FC70FBB0FA60F9E0F930F870F7BAD
:10F4AC000F6E0F620F560F4A0F3D0F310F250F19BC
:10F4BC000F0C0F000F00000F001C0028003400443C
:10F4CC000050005C0068007800840090009C00AC48
:10F4DC0000BB00C700D400D40004040404010401E0
:10F4EC0001040401010101010404040404040404E2
:10F4FC0004040101040404040404040404040404C6
:10F50C0004040404040404040404040404040404AF
:10F51C00040404040404040404040404040404049F
:10F52C00040404040404040404040404040404048F
:10F53C000404040404040404FA00000000000000A5
:10F54C0001000000000000004B0000003D3C0008E2
:10F55C00FF000000FA0000000000000001000000A5
:10F56C00000000004A0000003D3C0008FF000000C5
:10F57C00FA00000000000000010000000000000084
:10F58C00490000003D3C0008FF000000FA000000AC
:10F59C000000000001000000000000004800000016
:10F5AC003D3C0008FF000000FA00000000000000D5
:10F5BC000100000000000000470000003D3C000876
:10F5CC00FF000000FA000000000000000100000035
:10F5DC00000000005E000000A53E0008FF000000D7
:10F5EC00FA00000000000000FF0000000000000016
:10F5FC00FF00000000000000000000000000000000
:10F60C0000000000000000000000000000000000EE
:10F61C000000000000000000B0E70008007C0000C3
:10F62C0000000000FA160020355E000801140A1EC6
:10F63C000150082800FF00FFFF03390501030102F8
:10F64C000096000003000000FFFFFFFF0400000015
:10F65C00040000000000000000000000000000009A
:10F66C00000000000000000000000000000000008E
:10F67C00000000000000000000000000000000007E
:10F68C00000000000000000000000000000000006E
:10F69C00030000000000000063B60008D9B60008A3
:10F6AC00200020000000000000000000020000000C
:10F6BC0000000000030000000000000017B7000865
:10F6CC000000000008000000000000000000000026
:10F6DC0002000000000000001833002002020000AD
:10F6EC0004000000040000002000000020000000C6
:10F6FC000000000050220020E0220020000000004A
:10F70C0000000000000000000000000000000000ED
:10F71C0000000000000000000000000000000000DD
:10F72C0000000000000000000000000000000000CD
:10F73C0000000000000000000000000000000000BD
:10F74C0000000000000000000000000000000000AD
:10F75C00000000000000000000000000000000009D
:10F76C00000000000000000000000000000000008D
:10F77C00000000000000000000000000010000007C
:10F78C0005B2000861B20008A5B20008C5B20008B5
:10F79C00009600000000080000A24A041E1E000093
:04000005080001B935
:00000001FF
